:020000040800F2
:10000000888C0120E5020008ED020008EF020008DC
:10001000F1020008F3020008F502000800000000E9
:1000200000000000000000000000000025030008A0
:10003000F902000800000000BD030008CD0300081D
:10004000FF020008FF020008FF020008C92900089B
:10005000FF020008FF020008FF020008FF0200087C
:10006000FF020008FF020008FF020008FF0200086C
:10007000FF020008FF020008FF020008A129000893
:10008000FF020008FF02000869290008FF020008BB
:10009000FF020008FF020008FF020008FF0200083C
:1000A000FF020008FF020008FF020008FF0200082C
:1000B000FF020008FF020008FF020008FF0200081C
:1000C000FF020008FF020008FF020008212A0008C2
:1000D0004D2A0008552B0008FF020008FF02000807
:1000E000FF020008FF020008FF020008FF020008EC
:1000F000FF020008FF020008FF020008FF020008DC
:10010000FF020008FF020008FF020008FF020008CB
:10011000FF020008D12A0008FF020008FF020008C1
:10012000FF020008FF020008FF020008FF020008AB
:10013000FF020008FF020008FF020008FF0200089B
:10014000FF020008FF020008FF020008FF0200088B
:10015000FF020008FF020008FF020008FF0200087B
:10016000FF020008FF020008FF020008FF0200086B
:10017000FF020008FF02000800000000000000006D
:10018000FF020008FF020008FF020008FF0200084B
:10019000FF020008FF02000800000000FF02000844
:1001A000FF020008FF02000800000000000000003D
:1001B000FF0200080000000000000000FF0200082D
:1001C000FF020008FF020008FF020008FF0200080B
:1001D000FF020008FF02000800F002F800F06FF8CC
:1001E0000AA090E8000C82448344AAF10107DA4592
:1001F00001D100F064F8AFF2090EBAE80F0013F075
:10020000010F18BFFB1A43F001031847A04E00006E
:10021000D04E00000A444FF0000C10F8013B13F0E0
:10022000070408BF10F8014B1D1108BF10F8015B4F
:10023000641E05D010F8016B641E01F8016BF9D142
:1002400013F0080F1EBF10F8014BAD1C0C1B09D199
:100250006D1E58BF01F801CBFAD505E014F8016B0B
:1002600001F8016B6D1EF9D59142D6D3704700009D
:10027000103A24BF78C878C1FAD8520724BF30C8D2
:1002800030C144BF04680C607047000000230024A4
:1002900000250026103A28BF78C1FBD8520728BF96
:1002A00030C148BF0B607047752900F0FF80002007
:1002B00070471FB504F08DFC1FBD10B510BD00F0D8
:1002C00042FC114603B402F0D4FC03BCFFF7F1FF7B
:1002D00004F0A8FA00F05CFC03B4FFF7EEFF03BCE7
:1002E00000F064FC0948804709480047FEE7FEE744
:1002F000FEE7FEE7FEE7FEE7FEE7FEE7FEE7FEE7D6
:1003000004480549054A064B704700006D2A00085D
:10031000D901000888860120888C01208888012066
:10032000888801201EF0040F0CBFEFF30880EFF364
:100330000980816911F8021C91BB01B590E80F108A
:10034000E047BDE800508CE80300244B93E806002A
:10035000914208BF704741B91EF0100F10D12049DB
:10036000086820F0010008600AE02CE9F00F1EF098
:10037000100F08BF2CED108AC1F838C081F822E0B8
:100380001A6092F82210906B61F0FF0E1EF0100FB1
:1003900008BFB0EC108AB0E8F00F80F3098870470E
:1003A000104A13689942FAD801B552F821C00FC813
:1003B000E047BDE80050CCF80000704701B500F000
:1003C000E7FFBDE80140EFF3098CBEE701B501F09E
:1003D00049FABDE80140EFF3098CB6E79409012022
:1003E00034EF00E0E84F0008B2F120030AD5C2F173
:1003F000200301FA02F120FA03F300FA02F041EAC5
:100400000301704700FA03F14FF000007047B2F1AA
:1004100020030AD5C2F1200320FA02F001FA03F307
:1004200021FA02F140EA0300704721FA03F04FF08D
:10043000000170470FB41CB5074B06AA7B44694600
:100440000090059800F067FB0020694600F076FBFD
:100450001CBC5DF814FB0000FD06000070B50446EE
:1004600085690068C10601D5302600E02026C00756
:1004700007D070BDD4E9012130469047206A401C66
:1004800020626D1EF6D570BD70B504468569007892
:10049000C00707D170BDD4E9012120209047206A10
:1004A000401C20626D1EF6D570BD00002DE9F041A4
:1004B0000646002410687529314616A510D0AFF302
:1004C0000080002802DA404213A507E031688A075D
:1004D00001D512A502E0490704D511A5012401E0C8
:1004E000AFF3008000210A2206F1240709E0B0FBE7
:1004F000F2FCB0FBF2F302FB1C00303078541846DB
:10050000491C0028F3D123462A463046BDE8F04175
:1005100000F0A3BA000000002D0000002B00000036
:10052000200000002DE9F05F894604464FF0000AE4
:10053000DFF874B1FB44C0F820A02046E16888478A
:10054000002874D0252806D0D4E901219047206ADC
:10055000401C2062F1E700265F462046E16888479C
:100560002028054607DB312D05D2781910F8200C1C
:1005700008B10643F1E7B00701D526F00406C4F838
:100580001CA00027C4F818A02A2D09D0284602F084
:100590003EFB38B304EB8708303DC8F8185019E02B
:1005A00059F8041B204604EB87029161E1688847F3
:1005B000012F054618D1E069002820DA26F0200630
:1005C0001DE0D8F8180000EB800005EB4000303843
:1005D000C8F818002046E1688847054602F017FB76
:1005E0000028EED1012F0AD02E2D08D12046E16837
:1005F00088477F1C0546022F46F02006C4DBA06911
:10060000002803DA404246F00106A061F00701D05D
:1006100026F010066C2D0BD0682D09D04C2D39D04A
:100620006A2D35D0742D35D07A2D33D016E038E0D0
:10063000E1682F4620468847B842054609D16C2F0D
:1006400026D04FF48060E16806432046884705467F
:1006500004E06C2F1AD04FF4807006430DB3A5F15F
:100660004100192802D8203546F400664A4629463A
:10067000204626604E46FFF717FE80B101280BD0BA
:10068000F61D26F0070000F1080956E74020E4E7D0
:100690008020D8E70020D6E706F104094DE7284678
:1006A00052E7206ABDE8F09FB54A000010B5431E2E
:1006B00013F8014F002CFBD105E011F8014B002C81
:1006C00003F8014B03D0521EF7D20021197010BD60
:1006D00040EA010310B59B070FD1042A0DD310C8BF
:1006E00008C9121F9C42F8D020BA19BA884201D911
:1006F000012010BD4FF0FF3010BD1AB1D30703D059
:10070000521C07E0002010BD10F8013B11F8014B0E
:100710001B1B07D110F8013B11F8014B1B1B01D12A
:10072000921EF1D1184610BD40EA0103024630B5D1
:100730009B0710D14FF0013400E008C208C91D1B0F
:100740009D4315EAC41FF8D013F0FF0102F8011B06
:100750000DD01B0AF8E711F8013B002B02F8013B12
:1007600005D011F8013B002B02F8013BF3D130BD5D
:1007700010B5431C02E010F8011B71B18107FAD1DA
:100780004FF0013202C88C1A8C4314EAC211F9D01E
:10079000C01A0A0603D0C01E10BDC01A10BD0A043C
:1007A00001D0801E10BD0902FCD0401E10BD40EAE1
:1007B000010370B59B072ED14FF00136042A2AD3CE
:1007C00008C810C99D1B9D43121F15EAC61517D0F6
:1007D000D8B2E1B2401A50EA056110D198B2A1B284
:1007E000401A50EA05410AD123F07F4024F07F41AE
:1007F000401A50EA052102D1180EA0EB146070BD1A
:10080000A342DBD018BA21BA884201D9012070BDB9
:100810004FF0FF3070BD0AB9002070BD10F8013BE9
:1008200011F8014B63B1A3420AD1521E08D010F84F
:10083000013B11F8014B1BB1A34201D1521EEDD176
:10084000181B70BD032A40F2308010F0030C00F03A
:10085000158011F8013BBCF1020F624498BF11F8FA
:1008600001CB00F8013B38BF11F8013BA2F10402B3
:1008700098BF00F801CB38BF00F8013B11F003032B
:1008800000F02580083AC0F0088051F8043B083A8F
:1008900051F804CBA0E80810F5E7121D5CBF51F831
:1008A000043B40F8043BAFF30080D20724BF11F8AB
:1008B000013B11F801CB48BF11F8012B24BF00F810
:1008C000013B00F801CB48BF00F8012B704710B581
:1008D000203AC0F00B80B1E81850203AA0E8185038
:1008E000B1E81850A0E81850BFF4F5AF5FEA027CF9
:1008F00024BFB1E81850A0E8185044BF18C918C068
:10090000BDE810405FEA827C24BF51F8043B40F808
:10091000043B08BF7047D20728BF31F8023B48BFED
:1009200011F8012B28BF20F8023B48BF00F8012B2B
:10093000704702F0FF0343EA032242EA024200F05A
:1009400002B84FF000020429C0F0128010F0030C2E
:1009500000F01B80CCF1040CBCF1020F18BF00F8B2
:10096000012BA8BF20F8022BA1EB0C0100F00DB861
:100970005FEAC17C24BF00F8012B00F8012B48BFBF
:1009800000F8012B70474FF0000200B51346944663
:100990009646203922BFA0E80C50A0E80C50B1F1D7
:1009A0002001BFF4F7AF090728BFA0E80C5048BFEB
:1009B0000CC05DF804EB890028BF40F8042B08BF89
:1009C000704748BF20F8022B11F0804F18BF00F885
:1009D000012B70474FF0013C50F8042B51F8043BB9
:1009E0009A4221D1A2EB0C03934313EACC1317D103
:1009F00050F8042B51F8043B9A4215D1A2EB0C039A
:100A0000934313EACC130BD150F8042B51F8043B59
:100A10009A4209D1A2EB0C03934313EACC13DBD027
:100A20004FF00000704700BFD01A01BAB1FA81F14F
:100A300001F0180122FA01F0CB40C1F12001DBB234
:100A4000C0B2C01A2CFA01F3D11A914311EAC311B2
:100A5000E6D170477047704770472DE9F0470D4663
:100A600099469246044600F124080168880604D598
:100A7000E06921F01001216000E00120A84201DDC1
:100A8000471B00E00027A1697A1902EB0900081A48
:100A9000A0612078C00602D42046FFF7DFFC0026C4
:100AA00008E0D4E901211AF806009047206A401CAA
:100AB000761C20624E45F4DB2078C0060AD520461D
:100AC000FFF7CCFC06E0D4E9012130209047206AF2
:100AD000401C2062381EA7F10107F4DC07E0D4E9CE
:100AE000012118F805009047206A401C2062281E4A
:100AF000A5F10105F3DC2046FFF7C6FC20780006CF
:100B000002D50220BDE8F0870120FBE701694A1CFD
:100B100002610878704700B58FB0CDE9013100213E
:100B2000059105497944CDE9031011466846FFF760
:100B3000F9FC0FB000BD0000E5FFFFFF0A6802F8F6
:100B4000010B0A607047754600F02CF8AE460500B0
:100B50006946534620F00700854618B020B5FFF7D8
:100B6000CFFBBDE820404FF000064FF000074FF0EC
:100B700000084FF0000B21F00701AC46ACE8C009BB
:100B8000ACE8C009ACE8C009ACE8C0098D467047C4
:100B900010B50446AFF300802046BDE81040FFF7D3
:100BA0009BBB0000004870472486012001491820A3
:100BB000ABBEFEE726000200704710B500F1280129
:100BC00051E8002F12B9BFF32F8F04E0531E41E804
:100BD000003404B1F4E782B12C3001210AE0821C18
:100BE000D2E84F3FC2E8441F04B1F9E71A0608BF34
:100BF00010BD083000680028F1D1002010BD10B5EC
:100C000084465CF8303F8BB1CA784FF0000E05E0A7
:100C10001C46DB7893420ED26368A646002BF7D1C0
:100C20000022C1E9012E00F12C0208E00022C1E9F6
:100C30000122C16209E0C1E9014E04F1080211601C
:100C4000BEF1000F18BF0EF1040CCCF800102830D4
:100C500050E8001F4A1C40E8002303B1F8E710BD2C
:100C6000D1E90123002A0EBFC36293608B68191D6E
:100C7000002B08BF00F130010A607047014800688E
:100C8000704700BF10E000E007480178012905D156
:100C90000021017005484FF080610160044801683F
:100CA00041F00101016070478486012004ED00E0FD
:100CB00010E000E0024801684068081A704700BF71
:100CC00014E000E04FF0FF3070470000014800687A
:100CD0000130704714E000E002480068C0F30040B3
:100CE000704700BF10E000E040B10B490968B1FB5C
:100CF000F0F0411E0020B0EB116F02D04FF0FF303A
:100D00007047064AFF231370054A0623136051609B
:100D10000449906008707047D005012023ED00E081
:100D200010E000E08486012010B5930712D400F192
:100D30002803D00718D153E8000F084203D1BFF3AE
:100D40002F8F002005E020EA010243E8002404B1CF
:100D5000F1E710BD806AD20700EA010315D1002B2C
:100D600018BF10BD002010BD53E8000F00EA0102BB
:100D70008A4203D0BFF32F8F002005E020EA010252
:100D800043E8002404B1EFE710BD8B4218BF0020F8
:100D900010BD000080B5124A4FF0000E02F1440C65
:100DA000624606E01A6991420BD3891A03F10C02DC
:100DB0009E461368002BF5D10022C0E902E20161D2
:100DC00006E0C0E902E3016198601A69511A1961ED
:100DD000BEF1000F18BF0EF10C0CCCF8000080BD66
:100DE00080090120C16829B102690B691A440A61AE
:100DF00082688A608068044A00F10C03002808BFFA
:100E000002F144031960704780090120EFF3058166
:100E100029B9EFF3108111B9EFF3118111B16FF01E
:100E200005007047DFF804C000DF7047D51B0008DD
:100E3000EFF3058048B9EFF3108030B9EFF311807C
:100E400018B9EFF31480C00702D10448007A704744
:100E5000DFF804C000DF7047E91B000880090120AB
:100E6000EFF3058028B9EFF3108010B9EFF311808C
:100E700008B100F0BFBEDFF808C000DF704700BF58
:100E8000F51B0008EFF3058028B9EFF3108010B9C7
:100E9000EFF3118010B10348C0687047DFF808C055
:100EA00000DF7047800901201D1C000880B500F09C
:100EB00003F9EFF3058028B9EFF3108010B9EFF3D1
:100EC000118010B16FF0050080BDDFF808C000DFB1
:100ED00080BD00BF291C0008EFF3058028B9EFF39F
:100EE000108010B9EFF3118010B16FF0050070475A
:100EF000DFF804C000DF70477D1D0008EFF30580B8
:100F000028B9EFF3108010B9EFF3118010B16FF032
:100F100005007047DFF804C000DF70479D1D000822
:100F2000F8B50546EFF3058014460E4628B9EFF3F1
:100F3000108010B9EFF31180F0B16FF003000DB322
:100F400003BBFEB12978FA291CD12846FFF735FEEC
:100F500078B16A6A074600F10C013046FFF772FC6F
:100F60000CB1F87820703846FD6000F059FA002086
:100F700008E06FF0020005E02846DFF80CC03146BB
:100F8000224600DF01B0F0BD251E0008EFF3058307
:100F90002BB9EFF3108313B9EFF311830BB10020DA
:100FA0007047DFF808C000DF704700BF051F00086A
:100FB0002DE9F0410646EFF3058090460D4628B92D
:100FC000EFF3108010B9EFF3118018B36FF003073F
:100FD000EEB1E3B9DDB13078FA2818D106F10C0092
:100FE00000F0EFF888B1726A04460C302946FFF72A
:100FF00029FC0027F920C4E9015684F80380A77072
:101000002070204600F00CFA01E06FF0020738462D
:10101000BDE8F0813046DFF80CC02946424600DFCB
:10102000BDE8F08139200008EFF305822AB9EFF31B
:10103000108212B9EFF3118212B16FF00500704700
:10104000DFF804C000DF7047F9200008EFF30581E6
:1010500029B9EFF3108111B9EFF3118111B16FF0DC
:1010600005007047DFF804C000DF704789210008E1
:10107000EFF3058129B9EFF3108111B9EFF3118175
:1010800009B100207047DFF808C000DF704700BFDB
:101090004D220008EFF3058129B9EFF3108111B952
:1010A000EFF3118111B16FF005007047DFF804C054
:1010B00000DF7047B92200087047B0B50023D0B3F5
:1010C000C9B3032A37D886460F315EF8084F21F09E
:1010D000070CDEF804102346A4EB0E0421F00305F0
:1010E000641B644505D21C689E46002CF1D1002388
:1010F00021E0D0E9004363444360204450F8044CAD
:101100009C423EBF08384360DEF8041069B1DEF847
:10111000000021F0030141F80E004CEA0200714486
:101120004860CEF800108E4603E04CEA0200CEF88C
:1011300004000EF108031846B0BD80B5002218B3B4
:1011400011B300F10803A1F1080C4FF0000E634544
:1011500006D01A461B689646002BF8D1002213E0F1
:1011600051F8043C4268BEF1000F23F00303A2EBE8
:10117000030242604FF0010219BFDCF80000CEF814
:101180000000002041F8040C104680BD08B1420761
:1011900002D000221046704700221829FAD311F01D
:1011A0000703F7D11022C0E900120144A1F108039E
:1011B0008360002341F8083C81684A600122C360D3
:1011C000E8E710B5002817D0014600F1140252E8F4
:1011D000000F10B9BFF32F8F04E0036842E800341A
:1011E00004B1F4E740B1043151E8002F531C41E849
:1011F000003404B1F8E710BD002010BD00281FD056
:10120000C2688A421CD802698A4219D9B0B500F175
:10121000140213680B60BFF35F8F52E8003F0C6845
:101220009C42F6D142E8001505B1F2E7043050E8DF
:10123000001F4A1E40E8002303B1F8E70020B0BDBC
:101240006FF00300704784460020BCF1000F18BF08
:1012500000291AD0CAB1C3B180B54FF0000E02FB0D
:101260000130CCE9001ECCE90223CCE90403C1F132
:101270000100BDE8804003E09918013019600B4679
:101280000028F9D10020186001207047F8B5044605
:10129000807868B3E56821462846FFF7E1FC002026
:1012A00005F10C06214620703046FFF7A7FFA8681D
:1012B000E8B13046FFF785FFC8B10446284600F084
:1012C000F7F9002100220646002700F0B1FA304667
:1012D00000F04AFA81686A6A064604F10C00FFF7DA
:1012E000B1FAF920A7702070F068E07025E0F8BD31
:1012F000A568A86808B3407883281ED1284600F066
:10130000D7F9002100220646002700F091FA304666
:1013100000F02AFA064680686A6A04F10C01FFF7B9
:1013200091FAF06808B1E1780170277005F10C00BE
:101330002146BDE8F840FFF761BF28462146BDE8D9
:10134000F840FFF75CBC2DE9F041044600274FF060
:10135000010819E025466469E878000714D52F765E
:10136000A86888B1284600F0A3F9002100220646AB
:1013700000F05EFAC5E90367F06A0028686100D0F2
:101380000561F56285F81880002CE3D1BDE8F08195
:1013900070B5224C04F1560504F15A0628E0D6E84F
:1013A0005F1F4A1C904200D80022C6E8532F03B1A9
:1013B000F5E788B2E16D51F82000002828D00178C7
:1013C000F139082914D8DFE801F005130813130BCD
:1013D0000E131100216E88470AE0616E884707E00E
:1013E000A16E884704E0E16E884701E0216F8847DD
:1013F000B4F85400D5E85F1F11B9BFF32F8F04E094
:101400004A1EC5E8532F03B1F4E709047FF4C7AFC0
:101410000020BDE8704000F0F1B800BF8009012055
:1014200070B501461948B0F8542000F15603D3E8CE
:101430005F4FA24202D8BFF32F8F04E0651CC3E8C0
:10144000565F06B1F3E7A3B293421AD200F15803F4
:10145000D3E85F4F651CAA4200D80025C3E8565F59
:1014600006B1F5E7A2B2C36D43F82210417A002914
:1014700019BF0121817206484FF0805108BF0160F9
:1014800070BD0220BDE8704003F044BA800901201D
:1014900004ED00E010B58168B1B100F10C01D1E8B4
:1014A0005F2F12B9BFF32F8F04E0531EC1E8543FE2
:1014B00004B1F4E7110407D000F0FAF8002100228B
:1014C000BDE8104000F0B4B910BD0000012141702A
:1014D0000B4990F920C001F11C02114692684AB1F3
:1014E00092F920306345F8DCC0E90221886002F1FE
:1014F0000C0103E00022C0E90221083108607047B6
:101500008009012010B54A1C11D01F4A002402F1A5
:101510002C0C624603E0891A03F110021C46136882
:10152000E3B1DA699142F6D24FF0010E18E01649A4
:10153000002301F1300421461A460B6803F1100123
:10154000002BF9D14FF0FF31002AC1614FF00001AB
:10155000C0E9041216D002F1100413E04FF0000E9F
:10156000002CC0E90434C16118BF04F1100CCCF8A0
:101570000000BEF1000F08BF10BDDA6903F11404CA
:10158000511AD961206010BD80090120C26901692A
:10159000531C0AD021B1CB691A44CA6142694A611D
:1015A00042693AB90748C162704709B142694A6164
:1015B00042691AB11161002141617047014801631C
:1015C000704700BF80090120B0B50B4DEC6A1CB11B
:1015D000E0690138E06100D0B0BD204600F087F836
:1015E000204600F0B7F8246924B1E0690028F4D05F
:1015F00000206061EC62B0BD80090120B0B50546F5
:101600001448002D4469017A0CD0022905D194F9BF
:10161000200095F92010814212DC2846BDE8B04038
:1016200000F098B8022913D1456A8DB194F92000D1
:1016300095F920108142D8BFB0BD284600F057F878
:101640002046FFF743FF2846BDE8B04000F0CAB887
:10165000B0BD00BF8009012010B5044600202080E5
:10166000A07881070DD5C00605D41048216B406FC6
:10167000FFF763FD05E00D48216BD0F88400FFF70C
:10168000BDFDA078C00708BF10BD0849D1F888008B
:1016900020B12146BDE81040FFF7B0BDD1F8800071
:1016A0002146BDE81040FFF748BD00BF800901207A
:1016B000014680688268002A8A6000D0D1600021DB
:1016C000C160704791F920C00246806840B190F92E
:1016D00020306345F8DAC1E902020C30916004E081
:1016E0000020C1E9020202F1080001607047C168F0
:1016F00031B182688A60826802B1D1600021C16024
:101700007047B0B50446054603E02878F12803D1B8
:10171000ED68002DF9D1B0BD2046FFF7E8FF28465F
:101720002146BDE8B040FFF7CDBF10B50446407874
:10173000332818BF10BD94F82320616A2046FFF7B4
:10174000F3FA30B1014620460022BDE8104000F017
:101750006FB810BD01460120487002481C30FFF7E9
:10176000B1BF00BF8009012090F82210C9064FF0D8
:10177000200158BF6021806B0844704707484169C9
:1017800039B1086B8A6B824204D90068044A9042DE
:1017900000D17047012003F0BDB800BF80090120CF
:1017A000A52E5AE270B50B4C0B480021A26D666E57
:1017B00000F0C8FE094D002EA86209D0E26D08486D
:1017C000002100F0BFFEA864002818BF012070BDF2
:1017D000012070BD00500008354900088009012033
:1017E000D51800080221417001498861FFF7C6BF82
:1017F0008009012010B50D4C02460020237A022BEF
:1018000012D1636A83B160694270FFF77BFE606A40
:1018100081680029616202D004F11C02CA600021C3
:10182000C160FFF7DFFF012010BD00BF800901206C
:10183000B0B5044690F822001546C0064FF02000CF
:1018400058BF6020A26B81502046FFF79FFE2046C4
:101850001DB1BDE8B040FFF7D1BEBDE8B040FFF715
:1018600079BF0000B0B5FFF709FA194DE968286D96
:1018700001310028E96000D08047FFF7A5FE002075
:10188000FFF7BCFE296C11B3AA69A86B90421CBF7C
:10189000C5E90E21B0BDE96B11B10139E96316D17B
:1018A000297A022913D16C6A8CB190F8200094F83F
:1018B000201081420BD12046FFF719FFA86BFFF7DC
:1018C00049FF2046FFF78EFF286CC5E90E40B0BDEA
:1018D0008009012082B00B480821D0E91820FFF7C9
:1018E00055FB094D09496C46C5E913012146002203
:1018F0004FF0FF33FFF714FB10B9DDE90010884704
:10190000E86CF3E700500008800901201119000875
:1019100070B5144D6C6C1CB3206901260138206130
:101920001CE02069E0B9E06808B1A16881606864E2
:1019300004F1180100220023E86CFFF739FB18B10D
:101940000320214602F0E6FFE078012804D1616916
:101950002046FFF71FFA00E066706C6C002CE0D1A7
:1019600070BD00BF80090120EFF305822AB9EFF3B3
:10197000108212B9EFF31182CAB16FF00302A0B165
:1019800099B90178F62910D10C30D0E85F1F11B950
:10199000BFF32F8F04E04A1EC0E8532F03B1F4E7D2
:1019A0000022080408BF6FF0020210467047DFF8FB
:1019B00008C000DF704700BF71230008EFF3058106
:1019C00029B9EFF3108111B9EFF3118139B120B1C9
:1019D0000178F62904BF8089704700207047DFF83E
:1019E00008C000DF704700BFC9230008EFF305837C
:1019F0002BB9EFF3108313B9EFF311830BB1002070
:101A00007047DFF808C000DF704700BFD923000827
:101A1000EFF3058129B9EFF3108111B9EFF31181CB
:101A200009B3B0B5E0B10178F62919D1C18900F147
:101A30000C02D2E85F3F994202D8BFF32F8F04E037
:101A40005C1CC2E8554F05B1F3E7C28999B29142D7
:101A500024BF6FF00200B0BDFFF7E2FC0020B0BD74
:101A60006FF00300B0BDDFF808C000DF704700BFB3
:101A700059240008DFF804C000DFFEE7AD240008A9
:101A8000EFF3058028B9EFF3108010B9EFF3118060
:101A900010B1034840697047DFF808C000DF7047A5
:101AA000800901201D250008EFF3058129B9EFF316
:101AB000108111B9EFF3118111B14FF0FF30704770
:101AC000DFF804C000DF704729250008EFF3058325
:101AD0002BB9EFF3108313B9EFF311830BB100208F
:101AE0007047DFF808C000DF704700BF45250008D9
:101AF000EFF3058129B9EFF3108111B9EFF31181EB
:101B000011B16FF005007047DFF804C000DF7047C7
:101B100021270008EFF305822AB9EFF3108212B9EA
:101B2000EFF3118212B16FF005007047DFF804C0C7
:101B300000DF704759270008EFF3058129B9EFF35B
:101B4000108111B9EFF3118111B16FF005007047E9
:101B5000DFF804C000DF7047A5270008EFF3058C0D
:101B6000BCF1000F09D1EFF3108CBCF1000F04D1D0
:101B7000EFF3118CBCF1000F01D000207047DFF8AB
:101B800008C000DF704700BF65280008EFF305823A
:101B90002AB9EFF3108212B9EFF3118212B16FF08C
:101BA00005007047DFF804C000DF7047E128000837
:101BB000EFF3058129B9EFF3108111B9EFF311812A
:101BC00011B16FF005007047DFF804C000DF704707
:101BD0002D29000830B180B501461320FFF70AFE19
:101BE000BDE88040002070470148007A704700BF80
:101BF00080090120B0B50848C568FFF75BF80446C6
:101C0000FFF76AF818B10135FFF754F80446FFF7FB
:101C10005DF800FB0540B0BD800901200148C068A7
:101C2000704700BF800901202DE9F843504F387AF2
:101C3000012800F09580002840F0948007F108000A
:101C40009C21FEF7A0FEDFF82C81B8F81000A7F861
:101C50005400D8E90202D8E90B41FA6538642046FD
:101C6000FFF794FA08B1C7F88040D8E90541DFF8DA
:101C70000891D8E907562046C847D7F880100028B1
:101C8000284618BF214679673146C847D7F88010E3
:101C9000002818BF2946B967D8E909412046C84736
:101CA000D7F88010002818BF2146D8F83440F967CB
:101CB0003CB12168D4E902232046FFF7C4FAC7F8F3
:101CC0008440D8F838403CB12168D4E9022320464A
:101CD000FFF7B9FAC7F88840D8F83C403CB1216812
:101CE000D4E902232046FFF7AEFAC7F88C40D8F8B3
:101CF00040403CB12168D4E902232046FFF7A3FA13
:101D0000C7F89040D8F844403CB12168D4E9022398
:101D10002046FFF798FAC7F89440D8F848403CB1FD
:101D20002168D4E902232046FFF78DFAC7F89840CE
:101D3000D8F84C403CB12168D4E902232046FFF793
:101D400082FAC7F89C40D8F850403CB12168D4E9E9
:101D500002232046FFF777FAC7F8A0400120387227
:101D6000002001E04FF0FF3001B0BDE8F08300BF7C
:101D700080090120005000088D1100080648017AF2
:101D8000032904BF01207047022911BF4FF0FF3023
:101D9000032101720020704780090120B0B51D4C5D
:101DA000207A01281CD1FFF7FDFCC8B11A48FF2199
:101DB0001A4D8175817D026881F0FF01C2F3022214
:101DC000B1FA81F1C1F120018A4228BF511CFE22E3
:101DD00002FA01F1C17468681149FEF785FF10B17C
:101DE0004FF0FF30B0BDFEF76DFF2061FEF74CFFF6
:101DF00004F11C00FFF75CFCFFF7F4FC2878C00737
:101E00000CBF0320022080F31488022020720020DF
:101E1000B0BD00BF800901200CED00E000500008BB
:101E2000CD0300082DE9F84300284CD00F466FF091
:101E30000305002949D004460078FA2845D12046F8
:101E400099469046FEF7B9FE002842D00646204645
:101E50003146FEF705FF626A06F10C013846FEF7CF
:101E6000F1FCB8F1000F1CBFF07888F8000004F115
:101E70000C070025314638463570FFF7BFF9A068DA
:101E800018B33846FFF79DF90025F0B10646204605
:101E9000FFF70EFC002101220746FFF7C9FC384678
:101EA000FFF762FC8168626A074606F10C00FEF7E4
:101EB000C9FCF920B57031463070F868F0702046E2
:101EC000FEF79DFE01E06FF00305284601B0BDE876
:101ED000F083B9F1000F10D083204946FFF78AFC48
:101EE00040B1074841692046FFF7ECFBEFF309805A
:101EF000C0E902786FF00105E7E76FF00205E4E75B
:101F0000800901202DE9F84F002770B10D4661B11D
:101F100005F10F010446B0FA80F021F00306B6FA8D
:101F200086F10844202804D20027384601B0BDE8D5
:101F3000F08F06FB04F872B1D2F808A01368D2E95A
:101F40000490BAF1000F11D05FEA8A71ECD1D16828
:101F50003429E9D30DE000234FF000093449009300
:101F6000D1F8A00078B1FFF72CF912E0D168002970
:101F7000DAD1B9F1000F2FD000274045D5D319F0A1
:101F800003002BD0D1E7D1F8800034210122FFF7E4
:101F900094F882464FF0010BB9F1000F10D1BAF15D
:101FA000000F0DD0224F41460022F86FFFF785F851
:101FB000814638B148464146FEF7C3FC57461AE011
:101FC00057461AE0BBF1000F14D0D7F8A00060B15B
:101FD0005146FFF713F90DE00028A5D1BAF1000F23
:101FE000BCD000934FF0000BD6E7D7F880005146E5
:101FF000FFF7A3F800270BF1020B002F3FF495AF7A
:10200000002032464B46C7E90950C7E90B0000994A
:10201000C7E90110FA2087F802B02146387007F1AD
:102020000C00FFF710F90248024901677DE700BF85
:10203000800901208D1200082DE9F84338B30E46BF
:102040006FF00307002951D005460078FA284DD1DA
:10205000A86899469046E8B1407883281AD1284666
:10206000FFF726FB0021012204460027FFF7E0FBD3
:102070002046FFF779FB044680686A6A3146FEF71E
:10208000E1FBE06890B380F8008000272EE06FF05D
:1020900003072BE005F10C00FFF793F880B16A6AA3
:1020A00004460C303146FEF7CDFB0027F92084F8BA
:1020B00003802146A77020702846FEF7A0FD15E09A
:1020C000B9F1000F10D093204946FFF793FB40B1C0
:1020D000084841692846FFF7F5FAEFF30980C0E99F
:1020E00002686FF0010701E06FF00207384601B0A7
:1020F000BDE8F0838009012070B504462148456998
:102100004DB32CB32078F52822D1207E30B30E4673
:10211000E178CA0702D0E268AA422CD07EB38807D1
:102120000AD5E06895F9201090F920208A4203DA58
:1021300080F82010FFF7E5FA53203146FFF75AFBED
:1021400018B120462946FFF7BDFA6FF0010070BDB7
:102150006FF0030070BD4FF0FF3070BD0020C4E988
:102160000350E86A0028606100D00461EC6201203D
:102170002076002070BDFF2801D00130F8E76FF015
:10218000020070BD8009012010B5002852D004461D
:102190000078F5284ED1207EF0B3D4F814C0E06862
:1021A000BCF1000F1CBF2269CCF8102000F12C03F9
:1021B00021691A46002918BF01F11402C2F800C0B3
:1021C000E178890722D590F821C00BE093683BB1F4
:1021D00093F920304FFA8CF18B42C8BF5FFA83FC31
:1021E00002F114031A68002AF0D190F8201061451A
:1021F0000CD080F820C0FFF784FA07E02046FFF7F4
:1022000057FA6FF002010022FFF712FBA0680028C6
:10221000F4D10020FFF7F2F900202070A178C9075F
:1022200008BF10BD0849D1F8940030B12146FEF72F
:10223000E5FF07E06FF0030010BDD1F880002146F4
:10224000FEF77BFF002010BD8009012070B558B15A
:10225000D0E90065846884B1A10711D1C16800206C
:102260001C2938BF70BD16E0002500261149D1F8A1
:10227000940038B1FEF7A5FF0AE0C0680028F5D049
:10228000002070BDD1F880001C210122FEF715FF4F
:10229000044658B101206660E570A070F520112158
:1022A000207004F10800FEF76EFB00E000242046D9
:1022B00070BD00BF8009012070B504462B484069FD
:1022C00070B154B12178F52907D1217E11B1E268AE
:1022D000824209D06FF0020404E06FF0030401E0D1
:1022E0004FF0FF34204670BD01392176090601D038
:1022F0000024F7E7616909B122690A6100F12C0540
:1023000023692A46002B18BF03F114021160E178FB
:10231000890711D590F8211009E093682BB193F942
:1023200020304DB2AB42C8BF194602F114052A68ED
:10233000002AF2D180F82010A06890B12046FFF763
:10234000B7F90021002205460026FFF771FAC4E91B
:102350000356E86A0028606100D004610120EC6245
:10236000207600200024FFF749F9BBE7800901200F
:10237000B0B508B304460078F6281DD104F10C006E
:10238000D0E85F2F12B9BFF32F8F04E0531EC0E8CF
:10239000553F05B1F4E710041CBF0020B0BD71B17A
:1023A0006320FFF727FA20B1064841692046FFF76E
:1023B00089F96FF00100B0BD6FF00300B0BD6FF0A0
:1023C0000200B0BD8009012020B10178F62904BFC8
:1023D000808970470020704770B5054601384FF678
:1023E000FE730C460021984298BFAC4201D90846C2
:1023F00070BD4AB19068166870B181070FD1D2687C
:102400000021102AF3D314E000261149D1F89800D6
:1024100038B1FEF7D6FE0AE0D0680028F5D00021DA
:10242000E5E7D1F8800010210122FEF746FE60B1F9
:1024300001210022C5818481C0E901628170F621F9
:10244000044A017002498A6600E000200146CEE796
:102450008009012095140008B0B560B10178F62913
:1024600009D1816859B1FFF723F900210122002425
:10247000FFF7DEF901E06FF003042046B0BDC1892B
:1024800000F10C02D2E85F3F994202D8BFF32F8FD0
:1024900004E05C1CC2E8554F05B1F3E7C28999B26C
:1024A0006FF00200914238BF0020B0BD70B51A4DE8
:1024B000287A02282ED1686A002808BF70BD6C698E
:1024C000E06AFEF740FFA06918B100210022FFF783
:1024D000AFF9EFF30980A063686A81680029696237
:1024E00002D005F11C02CA600026C660FFF77AF927
:1024F0006E61E078C00704D12046BDE87040FFF768
:10250000ABB80420E6606070686B0028A06000D063
:10251000C4606C6370BD00BF800901200148406940
:10252000704700BF8009012040B10178F12905D131
:10253000417804291CBF90F9200070474FF0FF300C
:10254000704700002DE9FE4F10B380466AB102F1DA
:10255000100A9AE88006D2E900439668B6B1B0073F
:1025600016D1D068442813D317E04FF0180A00237F
:1025700000274FF000090024644A0293D2F8880033
:10258000CDE90014C8B1FEF71CFE1CE0D06820B1F4
:102590000025284603B0BDE8F08F37B10025B9F11A
:1025A000000FF6D017F00700F3D1BAF1000F38D0C2
:1025B000AAF101003728EBD835E0D2F88000442199
:1025C0000122FEF77AFD06464FF0010B67B95EB1B6
:1025D000B9F1000F0AD04D4849460022406FFEF77E
:1025E0006CFD98B107460FE035463EE04748484944
:1025F000D0F88400D1F854900028ECD0FEF7E1FD2B
:1026000020B107460BF1100B35462CE0BBF1000F53
:102610001CD03E49D1F88800E0B13146FEF7EEFD0E
:102620001DE04FF0180AB9F1000F06D00025B9F1EE
:10263000480FAED319F00700ABD1002E3FF49CAF8A
:10264000CDE9001402934FF0000BBFE74FF0000BF1
:10265000002707E0D1F880003146FEF76EFD002725
:102660004FF0010B00254BF0020B002D3FF491AF12
:102670000198182168600298E87040F2F11085F81E
:1026800002B0288005F10800FEF77DF907EB09008C
:10269000C5E90C79FD214038C5E90E08002085F810
:1026A0002F00C5F82B00C5F82700C5F8230085F8D2
:1026B0002210184985F821A085F820A0009E3960D5
:1026C0001349097849070AD511213A1D4FF0CC3337
:1026D000A1EB990101E008C201310029FBD1A96BEE
:1026E000002202E041F8220001320D2AFAD10A4A02
:1026F0004FF080700E62C1E90D28C8630348074996
:1027000001662846FEF77AFF43E700BF80090120F3
:1027100000500008A52E5AE2751A00082B17000871
:1027200010B5B0B104460078F12812D1607800F0FD
:102730000F0003281CBF6FF0020010BD2046FEF7FB
:10274000D6FF2046FEF722FF2046FEF757FF002067
:1027500010BD6FF0030010BD10B568B14A1E6FF0D8
:102760000304372A0AD80278F12A07D14278042ACA
:1027700006D16FF0020401E06FF00304204610BDA3
:1027800090F920204BB2934201D10024F6E780F863
:10279000211080F82010FEF7B4FF00200024FEF77F
:1027A0002DFFEBE770B5C8B104460078F12815D1CC
:1027B000607800F00F00012813D0032815D00228FC
:1027C0001CBF6FF0020070BD25496FF002000A7A4D
:1027D000022A18BF70BD496A69B970BD6FF0030065
:1027E00070BD2046FEF783FF05E02046FEF77FFF21
:1027F0002046FEF7CBFEE06AFEF7A5FDA06918B102
:1028000000210022FFF714F86078022811D1144D3E
:10281000EFF30980A063686A81680029696202D0C9
:1028200005F11C02CA600026C660FEF7DBFF6E6180
:1028300002E00020FEF7E2FEE078C00703D1204668
:10284000FEF70AFF0AE00020E06004206070044800
:10285000416B0029A16000D0CC604463002070BDB2
:1028600080090120F8B50E46002198B3012E31D819
:10287000144605464BB198681F6870B181070FD1A7
:10288000DA680021202A15D224E000271349D1F864
:102890008C0038B1FEF795FC0AE0D8680028F5D026
:1028A000002117E0D1F8800020210122FEF705FC6D
:1028B00070B10121C67081704FF4F971018000215F
:1028C000C0E90171C0E90311C0E90515C46100E068
:1028D00000200146084601B0F0BD00BF800901207C
:1028E000B0B578B105460C466FF00300C1B1297848
:1028F000F22918BFB0BD6878022806D12846FEF735
:1029000071FA08E06FF00300B0BD0748006D40B1F8
:1029100002206C61687028462146FEF73BFA0020D1
:10292000B0BD6FF00200B0BD8009012078B1017820
:10293000F2290CD1417802291CBF6FF002007047C8
:1029400080B501214170FEF74DFA002080BD6FF087
:102950000300704740F28D1CC2F2000C604740F249
:10296000010CC2F2000C60470B48006800F0020046
:1029700080B10948006820F0020007490860084655
:10298000806820F0010088600448006820F400009E
:10299000C1F80403704700000020014004230140F7
:1029A0000848406800F0200050B10648C06840F078
:1029B00020000449C8600846006F20F00100086745
:1029C00070470000006002401148006820F48060F9
:1029D0000F490860081D006820F48060091D086028
:1029E0000C48006820F480000A4908600948143047
:1029F000006840F480000749143108600648006808
:102A000020F0040004490860012004490870704760
:102A100008280040003C014010ED00E05C0501206A
:102A200010B50848806800F0020048B105484068C9
:102A300020F080000349486003480068FEF7E8FF83
:102A400010BD000000300140580501200648006814
:102A500000F0020038B104480838006820F0400057
:102A60000149083908607047083800401448006878
:102A700040F47000124908601248006840F00100FC
:102A80001049086000200F49083108600D480068AF
:102A90000D4908400B4908600C48091D0860081FD3
:102AA000006820F48020091F0860002005490C31CF
:102AB00008604FF0006002498039086070470000EC
:102AC00088ED00E000380240FFFFF6FE10300024E1
:102AD00010B51A48006800F08000E8B11848006896
:102AE00080681849098888420CD9154800684168EF
:102AF000144802880088401C124B1880885C0F49DB
:102B0000486009E00D48C06820F080000B49C860AB
:102B10000D480068FEF77CFF0848006800F02000C0
:102B200050B106484068C2B2084801780078401C9D
:102B3000064B18700648425410BD0000005000407B
:102B40004005012044050120480501204E050120D3
:102B5000246B012010B51A48006800F08000E8B12D
:102B60001848006880681849098888420CD91548B7
:102B700000684168144802880088401C124B188085
:102B8000885C0F49486009E00D48C06820F080006B
:102B90000B49C8600D480068FEF73AFF0848006816
:102BA00000F0200050B106484068C2B208480178E1
:102BB0000078401C064B18700648425410BD0000B7
:102BC0000010014034050120380501203C0501209A
:102BD0004C050120246A012000280DDB00BF00BF46
:102BE00000F01F02012191404209920002F1E0220F
:102BF000C2F8001100BF00BF70472DED020B019815
:102C000020F0004001909DED000B02B0704730387D
:102C10000A2801D2012070470020704710B50446F1
:102C200001F08AFE20B14FF0FF312068FEF7FCF979
:102C300010BD10B504462068FEF708FA10BD70B547
:102C400004460020FEF714FA2060206808B1012530
:102C500004E000252146052001F05CFE284670BDF9
:102C600010B5044601F068FE10B12068FEF712FAB4
:102C700010BD10B5FEF71AF910BD00000146084658
:102C80001E4A926842F001021C4B9A60122801D041
:102C900011280ED11A4A126822F48002174BC3F889
:102CA00004231A46D2F8042342F40002C3F8042392
:102CB00018E013280FD1124A126822F400020F4BB9
:102CC000C3F804231A46D2F8042342F48002C3F85E
:102CD0000423122006E00A4A126822F44002074B3D
:102CE000C3F8042340EA401242EA8022034B5A63AD
:102CF0001A46926842F080429A6070470020014074
:102D0000042301400148C06C80B27047002001409C
:102D100010B50446022C0DD1204600F091FB052091
:102D2000FEF774F84FF44040084908600520FEF7AC
:102D30006DF809E04FF0404004490860204600F07B
:102D40007FFB002001F06AF810BD00001808024067
:102D50008CB006462C22854901A8FDF7B8FD4FF03E
:102D6000000BD946002000903078012810D100F0E7
:102D7000BDFC0220FFF7CCFF9FED7D0A01F040FC77
:102D80000021012001F0F0FC00217A4841760AE0A0
:102D900030787E2805D18A2231467648FDF752FDEB
:102DA00001E000BFFEE7FEF797F800BF7148407EE4
:102DB000802808D10020704908700A46012190201F
:102DC00000F08AF9B0E06B48407E812805D101AA65
:102DD0002A21912000F080F9A6E06648407E8D28E7
:102DE00046D16448807E122831D1042000F0C6F913
:102DF00020B3052000F0C2F9B8B1062000F0BEF9FA
:102E000050B14FF0010B00205B4908700A460121C8
:102E10009D2000F061F987E00C20574908700A46B0
:102E200001219D2000F058F97EE00C2052490870E5
:102E30000A4601219D2000F04FF975E00C204E4913
:102E400008700A4601219D2000F046F96CE04948CF
:102E5000807E132868D1484908700A4601219D20C8
:102E600000F03AF94AF6AA204449086000BFFEE79C
:102E70004048407E8C2857D1BBF1000F54D03D4CC8
:102E80001A34A078E17800EB0109002504E0201D48
:102E9000405D8144681CC5B2E078A842F7DC6078E8
:102EA000217800EB0120484536D1A07850BB20792D
:102EB0000106607941EA0041A07941EA0020E17908
:102EC00040EA01072E48874201D207F580370425E2
:102ED00009E0201D415D384601F0E2FA00B105E04D
:102EE000681CC5B27F1CE078A842F2DC00BFE07825
:102EF000A84208D00E20204908700A4601219C20D3
:102F000000F0EAF810E010201B4908700A46012181
:102F10009C2000F0E1F807E00B20174908700A46F2
:102F200001219C2000F0D8F8FDF7ACFF80464FF05F
:102F3000000A00BFFDF7A6FFA0EB08004EF66021D7
:102F4000884203D24AF6AA200C4908600A4800F0D9
:102F50005DFA30B108490878064A694600F04EF833
:102F60008246BAF1000FE5D020E700005C4F000870
:102F70000000E14766720120F0720120003000403D
:102F800000000108014600207047014600207047FC
:102F90000020704710B504460022214609481EF063
:102FA00077FC012809D10021074829F0BDFB002248
:102FB000214604481EF06CFC02E00120FDF726FFCC
:102FC000002010BD250008100200080110B50446BD
:102FD00000222146074820F0F3FC072808D10021F1
:102FE000054829F0A1FB00222146024820F0E8FC18
:102FF000002010BD27000810030008012DE9F04152
:1030000005460E46144600273068052860D2DFE8E2
:1030100000F0030D273051007E2D06D18A21204675
:10302000FDF78FFC25700120306051E06088284357
:103030006080B4F8860028B960884FF6FF7101EA15
:1030400000206080B4F88600401C80B2A4F886009E
:10305000012804DD0020A4F886000220306037E05B
:1030600084F8855025710120A4F888000320306081
:103070002EE0863414F8010C284404F8010C608812
:10308000401C608034F88619601D4554B4F88600F1
:103090007F280CDAB4F88600401CA4F8860060880B
:1030A000B4F88810401A04D10420306001E00020F8
:1030B00030600DE014F8850F284420700020306047
:1030C00014F88509FF2801D1012700E0002700BF7F
:1030D00000BF3846BDE8F0812DE9F04106460D46B7
:1030E00017464FF00008442D3BD21F4806762A466B
:1030F00039461930FDF7A6FB032406E01A48005DA7
:10310000404400F0FF08601CC4B205F11900A04261
:10311000F4DCC8F1FF022046611CCCB212490A540B
:10312000201F887000204870104811490860084628
:10313000006884600C480968486000200D490880D8
:103140000B48006841680B4802880088401C094B06
:103150001880885C084948600846C06840F08000D4
:10316000C860BDE8F08100005E050120BC050120BB
:1031700040050120440501200050004000B50246F2
:1031800000BF3648006840F4F9703449086000BF59
:103190003248006800F480300028F9D101F0C0FA0C
:1031A0002E48001D006820F440702C49091D08605D
:1031B0000846006840F4007008600846006820F087
:1031C000F800086008460068022141EAC20108438D
:1031D0002249091D08600846006840F480300860F4
:1031E00001E001F0B9FA1D48006800F480300028C1
:1031F000F7D11A48001D006820F002001749091D88
:1032000008600846006820F0F8000860084600687A
:1032100020F44070086011480C38006820F4806089
:103220000E490C3908600846006840F48050086078
:103230000846006820F4805008600846006840F4A2
:103240008060086000F0AEFF00BF0448006800F432
:10325000F97008B1002000BD0120FCE70C3C0240E1
:103260000F2100E0491E002905DB0D48084490F8B5
:10327000000A0028F6D1002207E00A4800EB4110BE
:10328000805CFF2800D002E0521C102AF5DB00BF52
:10329000102A01D100207047024800EB4110FAE7E4
:1032A0000070FF1F0078FF1F014609480078094A97
:1032B0001278904201D100207047064802780078C9
:1032C000401C044B18700448805C08700120F3E730
:1032D0004C0501204D050120246A012001460020F3
:1032E0003C4A914203D2B1F1006F00D370E03A4AF8
:1032F000914204D2374A914201D3012068E0374A13
:10330000914204D2344A914201D3022060E0344A0F
:10331000914204D2314A914201D3032058E0314A0C
:10332000914204D22E4A914201D3042050E02E4A09
:10333000914204D22B4A914201D3052048E02B4A06
:10334000914204D2284A914201D3062040E0284A03
:10335000914204D2254A914201D3072038E0254A00
:10336000914204D2224A914201D3082030E0224AFD
:10337000914204D21F4A914201D3092028E01F4AFA
:10338000914204D21C4A914201D30A2020E0B1F1BB
:10339000016F04D2194A914201D30B2018E0184A58
:1033A000914204D2B1F1016F01D30C2010E0154A13
:1033B000914204D2124A914201D30D2008E0124AF0
:1033C000914204D20F4A914201D30E2000E00F2017
:1033D00070470000004000080080000800C000089E
:1033E00000000108000002080000040800000608B0
:1033F0000000080800000A0800000C0800000E0881
:1034000000001208000014080000160801460948D0
:103410000078094A1278904201D10020704706488E
:1034200002780078401C044B18700448805C0870D7
:103430000120F3E74E0501204F050120246B0120F8
:1034400010B50446022C17D12448006840F0400013
:10345000224908602248006840F400302049086092
:1034600040F281120021012000F03EF88322002169
:10347000022000F039F830E0012C17D1174800681D
:1034800020F04000154908601548006820F400301D
:10349000134908604FF4C0720021012000F048F881
:1034A00082220021022000F043F816E00B48006859
:1034B00020F04000094908600948006820F4003005
:1034C0000749086040F281120021012000F030F825
:1034D00083220021022000F02BF810BD00380040AC
:1034E0000000024030BF70472DE9F04104460D4610
:1034F000164604EB440000EBC4000C4901EB40010C
:10350000681C085C04EB440101EBC401074A02EBB0
:103510004101495D00EB012087B227EA06022946F6
:10352000204600F0B7F8BDE8F081000024720120C9
:103530002DE9F04104460D46164604EB440000EB2D
:10354000C4000C4901EB4001681C085C04EB440119
:1035500001EBC401074A02EB4101495D00EB012088
:1035600087B247EA06022946204600F093F8BDE8F4
:10357000F08100002472012070B540F608020A2193
:10358000002000F087F800240BE0002505E0294624
:10359000204600F051F8A81CC5B2152DF7DB601CC1
:1035A000C4B2032CF1DB4FF6FF720021084600F095
:1035B00071F84FF6FF720C21002000F06BF84FF409
:1035C00010720C210120FFF7B3FF40220C210220D2
:1035D000FFF7AEFF40F2011212210120FFF784FF36
:1035E000812212210220FFF77FFF44F242220A21AA
:1035F0000020FFF79DFF4FF6FF720421002000F02E
:1036000049F870BD30B5024602EB420303EBC2033A
:10361000084C04EB43044B1CE35C02EB420404EB58
:10362000C204044D05EB4404645C03EB042398B22C
:1036300030BD00002472012070B504460D464FF4E1
:10364000801012498861412141EA440105EB0121C2
:1036500088B200F0F1FF002000F0EEFF06461020D7
:103660000A498861301204EB440101EBC401084AA5
:1036700002EB4101485504EB440000EBC40002EBAF
:103680004002681C1654304670BD00000000024025
:103690002472012070B504460D461646301204EB24
:1036A000440101EBC4010F4A02EB4101485504EB10
:1036B000440000EBC40002EB4002681C16544FF4B7
:1036C000801009498861402141EA440105EB01214C
:1036D00088B200F0B1FF304600F0AEFF1020024982
:1036E000886170BD247201200000024070B5FE4860
:1036F000006840F48030FC490860012506E0FA4883
:10370000006800F4003000B104E06D1C25F07F403B
:103710000028F4D100BFF448001D006820F03F00ED
:10372000F149091D08600846006840F0080008607B
:103730000846006847F6C0718843EB49091D0860D8
:103740000846006840F4C05008600846006820F44D
:1037500040300860081F006800F4003080B108465F
:10376000006840F480000860081D006840F0010017
:10377000091D0860DC48006820F00100DA49086093
:10378000DA48006840F00600D8490860084600683A
:1037900040F4E0600860D4480830006840F480508D
:1037A000D149083108600846006840F400400860CC
:1037B000CD484030006840F08050CB49403108602F
:1037C000CB48006840F44040C9490860C6480068DA
:1037D00040F08070C449086000BFC548406800F4EC
:1037E00080400028F9D000BFBF48006800F000709A
:1037F0000028F9D0BC480830006840F00200BA49FF
:10380000083108600846006820F0010008600022C6
:1038100001210846FEF7EAF8B649086000220121B6
:103820000846FEF7E3F8B449086000220121084683
:10383000FEF7DCF8B1490860002201210846FEF7D6
:10384000D5F8AF490860002201210846FEF7CEF8FE
:10385000AC490860A4483030006840F00200A2493A
:1038600030310860A848006840F40050A64908605C
:103870000846006840F400400860A3482030006813
:1038800040F0E060A049203108600846006840F040
:10389000E04008609C48006840F480109A49086045
:1038A00008159949183108608F483030006840F099
:1038B00001008D49303108609448006840F4807000
:1038C000924908600846006840F4006008600846B5
:1038D000006840F4005008600846006840F400406A
:1038E0000860102088610846006A40F4A000086261
:1038F0000846006A40F0A06008620846006A40F08E
:10390000A04008620846006840F4002008600846AD
:10391000006840F4001008600846406A40F050011A
:103920007A484162406A40F4A06178484162006888
:1039300040F48030754908606B480830006840F4F6
:1039400080006949083108600846006840F08060DE
:1039500008606E48006840F00C006C4908606A48D6
:10396000006840F00300684908600846006840F0BD
:103970000C0008605C483030006840F004005A4990
:10398000303108606248006840F08050604908604B
:103990000846006840F080400860534844300068A2
:1039A00040F0100050494431086040F283605949AA
:1039B00088600846C06840F40050C8600846C06887
:1039C00040F00800C8600846C06840F00400C860C5
:1039D0000846C06840F02000C8602520FFF7FCF8CA
:1039E00041484030006840F480103F494031086051
:1039F00040F28360484988600846C06840F400503F
:103A0000C8600846C06840F00800C8600846C06842
:103A100040F00400C8600846C06840F02000C8605C
:103A20003520FFF7D9F830483030006840F40010F6
:103A30002D49303108603948394988673948C867A5
:103A4000302048670846006F08670846006F40F45A
:103A5000403008670846006F40F480400867084619
:103A6000006F40F4006008670846006F40F4806013
:103A700008670846006F08670846006F40F040007E
:103A800008670846006F40F010000867244884303B
:103A9000006840F00400C1F884000846D0F88400B3
:103AA00040F00100C1F884000F20FFF795F80E48A0
:103AB0004430006840F480500B49443108601A4893
:103AC000006840F40060184908600846006840F04B
:103AD000100008600846006840F0040008600846CE
:103AE000406840F0040021E000380240003C024001
:103AF000007000403C0501204805012058050120C8
:103B0000500501205405012000040240000002403D
:103B10000008024000100140005000400C380040F6
:103B200000600240246F01200030014048600846D8
:103B3000006840F0400008602320FFF74DF8FFF7D1
:103B40001BFD5A48006840F48040584908605848B6
:103B5000006840F40060564908600846006840F07C
:103B6000080008600846006840F004000860081D6E
:103B7000006840F00400091D08600846006840F035
:103B8000020008604948001D006840F48070474901
:103B9000091D08604748D0F8040340F44030454907
:103BA000C1F804030846C06A40F40010C862084621
:103BB000006940F0380008610846006940F0E060A4
:103BC00008610846006940F0605008610846C06816
:103BD00040F46000C8600846C06840F0E060C8601B
:103BE0000846406840F0200048600846406840F4BD
:103BF000807048601220FEF7EFFF2C48006840F408
:103C000080602A4908602C48006840F480002A49F6
:103C1000086029480830006840F4800026490831CF
:103C2000086022483430006840F001001F493431F8
:103C300008602248006840F48070204908601B48F2
:103C40003030006840F40070184930310860084690
:103C5000006840F4004008601948006840F4804063
:103C6000174908600320FEF7B7FF002419E004EBB2
:103C70004401144A02EB41106021FCF762FE04EBA0
:103C80004401114A02EB4110FF226021FCF751FE72
:103C9000962004EB44010C4A02EB41110870601CB1
:103CA000C4B2082CE3DB002070BD000040380240A5
:103CB0000038004000200140003C014000700040FE
:103CC00008280040246C0120246F012018B5044608
:103CD0004D292ED1102C2CD010680090012B24D00F
:103CE000022B1AD0032B0ED0042B1DD19DF80300FC
:103CF00010709DF8020050709DF8010090709DF8C2
:103D00000000D07012E09DF8020010709DF80100D4
:103D100050709DF80000907008E09DF80100107050
:103D20009DF80000507001E000BF00BF00BF0320FD
:103D300018BD0820FCE7000010B50446A06800B9D3
:103D400010BD4FF47A710E480068FDF70DFE0D4866
:103D5000046000200C4908800A48006841680A484D
:103D600002880088401C084B1880885C074948601E
:103D70000846C06840F08000C86000BFE0E700006F
:103D80003C050120340501203805012000100140C8
:103D900010B50446A06800B910BD4FF47A710E4802
:103DA0000068FDF7E1FD0D48046000200C49088023
:103DB0000A48006841680A4802880088401C084B8D
:103DC0001880885C074948600846C06840F0800059
:103DD000C86000BFE0E70000480501204005012061
:103DE000440501200050004090B14AF6AA210A4A39
:103DF00011604910116003215160B0F5805F00DD52
:103E00009014411E044A91604CF6CC41116000E0D0
:103E1000704700BFFCE70000003000400C49096813
:103E200021F440310A4A116040B11146096841F459
:103E3000003111600121074A117008E00449096846
:103E400041F48031024A11600021024A117070472A
:103E5000000002405D05012010B54FF0FF313848E9
:103E60000068FDF781FD002456E04FF4806035497D
:103E70008861C00388610846006880F440200860BB
:103E80000846006880F4401008604815886104EB1B
:103E900044002D4901EB40102C49C8670846006FCB
:103EA00020F4C05008672A48006820F400602849C0
:103EB00008606020254948674FF0007021498861FB
:103EC000400088610846006880F440200860084689
:103ED000006880F4401008601C48006F40F001004A
:103EE0001A49086702E00120FCF790FF1748006FAD
:103EF00000F001000028F6D115480830006800F0F5
:103F000080000028EFD112480830006800F002005D
:103F10000028E8D0601CC4B2082CA6DB0848006862
:103F2000FDF776FD4FF4807212210120FFF700FBB0
:103F30004FF4807212210120FFF7D6FA10BD000065
:103F40005405012000000240246F0120006002405F
:103F50000038004010B54FF0FF313A480068FDF7D7
:103F600003FD002454E04FF0806037498861401021
:103F700088610846006880F44020086008460068B0
:103F800080F4401008604815886104EB44002F4914
:103F900001EB40102E49C8670846006F40F40060EE
:103FA00008672C48006840F400602A490860302007
:103FB000274948674FF00070234988610846006828
:103FC00080F4402008600846006880F440100860D3
:103FD0001F48006F40F001001D49086702E0012002
:103FE000FCF714FF1A48006F00F001000028F6D11A
:103FF00018480830006800F080000028EFD115480C
:104000000830006800F002000028E8D0601CC4B24C
:10401000082CA8DB0B480068FDF7FAFC4FF480720F
:1040200012210120FFF784FA4FF48072122101203F
:10403000FFF75AFA0848007810B90120FFF7EEFEA2
:1040400010BD00005005012000000240246C01203A
:1040500000600240003800405D05012070B5044654
:104060000D4616464FF0FF312A480068FDF77CFCEC
:10407000022D09D104EB4401274A02EB41103246DC
:10408000264900F015FB3FE0012D1ED104EB440151
:10409000214A02EB411032462049183100F008FB5A
:1040A00004EB44011C4A02EB411032461B491E310D
:1040B00000F0FEFA04EB4401174A02EB41103246CD
:1040C0001649243100F0F4FA1EE0EDB904EB440186
:1040D000114A02EB411032461049891D00F0E8FAFE
:1040E00004EB44010C4A02EB411032460B490C31FF
:1040F00000F0DEFA04EB4401074A02EB41103246BD
:104100000649123100F0D4FA02480068FDF780FC3D
:1041100070BD000054050120246F01207C4D000873
:1041200070B504460D4616464FF0FF310948006849
:10413000FDF71AFC04EB4400074901EB4010074966
:1041400011F8351020F8116002480068FDF760FC96
:1041500070BD000050050120246C0120FC4B0008BC
:1041600070B504460D4616464FF0FF310A48006808
:10417000FDF7FAFB094A02EBC502911C04EB44026D
:10418000074B03EB4210324600F092FA02480068F7
:10419000FDF73EFC70BD000054050120FC4B0008FB
:1041A000246F01200748006840F00040054908607E
:1041B00000BF0448001F006800F480300028F8D1D8
:1041C00070470000103C02402DE9F04107460D46C3
:1041D00007FB05F404F0030020B104F00300C0F174
:1041E000040004440D480E49096846180C4800684C
:1041F00020440B49086008460068B0F5C04F06D35C
:1042000008460068001B08600020BDE8F0812146D8
:104210003046FCF796FB3046F7E70000240A012001
:10422000300501202DE9F0470F24102224492448AD
:104230001030FCF74DFA08B9BDE8F08700E0641EC5
:10424000002C05DB1F48204490F8000A0028F6D116
:104250000F2C00D1F0E7002C16DB00250EE01A48E9
:1042600000EB441050F82500184A02EB8501D1F804
:10427000E01F884200D003E0681CC5B2042DEEDBCD
:1042800000BF042D00D1D7E7641C00260DE00F48C5
:10429000304490F8E07F0C4800EB441000EB060837
:1042A0003946404600F0FCF8761C102EEFDB08483B
:1042B00004EB00090021484600F0F2F800BFBBE71C
:1042C000D0FF00080070FF1F0078FF1F00F00008FB
:1042D000007AFF1F0020704770B506460C46154651
:1042E00002E00120FCF792FD0748006800F48030EE
:1042F0000028F6D105483060032020604FF40030DC
:104300002860002070BD00000C3C024000000A083C
:10431000034600BF0748006800F480300028F9D148
:1043200005481860054808604FF480401080002060
:10433000704700000C3C024000000608000008081E
:1043400070B504461CB10848FEF7C8FF02E00748F4
:10435000FEF7C4FF05462846FEF710FF08B100200F
:1043600070BD0920FCE700000000080800000608F6
:104370002DE9F04704460B461546D5E90067A946E6
:104380004448006840F4F97042490860B3F5804F32
:1043900002DB0820BDE8F08784B1D8003E494158CF
:1043A000DFF8F4C0604440684FF0FF3A81EA0A0148
:1043B00080EA0A00014312D00820EBE7D800374911
:1043C0004158DFF8D8C0604440684FF0FF3C81EAB4
:1043D0000C0180EA0C00014301D00820DAE70CB19F
:1043E0002D4800E02D48804608EBC30800BF00BF01
:1043F0002848006800F480300028F9D100F090F9D6
:10440000002231E000BF2348006800F4803000281B
:10441000F9D12048001D006820F440701D49091D95
:1044200008600846006840F40070086008460068AC
:1044300040F00100086059F8220048F8220000BF4F
:104440001448006800F480300028F9D11148001D9C
:10445000006820F001000F49091D08600846006847
:1044600020F440700860521C022ACBD3FFF79AFE5A
:1044700000BFD8E9000170407940084301D008200E
:1044800088E70448006800F4F97008B1092081E762
:1044900000207FE70C3C02400000080800000608EE
:1044A00000B502460B461078FF2801D0082000BD59
:1044B00000BF1D48006840F4F9701B49086000BF48
:1044C0001948006800F480300028F9D100F028F97C
:1044D0001548001D006820F440701349091D08604C
:1044E0000846006808600846006840F0010008605F
:1044F000137000BF0C48006800F480300028F9D128
:104500000948001D006820F001000749091D0860E6
:10451000FFF748FE00BF0448006800F4F97008B1D6
:104520000920C4E70020C2E70C3C024010B5044655
:10453000012C09D1012212211046FEF7F9FF4FF498
:10454000FA70FCF763FC07E0012212211046FEF727
:10455000CBFF6420FCF75AFC10BD10B50446012CBB
:1045600004D180221221FEF7E3FF04E08022122111
:104570000120FEF7B9FF10BDB0EE401AF3EE001AAD
:1045800061EE211A80EEA12AB0EE420AFCEEC01ABA
:1045900011EE901A4FF6FF7202EA011001EE901A26
:1045A000F8EE611A70EE611AB3EE002A61EE821A1B
:1045B000B0EE610AFCEEC01A11EE901A01EE901AEC
:1045C000F8EE611A70EE611AB6EE002AF4EEC21A25
:1045D000F1EE10FA00DD491C40EA010290B270478A
:1045E00000B5F0EE402ADFED040AB0EE620AFFF7F4
:1045F000C3FF0249886000BD001B374C001001401A
:1046000000B5F0EE402ADFED040AB0EE620AFFF7D3
:10461000B3FF0249886000BD001B374C00500040CA
:104620000448006840F0807002490860FFF75EF8B7
:1046300000F020F87438024070B5044600210B48A1
:104640000068FDF791F90A48C460406840F08000B6
:10465000074948604FF47A7104480068FDF784F90F
:104660000348C06885B2284670BD00005805012087
:104670000030014010210020FEF7DEFF0A480068EC
:1046800040F00400084908600848006840F0040051
:10469000064908600846006840F002000860881576
:1046A000486030BF00BFFEE710ED00E00070004042
:1046B00070B5034614468D88A54200DA70BD88782F
:1046C000B0B1224604E040104FF6FF7505EA420201
:1046D00000F00105002DF6D00D786D1C5D5D8E7823
:1046E000B543D6B235430E78761C9D55121200E0C4
:1046F0002246487888B104E040104FF6FF7505EA7D
:10470000420200F00105002DF6D00D785D5D4E7877
:10471000B543D6B235430E789D5500BFCEE70000B5
:104720000948006800F0004028B1084806490C39E3
:1047300008600748086000BF0348001F006800F4D5
:1047400080300028F8D17047103C024023016745B3
:10475000AB89EFCD704700004AF6AA2001490860F6
:10476000704700000030004070B504460D46012C33
:1047700050D1012212210220FEF7DAFE4FF47A70A6
:10478000FCF744FB2DBB2648006840F0007024492C
:1047900008600846006840F0006008600846406A0B
:1047A00040F430211E484162406A40F430011C4808
:1047B0004162802212210220FEF7BAFE022212215B
:1047C0001046FEF7B5FE042212210220FEF78CFEF1
:1047D00025E01348006820F0007011490860084681
:1047E000006820F0006008600846406A20F430212C
:1047F0000B484162406A20F430010948416284223A
:1048000012210220FEF794FE022212211046FEF72A
:104810006BFE04E0812212210220FEF765FE70BDCE
:1048200000040240F8B500200090002633480068DC
:1048300000F0005050B1FCF739FB0022114630481F
:10484000FDF744F9FCF75AFB00BFFEE72D4800686E
:10485000401C10B32B48001F01684FF00060FEF7AA
:1048600079F80446284801682648001DFEF772F8CA
:1048700005462548001D0068A84207D1A54205D07D
:1048800041F28830FFF7B0FAFEF769F81D4800687A
:10489000A04203D00120009000E001268EB941F231
:1048A0008830FFF7A1FA1948016817480830FEF769
:1048B00051F804461548001D0068A04201D00120AF
:1048C00000900E484438006820F480500B49443969
:1048D0000860FFF7A7FC9DF8000050B1FCF7E6FA6E
:1048E000002269460A48FDF7F1F8FCF707FB00BF14
:1048F000FEE71BF085FB0020F8BD00007438024085
:1049000021460008FCFF0008F8FF0108F8FF050831
:10491000512D0008062809D2DFE800F0080304053D
:10492000060704E003E002E001E000E000BF00BF92
:1049300000BFFEE700BFFEE710B50648007830B9BB
:10494000FCF776FA012802DD0120024908700148CF
:10495000007810BDCC050120491058BFC1F140417D
:104960005B1058BFC3F140438B42EFF300807047A8
:1049700051EA030C17D41CF5801F58BFBCF5801FEB
:1049800000F10680994218BF704708BF90427047F7
:1049900007D711F5801F58BF13F5801F19D499420E
:1049A0007047894270471CF5801F08D5BCF5801FF1
:1049B000F7D58B4218BF704708BF824270474FF44B
:1049C000001C1CEB410F38BF1CEB430F01D28B4284
:1049D000704770B500F008F8922449004FF000517C
:1049E0004FF08053FFF7B8BF0EF1020E2EF0030E0A
:1049F0005EF8046B364205D4012A43EB030515F536
:104A0000001F12D8012841EB010C1CF5001F0CD827
:104A10000ED14FEAD17C15F5001F0CEB4C0C0CF1BC
:104A2000020C08BF4CEBD37C04E04FF0080C01E013
:104A30004FEAD37C0CEB4C0526FA05F606F0070688
:104A4000B6F1040C06D20EEB860CBDE870404CF0BB
:104A5000010C6047DFE80CF0090B02024FF0004147
:104A60004FF00000A1F5002170BD19461046012845
:104A700051EB010418BFD4F5001484BF002001F0ED
:104A8000004170BD0808A0F500114FEA31017047E0
:104A900043004FEAD30C4FEA3C0C43401FBF400792
:104AA0000CF1605113F0FE4F70471CF0006F03D102
:104AB00000200CF0004170470CF0004343EA5070B6
:104AC00010B540EACC0000F03EF800BF00000092B4
:104AD0004FEA0001FFF7D6BF4FF000414FF0000052
:104AE000A1F5002170474FF07E5209E011F000421D
:104AF00004D54042C1F1000138BF491E42F07E5248
:104B00000B0002F1706212BF20235FEA00017047C0
:104B1000B1FA81FCA3EB0C0301FA0CF120FA03FCBF
:104B200002EBC352C3F1200341EA0C0110FA03FC6B
:104B30005CEA416C42EB112018BF5FF0806C28BF2B
:104B400020F0010070470EF1020E2EF0030E5EF809
:104B5000044B244204D44FEA4102B2F17F4F11D8F2
:104B60004FEA4003B3F17F4F0CD80ED14FEAD07C0F
:104B7000B2F17F4F0CEB4C0C0CF1020C08BF4CEB6C
:104B8000D17C04E04FF0080C01E04FEAD17C0CEB43
:104B90004C0324FA03F404F00704B4F1040C06D225
:104BA0000EEB840CBDE810404CF0010C6047DFE8D0
:104BB0000CF0070802024FF00040A0F5800010BD85
:104BC0000846420018BFD2F1807288BF00F0004052
:104BD00010BD4FF04070E1EE100A7047436F7079DE
:104BE0007269676874284329203230323020416B63
:104BF000726F6E2042726173730000002F005F7F3E
:104C000000007F002E005E3F80007F002D005D1FB2
:104C1000C0007F002C005C0FE0007F002B005B07D2
:104C2000F0007F002A005A03F8007F002900590194
:104C3000FC007F00280059FE00007F002700587FFD
:104C400000007F002600573F80007F002500561F90
:104C5000C0007F002400550FE0007F0023005407B0
:104C6000F0007F0022005303F8007F002100520172
:104C7000FC007F00200052FE00007F001F00517FDB
:104C800000007F001E00503F80007F001D004F1F6E
:104C9000C0007F001C004E0FE0007F001B004D078E
:104CA000F0007F001A004C03F8007F0019004B0150
:104CB000FC007F0018004BFE00007F0017004A7FB9
:104CC00000007F001600493F80007F001500481F4C
:104CD000C0007F001400470FE0007F00130046076C
:104CE000F0007F0012004503F8007F00110044012E
:104CF000FC007F00100044FE00007F000F00437F97
:104D000000007F000E00423F80007F000D00411F29
:104D1000C0007F000C00400FE0007F000B003F0749
:104D2000F0007F000A003E03F8007F0009003D010B
:104D3000FC007F0008003DFE00007F0007003C7F74
:104D400000007F0006003B3F80007F0005003A1F07
:104D5000C0007F000400390FE0007F000300380727
:104D6000F0007F0002003703F8007F0001003601E9
:104D7000FC007F00000036FE00007F003107C0000D
:104D80001F00323F80007F00337F00007F0034FE31
:104D900000007F003401C000070035380000070024
:104DA00035070000070007060915222E0A16212DD7
:104DB0000B17232F050304110F10070606030F120C
:104DC00007041013080511140E0C0D02000107064C
:104DD0002B1E1C28271B202A2C1F1D290806071400
:104DE000121307060C1924000D1826010E1A2502AD
:104DF0002624251A1819060515092E22160A2D2112
:104E0000170B2F231D1B1C2624250605282A1E1CD4
:104E1000272C201B292B1F1D2C2A2B292728050571
:104E2000031E170B04201509051F160A2321222F24
:104E30002D2E05050F000E1810010C1A11020D1968
:104E40000806071412130404160A0000170B0000CA
:104E5000150900002321222F2D2E04042C200000F0
:104E60002B1F00002A1E00002927281D1B1C0404DC
:104E7000261A000025190000241800000E0C0D024F
:104E8000000104040410000005110000030F0000DD
:104E900008060714121303020514172E2B1C190001
:104EA0000312152D2A1B180D10070A232029260E80
:104EB00011080B221F28250C0F0609211E2724018B
:104EC0000413162F2C1D1A02030024272A2D150661
:104ED000040126292C2F1607050225282B2E17083A
:104EE000100D1A1D20230A130F0C181B1E21091266
:104EF000110E191C1F220B140120230A1C25071058
:104F00000D1E21091B24060F0C2A2D15272612031E
:104F1000002C2F1628191304012B2E1729181405FD
:104F2000021F220B1D1A08110E00100D2629202326
:104F30000A070F0C24271E2109060300181B2A2D1F
:104F4000151204011A1D2C2F16130502191C2B2EE5
:104F50001714110E25281F220B08000008003630F8
:104F6000343720426F6F746C6F6164657220312E2C
:104F700030300000000000000000000000000000D1
:104F80000000499602D2000000000000000000006E
:104F9000A4020120440000003003012000010000B1
:104FA0000100000000000000000000000000000000
:104FB00000000000E802012044000000300401204D
:104FC00000010000280000000000000000000000B8
:104FD000000000000000000020020120340000005A
:104FE00054020120500000000000000000040000F6
:104FF0000800000000000000020001000010000096
:1050000007000000E803000000000000E0010120AC
:105010001000000000000000000000000000000080
:10502000000000000000000000000000E00100207F
:10503000000001000000000000000000000000006F
:105040000000000000000000000000000000000060
:105050000000000000010000884F0008AC4F00086D
:10506000D04F000804000000A40201202C030120FE
:105070000000000000000000000000000000000030
:105080000000000000000000000000000000000020
:105090000000000000000000200201205402012056
:1050A0005254582056352E352E310000DC50000861
:1050B00000000020E001000070020008BC5200085F
:1050C000E0010020440801001402000840560008D6
:1050D000240A0120648200008C0200084FF0006165
:1050E0006F4A72B64AF6AA236E4C23606E4B1B6859
:1050F00043F4F9736C4C236000BF6B4B1B6803F4E3
:105100008033002BF9D1694B674C083C2360684B16
:105110002360654B1B1D1B6823F0F803624C241DA4
:10512000236023461B6843F00203236023461B6869
:1051300043F48033236000BF5B4B1B6803F4803370
:10514000002BF9D1584B1B1D1B6823F0F803564C5C
:10515000241D236023461B6843F00A032360234673
:105160001B6843F48033236000BF4F4B1B6803F47C
:105170008033002BF9D14C4B1B1D1B6823F0F80327
:10518000494C241D236023461B6843F0120323600F
:1051900023461B6843F48033236000BF424B1B68E7
:1051A00003F48033002BF9D13F4B1B1D1B6823F008
:1051B000F8033D4C241D236023461B6843F01A036B
:1051C000236023461B6843F48033236000BF364BC3
:1051D0001B6803F48033002BF9D1334B1B1D1B6874
:1051E00023F00203304C241D236023461B6823F068
:1051F000F803236023461B6823F44073236023468F
:105200001B6843F40073236023461B6843F00103CB
:10521000236000200FE003E04AF6AA23214C23601C
:10522000214B1B6803F48033002BF5D152F820305A
:1052300041F82030401CB0F5804FECD31A4B1B1DB9
:105240001B6823F00103184C241D236023461B68B0
:1052500043F00043236000BF134B1B6803F480330B
:10526000002BF9D100BFFEE710B502460B46581CD3
:1052700008B9002010BD0F48006840F480500D4C64
:10528000206001200C4CA060114603E00A4C086825
:105290002060091DD0188842F8D807480068E9E75F
:1052A00000000108003000400C3C0240230167452B
:1052B000AB89EFCD303802400030024001FF01FFE2
:1052C00001FF01FF01FF01FF01FF01FF01FF01FFDE
:1052D00001FF01FF01FF01FF01FF01FF01FF01FFCE
:1052E00001FF01FF01FF01FF01FF01FF01FF01FFBE
:1052F00001FF01FF01FF01FF01FF01FF01FF01FFAE
:1053000001FF01FF01FF01FF01FF01FF01FF01FF9D
:1053100001FF01FF01FF01FF01FF01FF01FF01FF8D
:1053200001FF01FF01FF01FF01FF01FF01FF01FF7D
:1053300001FF01FF01FF01FF01FF01FF01FF01FF6D
:1053400001FF01FF01FF01FF01FF01FF01FF01FF5D
:1053500001FF01FF01FF01FF01FF01FF01FF01FF4D
:1053600001FF01FF01FF01FF01FF01FF01FF01FF3D
:1053700001FF01FF01FF01FF01FF01FF01FF01FF2D
:1053800001FF01FF01FF01FF01FF01FF01FF01FF1D
:1053900001FF01FF01FF01FF01FF01FF01FF01FF0D
:1053A00001FF01FF01FF01FF01FF01FF01FF01FFFD
:1053B00001FF01FF01FF01FF01FF01FF01FF01FFED
:1053C00001FF01FF01FF01FF01FF01FF01FF01FFDD
:1053D00001FF01FF01FF01FF01FF01FF01FF01FFCD
:1053E00001FF01FF01FF01FF01FF01FF01FF01FFBD
:1053F00001FF01FF01FF01FF01FF01FF01FF01FFAD
:1054000001FF01FF01FF01FF01FF01FF01FF01FF9C
:1054100001FF01FF01FF01FF01FF01FF01FF01FF8C
:1054200001FF01FF01FF01FF01FF01FF01FF01FF7C
:1054300001FF01FF01FF01FF01FF01FF01FF01FF6C
:1054400001FF01FF01FF01FF01FF01FF01FF01FF5C
:1054500001FF01FF01FF01FF01FF01FF01FF01FF4C
:1054600001FF01FF01FF01FF01FF01FF01FF01FF3C
:1054700001FF01FF01FF01FF01FF01FF01FF01FF2C
:1054800001FF01FF01FF01FF01FF01FF01FF01FF1C
:1054900001FF01FF01FF01FF01FF01FF01FF01FF0C
:1054A00001FF01FF01FF01FF01FF01FF01FF01FFFC
:1054B00001FF01FF01FF01FF01FF01FF01FF01FFEC
:1054C00001FF01FF0182127EA31680834142034443
:1054D0009D0C121483080713EC4F520846D8B805E8
:1054E00001013905513A010259090157126E1C0890
:1054F000116F041A70041A71041A72041112201226
:10550000801A40042902111A01041A02041A040420
:105510001A08041A10041A20041A40042B808099D7
:105520003202320429C9321032203240192149CFC7
:10553000093921191E1A801E1A801E1A801E1A800F
:105540001E1A801E1A801E2A808119211A803F1A75
:10555000803F1A803F1A803F2808801080208040BA
:10556000809C1A02171A08133A20CF08086101809C
:105570000280048008B4C978492C2928292429AF3D
:1055800049CC29C839C429C029155922292A2932C8
:10559000491F1A20041A08040B2402807C112A8057
:1055A0004B191E3964191E3968191E496C5A01704D
:1055B0001A04043A0804494B2953293D594A2952EF
:1055C000295AD91F59945A40985A109C4A04A0113C
:1055D0002A01A43C80393D15293E1F0758090308BC
:1055E000911029451A14101CA813035300121A080D
:1055F000FF3630343720526563656976657220580E
:1056000014021501B515018106A960CBF427601BB2
:10561000142C60495E0F1B4D6F6E69746F5D811BAA
:10562000C842D41A3FDCEA3E10695C19802C07405E
:1056300036BC6113A050069C08D1B3FB02000000E9
:08FFF80040560000E8EEA0995C
:020000040802F0
:10000000E0F754FF002003F05DFC00200CF0E8F95D
:10001000002009F011FE00200EF014FE00200BF06D
:1000200029FC002003F040FF012003F071FC0120B7
:100030000CF0EAF9012009F09BFE01200EF016FEFB
:10004000012000F089FF012003F0BEFF022003F031
:100050005FFC02200CF0D8F9022009F089FE022092
:100060000EF004FE022000F077FF022003F0ACFF48
:10007000032001F0BDFB03200BF084FD032004F0FE
:10008000B9FD03200CF046FC03200BF0B9F9032066
:1000900000F0CCFB032003F069FD042001F0A8FB75
:1000A00004200BF06FFD042004F0A4FD04200CF0EC
:1000B00031FC04200BF0A4F9042000F0B7FB04206D
:1000C00003F054FD052003F0DFFB052000F00CFFDA
:1000D000062003F0D9FB062000F006FF00F0C0FF69
:1000E00001F084FB0BF012FD04F02EFD0CF0BAFBC6
:1000F0000BF054F900F04CFB03F010FD012141F22C
:10010000883000F0F9FFE0F7F9FEFEE72DE9F0474F
:1001100007464C488A464C4D8178089C1E469046BE
:100120004FF0000949B180F802904946002045F897
:100130002010401CC0B22128F9D3212C02D3062064
:10014000BDE8F08755F8240020B10078B84233D0DC
:100150000720F5E728210120E4F736F845F82400C8
:1001600000286CD0077055F824104846C1F8049058
:1001700055F82410C1F8089055F8241081F80C9017
:1001800055F82410C1F8149055F82410C1F81090B7
:1001900055F824204FF0FF31916155F824100022CA
:1001A000C1F8209055F82410C86101210846E1F7F4
:1001B0001DFC55F8241048625FEA0A0006D00128A9
:1001C00004D0BAF1040F1BD00E20B9E755F8240073
:1001D0004068C8B90C210120E3F7F6FF55F8241058
:1001E000486060B3C0F8008055F8240008214068DA
:1001F00006813046E3F7E8FF55F8241049681AE015
:1002000055F82400806808B10D2099E70C210120E1
:10021000E3F7DAFF55F82410886080B1C0F8008059
:1002200055F824000821806806813046E3F7CCFFAA
:1002300055F824108968486008B10F2080E70C2029
:100240007EE70000D805012038740120F0B586460D
:100250002348002250F8210044682189B1F1000CA4
:1002600002EB51000FD0D4E900540023042707EB20
:10027000C006A65906EB860607EB0616AE5976456C
:1002800004D9014604E04FF00000F0BD11D202464F
:10029000A1EB020000EBD07003F1010302EB600060
:1002A000DBB280B2102BE2D96046F0BD401E80B2B6
:1002B00001E06FF0030202EBC001615801EB810124
:1002C00007EB01116B5807EBC001615801EB81018D
:1002D00007EB011169588B42E7D10028E6D1F0BD48
:1002E000387401202DE9F74F5B4C1746804654F8CF
:1002F000271000688AB089694FF0000B084011464A
:10030000FFF7A4FF1FFA80FA54F82700406800891D
:100310000590504571D0D8E90210CDE9061082E071
:1003200080B200EB80090822089002EB0910085CFB
:100330000B99B1EB101F03D00321B1EB101F62D159
:1003400098F8041000F00F02C1F383018A4201D033
:10035000000758D1DDE90612C8E9021255F8270056
:100360004FF0010B41680B680C2101EB09115A5841
:10037000A2B18DF800704268136803EB0912CDE951
:10038000012800F10C02039200228DF81020406831
:1003900000684158684688470A285BD000242E4AE6
:1003A00052F8270040680168142001EB091100EBA6
:1003B000C4000858C3B2042B03D010F0FF0F1DD0A7
:1003C0001DE0102000EBC4000144099008F1080072
:1003D00000F0E2FA054620480E4650F82700406833
:1003E0000168099801EB0911084400F043FB4540FE
:1003F000354304D04FF0000B08E00FE00824641CE4
:10040000A4B2082CCBD3BBF1010F0AD00AF1010032
:1004100005991FFA80FA8A4505D108460DB0BDE856
:10042000F08F0898FAE70C4D042303EBCA0055F847
:100430002720516892694C680968205800EB8004B5
:1004400003EB0413D8F80040CB5814401340A342E8
:100450003FF466AF0598E1E738740120F0B5074630
:100460001648002250F8210044682189B1F1000C9F
:1004700002EB51000ED0D4E90056002336F830408C
:1004800004EB840405EB04142488A4B2BC4204D910
:10049000014604E04FF00000F0BDFDD20246A1EBA2
:1004A000020000EBD07003F1010302EB6000DBB24D
:1004B00080B2102BE2D96046F0BD000038740120F4
:1004C0002DE9F05F044670484FF6FF7E002250F899
:1004D000240075464068B0F80880D0E900100BE0B1
:1004E00002EB820301EB03131B689EB2AE4201D202
:1004F0009DB21746521C92B24245F1D307800123A8
:1005000023E00022F44600EBC30B18E03BF8086C34
:1005100002EB820506EB860601EB051501EB0616DC
:10052000D5F800A036881FFA8AF5B6B2B54204D9CC
:10053000654502D21FFA8AFC1746521C92B2424508
:10054000E4D320F833705B1C9BB24345D9D3DFF86A
:1005500038B14FF0FF3A56465BF8242052681589AF
:10056000002209E002EB820301EB03135B68B34254
:1005700000D21E46521C92B2AA42F3D300231A465E
:100580000DE003EB830701EB07177F68B74204D147
:1005900000EBC207521C92B27B605B1C9BB2AB4269
:1005A000EFD32CE00023564600EBC20813E058F8C6
:1005B00004CC03EB83070CEB8C0C01EB071701EB6E
:1005C0000C1C7F68DCF804C0674502D9B74200D232
:1005D0003E465B1C9BB2AB42E9D300230DE003EB2C
:1005E000830701EB07177F68B74204D100EBC2070E
:1005F000521C92B27B605B1C9BB2AB42EFD3AA420F
:10060000D0D35BF824005F468068002839D00025ED
:100610004FF004082FE04E46416865F30F0608EBE3
:10062000C50064F317460E5057F82410002389685C
:1006300049680A1801211548E1F790FA57F8241083
:1006400005EB45038968496841F8350057F82410DF
:1006500089680A6808EB8301515811B146F0807926
:1006600005E0082101EB830126F080795158E1F77C
:100670008DFA6D1CADB257F8240080680189A9423B
:10068000C9D8BDE8F09F000038740120990A02081B
:10069000017C002904D08068017941F0400101719A
:1006A000002070477CB50546A9680879C0F383042B
:1006B000083122466846E0F70AF900216A4609E057
:1006C000601A1044AE6810F8013C01F10800335480
:1006D000491CC9B2A142F3D300207CBD30B58BB018
:1006E0000446A068007A502849D1227809A922201E
:1006F00001F0CEF8A0680088000A0890214D9DF80E
:100700002410284602F086FA9DF82010884236D040
:100710009DF8242008A9284603F052F99DF82410DA
:10072000684600F057F9059800F06040FF300590EA
:100730009DF82010049861F31C0004909DF824108B
:10074000684600F077F922780AA90D2001F0A0F898
:100750000D4C9DF828206946204601F099F89DF837
:1007600020108DF813109DF828206946204603F0CC
:1007700027F99DF828204021044802F0A5FA0BB083
:100780000A2030BD22000200450008108700080042
:10079000F0B589B024216846E0F7F5F84FF48060A1
:1007A0000590E2F7F5FB002211462020E1F71EF943
:1007B0001A4C2021002260600846E1F717F9A0607A
:1007C0000024174D671EFF2655F82400A8B12046C7
:1007D000FFF776FE55F824003946406AE1F7C4F881
:1007E00055F82400467355F824000C30E2F7CDFB91
:1007F00055F82400406AE1F70BF9641CE4B2212C9F
:10080000E2D36A4600210748E1F760F96A46002111
:100810000548E1F75BF909B00020F0BDD8050120DB
:10082000387401201D0B0208A50E020810B588B00F
:1008300004460623174A012100200094FFF766FCB6
:10084000214602A800F0C6F8002003904FF6FF7082
:10085000049011480590069820F0005006900698E4
:1008600020F0804006900D48069960F31C01069127
:10087000079921F000510791079921F080410791D4
:10088000079960F31C010791214602A800F0D2F8F5
:1008900008B010BD683A03080000FF1F0000EF1801
:1008A0002DE9F05F834650688946C0F30341C900D3
:1008B000C0F3035208390A44010A521A55B2C0F370
:1008C0000362D200083A02EB1070401A44B20120D1
:1008D00088404FF0000A401E514600FA05F62246B5
:1008E000DFF782FD0746DBF80000884630405146BE
:1008F000621B03D52A1BDFF78AFD01E0DFF774FDD9
:10090000D9E90032BB4322EA080203430A43C9E99A
:100910000032BDE8F09F2DE9F05F834650688A46BB
:10092000C0F30341C900C0F3035208390A44010A65
:10093000521A54B2C0F30362D200083A02EB1070AC
:10094000401A45B201208840401EC11707460E4696
:100950002A46DFF749FD8046894638463146224619
:10096000DFF742FD06460F46DBE9000100EA08001A
:1009700001EA0901621B03D52A1BDFF748FD01E0EC
:10098000DFF732FDDAE90032B343BA4303430A43E7
:10099000CAE90032BDE8F09F70B505464868C0F36B
:1009A0000361C900083901EB1072010A501A42B202
:1009B00001208840401E1446C117DFF715FD02468E
:1009C000D5E9000310402246BDE870401940DFF72A
:1009D0001EBD000070B50C4D0C46064655F82400AF
:1009E0004FF0FF31406AE0F7BFFF55F8241018229E
:1009F00030460C31DFF76BFF55F82400406AE1F711
:100A000007F8002070BD00003874012070B5084D53
:100A100004464FF0FF3155F82400406AE0F7A4FF88
:100A200055F824100C7B486AE0F7F2FF204670BDB1
:100A30003874012070B50E4D0C46064655F824005A
:100A40004FF0FF31406AE0F78FFF55F8240018227D
:100A500031460C30DFF73BFF55F824000C30E2F74D
:100A600094FA55F82400406AE0F7D2FF002070BDE8
:100A70003874012041680068C1F30342D200C1F319
:100A80000353083A13440A0A991A012393405B1E40
:100A90008B401840C840704770B5044600681D4D33
:100AA000C10120D520F08070C0F30741206055F8C7
:100AB000211080B28968496851F83000E1F778F870
:100AC00020680826C0F3074180B255F8211000EBDA
:100AD000400306EB83038A6811685268C95852F8CC
:100AE0003000E1F753F80C488068E0F767FF002812
:100AF0000FD02068C0F3074180B255F8212000EBE9
:100B000040009268126852F82000BDE8704000F082
:100B10007BB970BD38740120D80501201FB5214E66
:100B20002148E2F72FFA2148E2F734FA002456F878
:100B3000240068B3406A4FF0FF31E0F715FF1B480F
:100B4000016856F82400026AC56901EA02031540EB
:100B5000AB421ED115480DF1040C001D0DC80091CB
:100B60008CE80D00224601216846FFF7BBFB0546D5
:100B700056F82400406AE0F74BFF56F8240040681E
:100B80000089A84208D028462246694600F010F89D
:100B900002E0406AE0F73CFF641CE4B2212CC6D3BB
:100BA000BEE7000038740120F0770120C0750120F5
:100BB0002DE9FF5F08311646002500EB800A4FF053
:100BC000100B4FF001090391384850F82600406897
:100BD00001680BEBC50001EB0A110C1820790628FF
:100BE0005AD2DFE800F059032E505A5A2068010EFD
:100BF0000FD0B9EB106F50D121460398FFF7CCFE10
:100C0000E3F771FF00EE100A3146206800F04EFD58
:100C100043E021460398FFF7BFFE01466068C0F33A
:100C20000342D200C0F30353083A1A44000A131ACD
:100C300009FA00F2521E9A403346206802F008FD7D
:100C40002BE021460398FFF7A7FE0746029660684F
:100C50008846C0F30341C900C0F3035208390A446F
:100C6000C0F30721521A09FA01F0C117401E41F1E1
:100C7000FF31DFF7B9FBCDE9000143463A46206872
:100C800001F0F6FB09E00A48224600EB06100830A6
:100C90002168FFF740FE00E008256D1CEDB2082D2D
:100CA00092D304B00020BDE8F09F0000387401200A
:100CB000D07501202DE9F04F8846524989B001EBEB
:100CC000081700214F4A39607960B96002EB0816B5
:100CD0000D464FF0100BA2F5CC7A00EB80090836D8
:100CE000F9605AF82800406801680BEBC50001EB79
:100CF00009110C18207906282ED2DFE800F02D0308
:100D00001025292E424605A9206800F0C1FD0228C1
:100D100023D13146224605A8FFF7C2FD1DE041461A
:100D2000206800F03BFDC0B2082816D8A8B14246A2
:100D300006A9206800F0ACFD02280ED131462246FB
:100D400006A8FFF7E8FD08E0314622462068F8E7EC
:100D5000224631461046DFE708256D1CEDB2082D0E
:100D6000BFD35AF828000823544641680A6803EBA9
:100D700009110423515C3A7961F385023A714168A3
:100D80000A6803EB09115158396041680C220B685D
:100D900002EB09115A58A2B18DF80080426813681D
:100DA00003EB0912CDE9012700F10C0203920122A5
:100DB0008DF81020406800684158684688470A2826
:100DC0001CD054F828004FF0FF31406AE0F7CCFD0A
:100DD00054F828305A6952B11046196901E04008A8
:100DE0004900C407FBD03868904308433860586A0C
:100DF000E0F70EFE3846E2F7E9F8002009B0BDE85A
:100E0000F08F0000D075012070B5244D0C46C0F362
:100E1000074255F824100978914201D0072070BD8F
:100E200080B22146FFF71AFB81B255F824004068D2
:100E300002898A4201D1052070BD426832F83150E2
:100E4000016805EB8502082000EB0210085C01092F
:100E500003D00121B1EB101F01D10B2070BD204642
:100E6000FFF7D4FD012816D00D4E4FF0FF31B068CA
:100E7000E0F77AFD09493078883121F8305001EBEC
:100E8000C001401C8C7000F01F0030707068E0F7EB
:100E9000BFFD002070BD102070BD0000387401201F
:100EA000D80501200E4C0F4F4FF0FF380120DFF71F
:100EB000ADFF41466068E0F757FD607857F83010A5
:100EC000401C00F01F0060708EB2C1F30745A0689F
:100ED000E0F79EFD29463046FFF7ECFEE6E700000E
:100EE000D8050120C074012010B588B00446042341
:100EF000184A012102200094FFF708F9214602A8B0
:100F0000FFF768FD48F2810003904FF6FF700490F0
:100F100000020590069820F000500690069840F0D8
:100F200080400690069800F0604080300690079858
:100F300020F000500790079840F0804007900798F5
:100F400000F06040FF300790214602A8FFF772FDD5
:100F500008B010BDA43C030810B588B004460123B6
:100F6000164A194608200094FFF7D0F8214602A837
:100F7000FFF730FD38200390FF20049000200590FB
:100F8000069840F000500690069840F08040069089
:100F9000069860F060400690079840F00050079077
:100FA000079840F080400790079860F060400790F5
:100FB000214602A8FFF73EFD08B010BD742F0308BC
:100FC0002DED048B4FF0FF36124C9FED139ADFEDA1
:100FD000138ADFED139A04F10C05E2F783FA00F0AF
:100FE00079F894ED011A3146A068C1EE000A20EEAE
:100FF000890AF0EE480AB0EE408A00EEA88AE0F7CF
:1010000013F828EE290A85ED010AA068E0F742F8F6
:10101000E3E7000034060120CDCC4C3D3333733F71
:101020000000C84238B568460AF0F4FD009888B15F
:10103000E0F73AFD044631210098E0F76BFD00B17E
:10104000FEE768460AF0E6FD0028FAD0214600983F
:10105000E0F760FDE0F714FDE0F76EFD38BD00003D
:1010600010B5164C2078002827D101202070144894
:10107000DFF7FEFFA06073B600F02CF884ED010AE4
:1010800063B624210F48DFF77EFC0E4C0820224671
:10109000A06100210C48E0F719FD1020A061224654
:1010A00000210A48E0F712FD3020A0612246BDE889
:1010B000104000210648E0F709BD10BD34060120AC
:1010C00034F80208007A0120C10F02082D1102082D
:1010D0002510020810B5DFF7C3FE0446002141F2D7
:1010E0008830491C8142FCD3DFF7BAFE001B00EEBA
:1010F000100AB8EE400A10BD70B50B4C0546617081
:101100004FF0FF31A068DFF78FFF04F10C00690892
:10111000018000214180A068DFF7BCFF2846BDE8C0
:101120007040E3F717BB0000340601200E4C4FF06F
:10113000FF37A4F10C05DFF7A5FE06462088DFF790
:1011400065FE68780028F6D0E3F706FB3946A86804
:10115000DFF76AFFDFF796FE2188401A801B608068
:10116000A868DFF797FFE6E7400601202DE9F05F6A
:101170006E4E04464FF0000A56F824004FF0060B5E
:101180004FF0040840684FF0080990B300272AE0A8
:10119000406807EB47054FF0FF3150F82500DFF7B7
:1011A00043FF56F8240008EB850341684868096846
:1011B000C35A03EB830308EB8302895809EB8502CA
:1011C000815056F8241049684A680BEB850122F8D3
:1011D00001A056F824004068406850F82500DFF769
:1011E00059FF7F1CBFB256F8240040680189B942FC
:1011F000CED856F824008068B0B300272EE04068AF
:1012000007EB47054FF0FF3150F82500DFF70CFFE3
:1012100056F8240008EB8503816848680968C35ABA
:1012200003EB830308EB8302114491ED000A09EB01
:101230008501084480ED000A56F8241089684A6840
:101240000BEB850122F801A056F824008068406865
:1012500050F82500DFF71EFF7F1CBFB256F82400B0
:1012600080680189B942CAD856F82400C068E8B33A
:10127000002552E040684FF0FF3100EB0510006898
:10128000DFF7D2FE56F8241009EB0513C968496848
:1012900021F803A056F8240008EB0511C36858682C
:1012A0001B6830F801C009EB0C1C33F80C300BEB59
:1012B000051C20F80C3056F82400D0F80CC0DCF8DF
:1012C0000400DCF80070435A08EB0311795871B13F
:1012D0004FF00C0C0CEB051C50F80C0090B109EB16
:1012E0000312BA5A72B1DFF7ADFA0BE01BE00C2122
:1012F00001EB0511405828B109EB0311795A09B1E6
:10130000DFF71FFB56F82400C068406800EB0510AB
:101310000068DFF7BFFE6D1CADB256F82400C06850
:101320000189A942A6D80020BDE8F09F34730120AE
:101330002DE9F047804662488A46624F0178089C52
:101340001D4616464FF0000949B180F80090494605
:10135000002047F82010401C80B22028F9D3202C10
:1013600002D30C20BDE8F08757F8240020B10178A3
:10137000414517D00D20F5E714210120E2F724FFA5
:1013800047F82400002876D080F8008057F8241011
:10139000C1F8049057F82410C1F8089057F82410A9
:1013A000C1F80C905FEA0A0008D0012826D0102866
:1013B00043D0BAF1110F5FD00B20D3E757F82400C8
:1013C0004068C8BB0C210120E2F7FEFE57F824104C
:1013D0000028486071D0066057F824000C2140684E
:1013E00005812846E2F7F0FE57F8241000284968E6
:1013F000486062D0204601F0CFF95CE057F8240045
:101400008068C8B90C210120E2F7DEFE57F82410ED
:10141000886080B3066057F824000C21806805813D
:101420002846E2F7D1FE57F824108968486010B3C7
:10143000204600F079F83EE022E057F82400C0682A
:10144000F0B90C210120E2F7BFFE57F82410C86064
:1014500088B1066057F824001021C068058128462D
:10146000E2F7B2FE57F82410C968486018B1204668
:1014700000F05CFB1FE020E057F82400006908B191
:101480000F206FE70C210120E2F79EFE57F8241091
:10149000086190B1066057F82400022100690581B7
:1014A0002846E2F791FE57F824100969486020B1F8
:1014B000204602F077F9002054E70E2052E70000A2
:1014C000D405012034730120F0B58646154800226A
:1014D000042550F82100114686683389D6E9007446
:1014E0009C4602EB530000EB400605EB8606A65B2C
:1014F00006EB860637F82660B6B2764501D9034674
:1015000001E00DD20246A3EB020000EBD07001F126
:10151000010102EB6000C9B280B21029E3D9604634
:10152000F0BD0000347301202DE9F05F31494FF622
:10153000FF7251F820008068D0E90047B0F80890A9
:1015400000200AE000EB800154F821108BB2934296
:1015500001D28AB20546401C80B24845F2D3BD8014
:101560002548DFF785FD386005EB850004EB80003A
:101570004FF0000B90ED010A012087ED020AA7F859
:1015800006B031E008EB480A00204FF6FF7C07EB7D
:101590008A0614E036F8083C00EB800103EB830375
:1015A00054F8211034F823308AB29BB29A4204D9FD
:1015B000624502D21FFA81FC0546401C80B24845B4
:1015C000E8D3B5800C48DFF753FD47F82A0005EB58
:1015D000850004EB800090ED010A08F1010086ED22
:1015E000020AA6F806B080B280464845CAD3BDE8D4
:1015F000F09F00003473012004F6020808B59FED47
:10160000050A0A468DED000A694600F041F99DED94
:10161000000A08BD0000C07FF0B5234F054601EB6E
:10162000410157F8250089B016468068406800EBF4
:1016300081044FF0FF312068DFF7F6FC94ED020AD9
:1016400002208DED070A307057F8250010228168BE
:101650000B68A18801EB810102EB81015958E1B1CE
:101660008DF80050816804AF0B68A18801EB8101FF
:1016700053F821100191002107AB03938DF8081056
:10168000A31D87E84A0080680168A08800EB8000FD
:1016900002EB80000958684688472068DFF7FAFCAB
:1016A0009DED070A09B0F0BD3473012008B50A4664
:1016B0008DED000A694602F083F908BD2DE9F0417D
:1016C000DFF8D480064601EB410158F8260088B0C7
:1016D0001D4680681746406800EB81044FF0FF31DB
:1016E0002068DFF7A1FC58F82600102281680B68FB
:1016F000A18801EB810102EB81015958E1B18DF81C
:10170000006081680B68A18801EB810153F821100A
:10171000019101218DF80810A11D05910021069568
:10172000CDE9037180680168A08800EB800002EBBE
:1017300080000958684688472878072826D058F836
:101740002600A1880822806801EB810102EB81025A
:10175000006897ED000A0244D2ED000AF4EEC00AD8
:10176000F1EE10FA01DD05200FE00C2202EB810101
:101770000844D0ED000AF4EEC00AF1EE10FA01D2EE
:10178000062002E084ED020A042028702068DFF7BA
:1017900081FC08B0BDE8F0813473012030B5124DF2
:1017A0000C46C0F3074255F824100978914212D133
:1017B000010E03D00121B1EB106F01D1042030BD27
:1017C00080B2214600F082F955F8241080B2C96831
:1017D0000A89824201D1002030BD4968062202EB0D
:1017E0000010085A30BD00003473012000207047FB
:1017F00038B5044600212623144A08460094FFF712
:1018000097FD1723124A102100200094FFF790FD46
:101810002023104A112100200094FFF789FD0E4873
:101820004470032C02D0042C05D008E00BA1801CCE
:10183000DEF77AFF03E00FA1801CDEF775FF22467A
:10184000BDE838400449114802F0BAB8F02F030847
:10185000E8330308E83203081C0901203630343726
:10186000204D6F6E69746F722031205365747469F6
:101870006E67730036303437204D6F6E69746F7247
:1018800020322053657474696E6773000A0000107B
:10189000F8B50E46324D144601218DF8001055F86A
:1018A0002410C0F307420978914201D00D20F8BD01
:1018B000010E07D0012917D0102928D0112938D0BE
:1018C0000B20F8BD80B2214600F036FF55F82410F9
:1018D00080B249680989814236D0C1B26A46204641
:1018E00001F0AAF9306037E080B22146FFF7ECFD45
:1018F00055F8241080B289680989814224D0C1B288
:101900006A462046FFF788FE86ED000A24E080B292
:10191000214600F0DBF855F8241080B2C968098927
:10192000814211D0C1B26B463246204600F030FAF7
:1019300012E080B2214601F00BFF55F8241080B26E
:1019400009690989814201D10A20F8BDC1B26B46FB
:101950003246204601F082FF9DF80000F8BD0000ED
:10196000347301202DE9F041274D14460E4655F8F9
:101970002410C0F307420978914202D00D20BDE83F
:10198000F081010E4FF004074FF00C0803D001293D
:101990001AD00B20F3E780B2214600F0CDFE55F8B7
:1019A000241080B249680A89824218D04A6800EB44
:1019B000400007EB8000105A096800EB800208EB3A
:1019C0008200085830601CE080B22146FFF77CFDA1
:1019D00055F8241080B289680A89824201D10A2010
:1019E000CDE74A6800EB400007EB8000105A096819
:1019F00000EB800208EB8200084490ED000A86EDBF
:101A0000000A0220BBE70000347301207FB50C46BA
:101A10000A7805466946FFF73BFF9DF80C00012652
:101A200008B1029808E08DF80C60BDF80210BDF80E
:101A30000000E2F7C9FB0290F0B3207AF8B1BDF8DC
:101A40000410BDF80020481C521E1040BDF80620AE
:101A5000904201D107202DE0BDF80220029801FB41
:101A60000200E168DEF7EEFEBDF80400BDF80010EC
:101A7000401C491E0840ADF8040004201AE0BDF8DF
:101A80000400BDF80610884202D1A069067015E076
:101A9000BDF80220029801FB0201E068DEF7D2FEE9
:101AA000BDF80600BDF80010401C491E0840ADF806
:101AB00006000220A16900E006E00870227869466D
:101AC000284601F07DFF7FBD0E20F3E7F0B5844688
:101AD00015480022042550F821001146C6683389B4
:101AE000746836681F4602EB530005EB001E34F89D
:101AF0000EE006EB0E1EBEF800E01FFA8EFEE64575
:101B000001D9034601E00DD20246A3EB020000EB2F
:101B1000D07001F1010102EB6000C9B280B210295E
:101B2000E3D93846F0BD0000347301202DE9F05FA1
:101B30003F494FF6FF7251F82000C068D0E90057C6
:101B4000B0F808A0002009E005EB001109688BB28D
:101B5000934201D28AB20646401C80B25045F3D36C
:101B6000BE803448DFF784FA4FF0000B386005EB95
:101B70000614A7F808B02089F880218951B1012006
:101B8000E2F722FBF86058B1616831B12289DEF7D3
:101B900059FE05E0C7F80CB002E02189DEF7D1FE5E
:101BA000012040E000204FF6FF7307EB081413E01C
:101BB00034F80CCC05EB001105EB0C1C0968BCF8E3
:101BC00000C08AB21FFA8CFC624503D99A4201D246
:101BD0008BB20646401C80B25045E9D3A68015481A
:101BE000DFF746FA206005EB0610A4F808B001897B
:101BF000E18001895A46814661B10120E2F7E4FAA9
:101C0000E06068B1D9F8041031B1B9F80820DEF706
:101C100019FE05E0E26003E0B9F80810DEF791FE76
:101C200008F1010080B280465045BBD3BDE8F09F6B
:101C30003473012004F6020810B5044611482178D7
:101C400001F0F2FD0146E068DEF76EFD207A18B182
:101C5000A1690720087010BD2178172000F0DAFF75
:101C6000C1B2094800F0D6FF21788842F3D1054877
:101C7000401E01F0D9FD0146E068BDE81040DEF7E6
:101C800053BD0000030000114400080010B50446D5
:101C9000207A00280AD121780D2000F0BBFFE168EE
:101CA000C2B2BDE810400248FFF7F2BD10BD00000F
:101CB0003B0008101CB50146CC68087A002815D1F5
:101CC0004868A0F180501D3811D0012811D0022899
:101CD00012D0032813D00020002807D00A786946C4
:101CE000FFF7D6FD6946204600F0B2F81CBD054856
:101CF000F2E70448401CEFE70248801CECE701488B
:101D0000C01CE9E7190000107FB5054600200290CD
:101D100003900024EE68287A002836D12A78694694
:101D20001A48FFF7B5FD072202A96846DEF7D0FC86
:101D300000B1012415482A786946401CFFF7A8FD28
:101D4000072202A96846DEF7C3FC08B1641CE4B2AE
:101D50000E482A786946801CFFF79AFD072202A9DF
:101D60006846DEF7B5FC08B1641CE4B207482A787F
:101D70006946C01CFFF78CFD072202A96846DEF702
:101D8000A7FC08B1641CE4B234717FBD19000010D7
:101D90002DE9F0432D4F054687B057F825001E4624
:101DA0009146C068406800EB01144FF0FF31206895
:101DB000DFF73AF957F82500A1880822C06802EB3E
:101DC00001120068825A0AB1E1680FE04FF004087E
:101DD00008EB01114058DEF7CBFC024657F825000E
:101DE000A388C068016808EB031009584846DEF76D
:101DF00029FD0220307057F82500A388C1680A68C1
:101E00000C2101EB0313D258D2B18DF80050C268F7
:101E1000A388126802EB03121268019200228DF867
:101E2000082004F108020592A21D0696CDE903924E
:101E3000C068A288006801EB0211415868468847D3
:101E40002068DFF727F907B0BDE8F083347301207D
:101E50002DE9F0410446087800250204487842EA5A
:101E600000208A780243C878070642EA10260879DB
:101E700047EA004346EA104248798F79060E43EA62
:101E8000002007431643B80F40EA8600C0F30B0258
:101E900010A12046DEF7CEFAC6F346402071C6F305
:101EA000862060710D4827F04042824200D90246E8
:101EB0000BA1A01DDEF7BEFAE5732046DEF758FC45
:101EC0000F2805D22046BDE8F04107A1DEF72CBC63
:101ED000BDE8F0812530347500000000FFC99A3B51
:101EE0002530397500000000496E76616C69642008
:101EF00050494E0001460148FFF788BD1800081000
:101F000010B504460D48217800F084FE217A19B1FD
:101F1000A1690720087010BDB0F5302F08D0B0F5CA
:101F2000E02F05D0E068BDE8104005A1DEF7FCBB5E
:101F3000E068BDE8104004A1DEF7F6BB0900080028
:101F4000322E342047487A00393030204D487A000C
:101F500070B504461D48217801F066FC0146E06832
:101F6000DEF7E2FB207A18B1A1690720087070BD86
:101F7000164D17496068174B6D1E884210D101221B
:101F80001146184600F04FFE0028F0D02178284670
:101F900001F04AFC0146E068BDE87040DEF7C4BBD2
:101FA0000B49491C8842E2D102220121184600F067
:101FB0003AFE0028DBD02178284601F035FC0146A6
:101FC000E068BDE87040DEF7AFBB00000300081119
:101FD0000D0008105F00080010B50446207A0028A4
:101FE00003D0A1690720087010BDE1F739F9014657
:101FF0000029F9D0E068BDE810401022DEF722BCCD
:1020000001460148FFF702BD2400081001460148BF
:10201000FFF7FCBC2600081010B50446207A002803
:102020000AD12178054800F0F5FDE168C2B2BDE8AB
:1020300010400420FFF72CBC10BD00004400080035
:1020400010B50446207A00280FD121780B4800F003
:10205000E1FDC2B21620E168FFF71AFCE0684FF01C
:10206000000201680B0601D4026010BD21F080015E
:102070000160E0685A29F8D9026010BD44000800E8
:1020800010B50446207A00280AD12178054800F0CE
:10209000C1FDE168C2B2BDE810400720FFF7F8BB00
:1020A00010BD00004400080010B50446207A002846
:1020B0000AD12178054800F0ADFDE168C2B2BDE863
:1020C00010400120FFF7E4BB10BD000044000800F1
:1020D00010B50446207A00280ED12178074800F078
:1020E00099FDC2B21620E168FFF7D2FBE0680178E3
:1020F000090601D50021016010BD00004400080060
:1021000010B50446207A00283DD160681E4AA0F52B
:102110000021463916D0A0F5002147391DD0A0F581
:1021200000214A3924D0A0F500214B392BD1217848
:10213000104600F06FFDE168C2B2BDE81040062015
:10214000FFF7A6BB2178104600F064FDE168C2B23B
:10215000BDE810400220FFF79BBB2178104600F03D
:1021600059FDE168C2B2BDE810400320FFF790BB03
:102170002178104600F04EFDE168C2B2BDE8104083
:102180000520FFF785BB10BD440008001CB50446C0
:10219000207A002832D1227801A91F48FFF778FB66
:1021A0009DF80420FF2A30D069460A20FFF770FB13
:1021B000E1689DF804000870E168009848709DF897
:1021C000042008210B2000F02EFD28B1E0680179E1
:1021D00041F00101017104E0E068017921F00101A1
:1021E00001719DF804204FF400610B2000F01BFDED
:1021F00028B1E068017941F0100101711CBDE0686F
:10220000017921F0100101711CBDE168FF20087007
:10221000E168002048701CBD4400080030B587B05C
:102220000446207A002823D0124D22786946284699
:10223000FFF72EFBE0680168CDF805104068CDF887
:10224000090022786946284601F0BAFB6D1C227805
:1022500069462846FFF71CFBE0680168CDF80510C9
:102260004068CDF8090022786946284601F0A8FBAD
:1022700007B030BD0500081010B50446E168207AAB
:10228000002810D1C869B0F5E02F0DD0B0F5302F7F
:102290000AD0B0F5981F07D022780848FFF7F8FA5F
:1022A00021691820088010BD04482278401CFFF7DF
:1022B000EFFA21691B20088010BD000005000810FE
:1022C00010B5C468017A002906D10178034800F0EE
:1022D000A1FCA1780843A07010BD00008B0008008D
:1022E00038B50446E568207A002816D12278694678
:1022F0000A48FFF7CDFA094821782E3000F08AFC11
:10230000E870064821782D3000F084FCA8709DF814
:102310000020291D0248FFF7BBFA38BD6000080005
:1023200019000010017A002905D1C1680278891CC2
:102330000148FFF7ADBA70478A0008001CB5044693
:10234000207A002808D1227869460448FFF7A0FACD
:102350006946E068FFF77CFD1CBD00003C000810EA
:1023600010B592B0C468017A002907D10278694695
:102370000348FFF78DFA9DF80000207112B010BDE0
:102380003A00081010B592B00446207A002812D105
:10239000227811A90948FFF77BFA22786946084894
:1023A000FFF776FA9DF84410684600EBC101891CDE
:1023B000E068FFF74DFD12B010BD00008A00080074
:1023C0003F00081030B587B00446207A002821D09D
:1023D000114D227869462846FFF75AFAE0680168ED
:1023E00004914068059022786946284601F0E8FA91
:1023F0006D1C227869462846FFF74AFAE0680168B2
:10240000CDF813104068CDF81700227869462846A9
:1024100001F0D6FA07B030BD0500081070B5C568E8
:10242000007A002812D028780B280FD20024084EFA
:1024300009E0C4EBC4004119491C06EB0410FFF786
:1024400007FD641CE4B22878A042F2D870BD0000F9
:102450008485012010B5C468017A002904D101786F
:10246000024800F0D7FBA07010BD00008C000800EF
:102470002DE9FF4107460AA890E870002046AC46C7
:10248000CDE9002308E05FEA5C0C4FEA30000199D7
:1024900092184941CDE90021C107F4D031463846B0
:1024A000FFF77CF9C0B2082819D8C0B1324602A99A
:1024B0003846FFF7EDF9DDE9022322EA040123EAB9
:1024C0000500DDE9002311431843CDE90010324631
:1024D0006946384601F074FA04B0BDE8F08107207F
:1024E000FAE700002DE9F041274F054688B057F87C
:1024F00025001E469046C068406800EB01144FF06E
:10250000FF312068DEF790FD57F82500A388C168E9
:102510000A680C2101EB0313D258D2B18DF8005098
:10252000C268A388126802EB0312126801920122AA
:102530008DF8082004F108020592A21D0696CDE947
:102540000382C068A288006801EB02114158684606
:1025500088473078072811D057F82500A288C0682E
:102560000168082000EB02100A5A2AB14146E068CF
:10257000DEF768F9042000E0072030702068DEF7FD
:1025800089FD08B0BDE8F0813473012038B50446F8
:10259000694622781320FFF77BF9BDF800007138F7
:1025A00001B200914FF46170814201DD009003E0BF
:1025B0000648814200DA0090207A002805D1BDF952
:1025C0000000E16800F56170086038BD7CFCFFFF29
:1025D00038B50446694622781020FFF759F900986B
:1025E000C0F30061C0F30B00227A002A04D121B1AC
:1025F000E16800F56170086038BDE168C0F56170A0
:10260000086038BD38B50446694622781120FFF7C6
:102610003FF9BDF80000713800B200904FF4E1615D
:10262000884201DD009103E00949884200DA009107
:10263000207A002807D1BDF90000002804DAE168FB
:1026400000F56160086038BDE168086038BD0000D1
:10265000F8F8FFFF38B50446694622781220FFF7E4
:1026600017F9BDF80000713000B200904FF4E1613D
:10267000884201DD009103E00949884200DA0091B7
:10268000207A002807D1BDF90000002804DAE168AB
:1026900000F56160086038BDE168086038BD000081
:1026A000F8F8FFFF38B50446694622780F20FFF797
:1026B000EFF80098C0F30061C0F30B00227A002A03
:1026C00002D111B1E168086038BDE168C0F5616010
:1026D000086038BD38B50446694622781420FFF7F3
:1026E000D7F8BDF80000713001B200914FF461706D
:1026F000814201DD009003E00648814200DA00904B
:10270000207A002805D1BDF90000E16800F561706C
:10271000086038BD7CFCFFFFF8B50C461546064640
:10272000114600F077FAA04300902A4669463046E9
:1027300001F046F9F8BD0000F0B5864615480022C4
:10274000042550F82100114646683389D6E9007403
:102750009C4602EB530000EB400605EB8606A65BA9
:1027600006EB860637F82660B6B2764501D90346F1
:1027700001E00DD20246A3EB020000EBD07001F1A4
:10278000010102EB6000C9B280B21029E3D96046B2
:10279000F0BD0000347301202DE9F05F2F494FF6A2
:1027A000FF7251F820004068D0E90047B0F8089067
:1027B00000200AE000EB800154F821108BB2934214
:1027C00001D28AB20546401C80B24845F2D3BD8092
:1027D0002348DEF74DFC386005EB850004EB8000F4
:1027E0004FF0000B4068B860A7F806B001202FE05A
:1027F00008EB480A00204FF6FF7C07EB8A0614E03E
:1028000036F8083C00EB800103EB830354F82110F9
:1028100034F823308AB29BB29A4204D9624502D27C
:102820001FFA81FC0546401C80B24845E8D3B580BC
:102830000B48DEF71DFC47F82A0005EB850004EB8A
:1028400080004068B06008F10100A6F806B080B2D0
:1028500080464845CCD3BDE8F09F0000347301208A
:1028600004F6020870B50446207A00281ED02278AB
:102870004FF480310B2000F027FAE0680068002850
:1028800014D14FF40055227829460B2000F0CBF9E3
:1028900000280BD0227829460B20FFF73DFF227835
:1028A000BDE870400021232000F0CCBE70BD0000C8
:1028B00070B50446E068217A002913D001680A48FF
:1028C00088430FD14FF40045227829460B2000F0B1
:1028D000AAF9002806D122782946BDE870400B20CD
:1028E00000F0F2B970BD00000000030370B50446AB
:1028F0000D4D207A002810D00C492278881E02F055
:10290000CDFC032803D0A1690320087070BD2146C7
:102910002846BDE87040FFF779B821462846BDE853
:102920007040FFF773B800000E00001006000007AB
:1029300070B50446207A002825D0E068124E007851
:10294000F51201280FD021780D2000F063F9C2B2F2
:1029500080213046FFF7E0FE22782946BDE870402E
:102960000B20FFF7D9BE21780D2000F053F9C2B239
:102970008021304600F0A8F922782946BDE8704051
:102980000B2000F0A1B970BD5F0008007FB50446C0
:10299000207A00281DD00F4D227869462846FEF780
:1029A00077FFE0689FED0C1A0068323000EE100AE5
:1029B000F8EE400A81EE200A8DED020AF7EE000AD9
:1029C00030EEC00A8DED030A22786946284600F0F1
:1029D000F7FF7FBD13000010000048427FB504469A
:1029E000207A00281DD00F4D227869462846FEF730
:1029F0004FFFE0689FED0C1A0068323000EE100ABD
:102A0000F8EE400A81EE200A8DED020AF7EE000A88
:102A100030EEC00A8DED030A22786946284600F0A0
:102A2000CFFF7FBD120000100000484270B5044681
:102A30000D4D207A002810D00C492278C81E02F0D3
:102A40002DFC032803D0A1690320087070BD214626
:102A50002846BDE87040FEF7D9BF21462846BDE8AC
:102A60007040FEF7D3BF00000D0000100600000705
:102A70007FB50446E068217A002925D00078134EFE
:102A8000012805D0022806D0032807D0354607E0E4
:102A90000E4D6D1C04E00D4DAD1C01E00B4DED1C09
:102AA000227802A93046FEF7F3FE227869462846CE
:102AB000FEF7EEFE22786946304600F081FF22786C
:102AC00002A9284600F07CFF7FBD0000190000101D
:102AD00070B50446E568207A00281FD022784FF4AC
:102AE00000710B2000F0F0F822784FF480510B2099
:102AF00000F0EAF80A48296888430FD14FF480456E
:102B0000227829460B2000F08EF8002806D1227882
:102B10002946BDE870400B2000F0D6B870BD00001B
:102B20000000030308B5017A002921D0C1680978A3
:102B3000062904D2DFE801F00306090C1014002175
:102B4000009110E0642100910DE0FA2100910AE06B
:102B50004FF4FA71009106E04FF47A71009102E0AF
:102B60004FF4FA610091027869461C2000F028FFBA
:102B700008BD08B5C168027A002A20D00978062964
:102B800004D2DFE801F00306090C101400210091C3
:102B900010E0642100910DE0FA2100910AE04FF469
:102BA000FA71009106E04FF47A71009102E04FF45F
:102BB000FA610091027869461B2000F001FF08BD10
:102BC000017A002905D0C1680A780178014800F02F
:102BD00039BD70476000080010B50446207A00280F
:102BE00014D0227801210B2000F01DF800280DD010
:102BF00021780D2000F00EF8C2B2E0680078BDE840
:102C00001040C0F13801024800F01CBD10BD0000AA
:102C10006E00080008B500230A4669460093FEF7D7
:102C200037FE009808BD10B50C461146FFF7F2FFBD
:102C3000204000D0012010BDF0B5224F054601EB29
:102C4000410157F8250089B016464068406800EBFE
:102C500081044FF0FF312068DEF7E6F9A0680790A5
:102C60000220307057F82500102241680B68A188B7
:102C700001EB810102EB81015958E1B18DF800505F
:102C8000416804AF0B68A18801EB810153F8211062
:102C90000191002107AB03938DF80810A31D87E86D
:102CA0004A0040680168A08800EB800002EB8000C9
:102CB0000958684688472068DEF7ECF9079809B09C
:102CC000F0BD000034730120F8B50C4615460646E9
:102CD0001146FFF79FFF204300902A466946304681
:102CE00000F06EFEF8BD0000017A002903D00178E3
:102CF0000148FEF789B870470100020110B504468B
:102D000007482178FFF786FF207A002807D022782D
:102D100003480121BDE810400A3800F093BC10BD03
:102D20001E00020070B504460D4D207A002810D018
:102D30000C492278881D02F0B1FA032803D0A1695A
:102D40000320087070BD21462846BDE87040FEF79C
:102D50005DBE21462846BDE87040FEF757BE000024
:102D6000150008101400080770B50446E568207ABD
:102D7000002813D0227802210948FFF754FF0028C9
:102D80000CD02878042803D1217805200CF066FBAC
:102D900021782878BDE870400CF060BB70BD000061
:102DA0001800080070B504460D4D207A002810D098
:102DB0000C492278481D02F071FA032803D0A1695A
:102DC0000320087070BD21462846BDE87040FEF71C
:102DD0001DBE21462846BDE87040FEF717BE000024
:102DE000140008101400080770B50446207A002863
:102DF00039D0E06800781C4D032812D0042821D077
:102E0000032204210B20FFF787FC042211460B202C
:102E1000FFF782FC22782846BDE87040FF2100F0D1
:102E200011BC042211460B20FFF776FC032204217B
:102E30000B20FFF749FF22782846BDE870400521A6
:102E400000F000BC032204210B20FFF765FC0422E4
:102E500011460B20FFF738FF22782846BDE8704066
:102E6000062100F0EFBB70BD6700080038B50446CE
:102E7000207A002803D0A1690720087038BD227885
:102E800069460B48FEF704FD9DF800100D20FFF782
:102E9000C1FEC2B2064810210F30FFF7C4FE18B1C0
:102EA000E1680120086038BDE1680020086038BD95
:102EB0004400080010B58AB00446207A002833D0B8
:102EC00000214FF4002009F0A7FE00282CD0A169B2
:102ED0000720087022781548E16800F071FD21781C
:102EE000134802F075FC01281ED111482178801C7E
:102EF00002F06EFC227801A90E48FEF7C9FCE068DA
:102F000001A9007801EB800090ED010AB8EE400ABB
:102F1000E1F766FB06482178401C02F059FC0128C5
:102F200002D1A169042008700AB010BD0700080092
:102F300011000807080008107CB50446E068057811
:102F4000124E227801A93046FEF7A2FC227869468B
:102F50003046FEF79DFC002101A89DF800200CE002
:102F600043185B78AB4206D1084469444078487006
:102F70008DF8015003E0491CC9B28A42F0D822788A
:102F80006946304600F01CFD7CBD000009000810B9
:102F900010B50446217AA069002919D007210170D3
:102FA0006068A0F50020801F03D0A169032008708D
:102FB00010BD22780848E16800F002FD217807483A
:102FC00002F006FC0128F3D1A1690420087010BDAD
:102FD0000121017010BD000007000800070008076C
:102FE000F8B50446174E207A00280AD00122102195
:102FF0003046FFF791FB022210213046FFF78CFB91
:10300000F8BDE0689625016801B905600D48227891
:1030100069464338FEF73CFC9DF80000032804D0C5
:10302000042808D0E0680560F8BD01221021304670
:10303000FFF74AFEF8BD022210213046FFF744FE9A
:10304000F8BD00008700080070B5C468017A002947
:1030500003D080690721017070BD074D012128460A
:10306000FFF7D8FD206002212846FFF7D3FD216835
:103070000844206070BD0000930008002DE9FF5F48
:103080000446994D207A2E1D6F1C05F10308A5F109
:103090000609A5F1050A05F1020B00287AD060683F
:1030A000A0F5002077380C2875D2DFE800F0060D77
:1030B000151D252D353D464F5861227869468B48B0
:1030C000FEF7E6FB28465BE0884822786946801CCC
:1030D000FEF7DEFB304653E0844822786946401C08
:1030E000FEF7D6FB38464BE0804822786946C01C84
:1030F000FEF7CEFB404643E07C4822786946801DBF
:10310000FEF7C6FB48463BE0784822786946C01D7A
:10311000FEF7BEFB504633E0744822786946001D36
:10312000FEF7B6FB58462BE0704822786946401DF2
:10313000FEF7AEFB6C48401D22E06C4822786946E1
:103140000830FEF7A5FB6848001F19E067482278A1
:1031500069460930FEF79CFB6348C01E10E06348D7
:10316000227869460A30FEF793FB5F48801E07E02D
:103170005E48227869460B30FEF78AFB5A48401EAB
:10318000E2680299126851F82210594A11440D2937
:1031900031D201E039E036E0DFE801F02B070A0D1B
:1031A000101316191C1F222528000021039122E06C
:1031B000012103911FE0022103911CE003210391EF
:1031C00019E00421039116E00521039113E0062183
:1031D000039110E0072103910DE0082103910AE01B
:1031E0000A21039107E00921039104E00B210391D7
:1031F00001E00C21039122789DF80C1000F022FAD6
:1032000020780BF09BFFBDE8FF9F6068A0F50020D1
:1032100077380C28F7D2DFE800F0060C12181E24CD
:103220002A3037424D58227803A92846FEF730FB52
:1032300055E0227803A93046FEF72AFB4FE02278BA
:1032400003A93846FEF724FB49E0227803A940464B
:10325000FEF71EFB43E0227803A94846FEF718FB61
:103260003DE0227803A95046FEF712FB37E02278B2
:1032700003A95846FEF70CFB31E01B48227803A94E
:10328000401DFEF705FB2AE01748227803A9001F1E
:10329000FEF7FEFA9DF80C00083803901FE0124874
:1032A000227803A9C01EFEF7F3FA9DF80C00083837
:1032B000039014E00C48227803A9801EFEF7E8FA78
:1032C0009DF80C000838039009E00748227803A90C
:1032D000401EFEF7DDFA9DF80C0008380390E16807
:1032E0009DF80C0008608EE7240008002B000810F1
:1032F000CCFFF7EE70B504460D4D207A002810D0B3
:103300000C492278881D01F0C9FF032803D0A16968
:103310000320087070BD21462846BDE87040FEF7C6
:1033200075BB21462846BDE87040FEF76FBB000024
:10333000150008101400080730B585B0044604A92C
:1033400022781948FEF7A4FA184D9DF81020694616
:103350002846FEF79DFA207A70B1E06890ED000AE9
:10336000B8EE400A8DED010A9DF810206946284606
:1033700000F026FB05B030BD9DED000ADDED030A2F
:103380009DED021A20EE200ADDED010A00EE810A11
:103390008DED000AF2EE040AE06820EE200ABCEE91
:1033A000C00A80ED000ADFE760000800130000108B
:1033B00070B504460D4D207A002810D00C492278B3
:1033C000481D01F06BFF032803D0A169032008709A
:1033D00070BD21462846BDE87040FEF717BB214668
:1033E0002846BDE87040FEF711BB0000140008102D
:1033F00014000807017A002904D002780821024845
:10340000FFF762BC70470000870008007FB50546E3
:10341000EC68374E2A7869463046FEF739FA287A42
:103420003449D0B36A6800208A421BD12168090E52
:103430008DF802102168090C8DF803102188090A03
:103440008DF8041021788DF805108DF806008DF8A0
:1034500007008DF8080027482A780221801CFFF712
:1034600033FC14E02168090E8DF809102168090C5D
:103470008DF80A102188090A8DF80B1021788DF833
:103480000C108DF80D008DF80E008DF80F002A78C5
:103490006946304600F094FA7FBDFFE768688842CD
:1034A00012D19DF8050020609DF8041040EA01202B
:1034B00020609DF8031040EA014020609DF8021052
:1034C00040EA01602060E7E79DF80C0020609DF86D
:1034D0000B1040EA012020609DF80A1040EA0140EC
:1034E00020609DF8091040EA01602060D4E70000E8
:1034F000390008108500080030B585B0044604A9DD
:1035000022781948FEF7C4F9184D9DF81020694635
:103510002846FEF7BDF9207A70B1E06890ED000A08
:10352000B8EE400A8DED010A9DF810206946284644
:1035300000F046FA05B030BD9DED000ADDED030A4E
:103540009DED021A20EE200ADDED010A00EE810A4F
:103550008DED000AF2EE040AE06820EE200ABCEECF
:10356000C00A80ED000ADFE76000080012000010CA
:1035700030B587B00446207A002820D02178114841
:10358000FFF748FBC5B2217801A8FDF723FAE068F0
:1035900000780290217801A8FDF74CFA294601A88D
:1035A000FDF718FA029820F0FF000290E1680298F7
:1035B000097808430290294601A8FDF73BFA07B0B5
:1035C00030BD00006000080030B597B00446207A96
:1035D000002830D0227801A91848FEF759F922783E
:1035E00016A91748FEF754F9144D2278AD1D13A9FA
:1035F0002846FEF74DF916988DF84E0080308DF86C
:103600004F00E06801A90078C0EBC000084450F802
:10361000011F14918188ADF8541080798DF85600FF
:10362000227813A9284600F0CBF905482278042116
:10363000801EFFF749FB17B030BD00003A000810AC
:103640008900080008B50091694600F0B9F908BD85
:10365000F8B51F46154606461446009103E000984B
:10366000640840000090E007F9D019463046FFF7A3
:10367000D1FA0099A843084300903A46694630467B
:1036800000F09EF9F8BD00002DE9F041DFF8BC80A4
:10369000064601EB410158F8260088B01D464068F7
:1036A0001746406800EB81044FF0FF312068DDF7DA
:1036B000BBFC58F82600102241680B68A18801EB7A
:1036C000810102EB81015958E1B18DF80060416838
:1036D0000B68A18801EB810153F8211001910121B0
:1036E0008DF80810A11D059100210695CDE9037103
:1036F00040680168A08800EB800002EB8000095858
:1037000068468847287807281AD058F82600406865
:103710000168A08800EB8002082000EB82000B58B3
:103720003868834201D9052009E00C2303EB8202AB
:103730008958814201D2062001E0A060042028704F
:103740002068DDF7A7FC08B0BDE8F08134730120E4
:10375000F0B506461248002250F8210011460469CF
:10376000238930CC1F4602EB530035F810C034F8E3
:103770003CC01FFA8CFCB44501D9034601E00DD2D0
:103780000246A3EB020000EBD07001F1010102EB55
:103790006000C9B280B21029E7D93846F0BD0000F8
:1037A000347301202DE9F0471E494FF6FF7633466A
:1037B00051F820000069D0E900270589002009E0C0
:1037C00052F830101FFA81FC9C4501D28BB204469E
:1037D000401C80B2A842F3D33C800120B2461DE0D9
:1037E0000021564607EB400812E038F802CC52F8A8
:1037F000313032F83CC099469BB21FFA8CFC6345CD
:1038000004D9B34202D21FFA89F60C46491C89B288
:10381000A942EAD327F81040401C80B2A842DFD367
:10382000BDE8F0873473012010B50C4680B2FFF775
:103830008FFF094980B251F8241009690A89824230
:1038400001D1002010BD4A68096832F81000042236
:1038500002EBC000085810BD3473012010B51C469F
:10386000084B53F82000006909C833F811100423ED
:1038700003EBC10141581046DCF756FF02202070CF
:1038800010BD00003473012038B5044615230B4ADF
:10389000002102200094FDF74BFD0323084A01217B
:1038A00002200094FDF744FD054A04233C32102118
:1038B00002200094FDF73CFD38BD0000E43D030804
:1038C000883F030838B5044675230E4A00210820B6
:1038D0000094FDF72DFD05230B4A012108200094DB
:1038E000FDF726FD2B23094A102108200094FDF73F
:1038F0001FFD054A59236432112108200094FDF769
:1039000017FD38BD44F80208680103089404030851
:1039100038B504461C231A4A002108200094FDF7FC
:1039200007FD0423174A012108200094FDF700FD3C
:10393000144A1D235032102108200094FDF7F8FC92
:103940000F4A1E23F03A112108200094FDF7F0FCE5
:103950000D484470012C02D0022C05D008E00BA1C8
:10396000801CDCF7E1FE03E00EA1801CDCF7DCFE2E
:103970002246BDE838400449104800F021B8000054
:10398000EC2103081C240308BE080120363034371C
:1039900020526563656976657220312044656275E1
:1039A00067000000363034372052656365697665FC
:1039B0007220322044656275670000001200081012
:1039C000F8B50E46274D144603218DF8001055F822
:1039D0002410C0F307420978914201D00D20F8BDB0
:1039E000010E05D0012915D0102925D00B20F8BDD6
:1039F00080B22146FEF7A0FE55F8241080B2496837
:103A00000989814223D0C1B26B4632462046FFF776
:103A10003BFE24E080B22146FDF756FD55F8241008
:103A200080B289680989814211D0C1B26B463246A1
:103A30002046FDF743FE12E080B22146FEF746F82D
:103A400055F8241080B2C9680989814201D10A2041
:103A5000F8BDC1B26B4632462046FEF743FD9DF8E5
:103A60000000F8BD347301202DE9F04706462948CF
:103A70008946294D4178089C98469246002739B1DD
:103A80004770002045F82070401CC0B22028F9D3B0
:103A9000202C02D30220BDE8F08755F8240020B185
:103AA0000078B0420CD00520F5E708210120E0F7AE
:103AB0008BFB45F8240058B3067055F82400476086
:103AC000B9F1000F01D00320E5E755F82400406864
:103AD00008B10820DFE70C210120E0F775FB55F85D
:103AE00024104860A0B1C0F800A055F8241040464A
:103AF0004968A1F808800C21E0F766FB55F824100E
:103B00004968486020B1204600F09CF80020C2E7D8
:103B10000720C0E7E705012000790120F0B589B052
:103B200024216846DCF72FFF4FF4806000240C4E00
:103B30000C4D0127059056F8240048B1406838B173
:103B4000287828B92F706A4600210748DDF7BEFFA4
:103B5000641CE4B2202CEED309B00020F0BD0000BC
:103B600000790120E7050120293D020808B5002160
:103B700000900123024A0846FFF776FF08BD0000C7
:103B8000903C030838B5044623202178FFF742F81B
:103B900080B14FF48055227829460B20FFF743F877
:103BA00030B1227829460B20FEF7B6FD002038BD43
:103BB000012038BD227869460D20FDF769FE9DF889
:103BC0000010FF290AD0064800F092F8012803D01F
:103BD000022801D0002038BD012038BD002038BDAA
:103BE00002000800F0B5864615480022042550F86A
:103BF0002100114646683389D6E900749C4602EBE1
:103C0000530000EB400605EB8606A65B06EB860636
:103C100037F82660B6B2764501D9034601E00DD2E9
:103C20000246A3EB020000EBD07001F1010102EBB0
:103C30006000C9B280B21029E3D96046F0BD00002F
:103C4000007901202DE9F05F27494FF6FF7B5A46A6
:103C500051F8200040680789D0E9006081460020C3
:103C60000AE000EB800156F821108BB2934201D29A
:103C70008AB28046401C80B2B842F2D3A9F80480D0
:103C80001A48DDF7F5F90124C9F8000028E004EB33
:103C9000440A0020DC4609EB8A0514E035F8083CAC
:103CA00000EB800103EB830356F8211036F8233034
:103CB0008AB29BB29A4204D9624502D21FFA81FCB1
:103CC0008046401C80B2B842E8D3A5F8048007487B
:103CD000DDF7CEF949F82A000020641CA871A4B2CF
:103CE000BC42D4D3BDE8F09F0079012024F602083D
:103CF00070B50C4680B2FFF775FF0A49C0B200EB01
:103D0000400051F824104968496801EB80044FF0E5
:103D1000FF312068DDF788F9A5792068DDF7BAF969
:103D2000284670BD007901201CB50026384C54F897
:103D30002600002866D04068002863D01420DDF7F4
:103D400065F854F8260000274068D0E900B852E032
:103D50000220DDF75BF807EB470A08EB8A05A88825
:103D600000EB80000BEB8004216989B38DF80060C3
:103D70005BF820000190216968468847814658F821
:103D80002A004FF0FF31DDF74FF9A87901280AD05A
:103D900002281ED0B9F1010F27D10120A871DDF74B
:103DA00071F8A86021E0B9F1010F02D00020A871DC
:103DB0001BE0DDF767F8A968401AE188884214D350
:103DC0000220A871D4E902103246FEF77DFF0CE014
:103DD0000FE0207948B9B9F1000F06D10020A87191
:103DE000D4E902103246FEF797FC58F82A00DDF7B6
:103DF00051F97F1CBFB2064850F826004068008980
:103E0000B842A5D8761CF6B2202E8FD38DE70000DD
:103E10000079012038B5027869462248FDF738FD5F
:103E2000204D204C9DF800101B354334032902D04F
:103E300004291BD034E02320FEF7ECFE80B30122DE
:103E400008212846FEF7EFFE20B10122602120461E
:103E5000FEF73AFF012204212846FEF7E4FEF8B1FE
:103E6000012280212046FEF72FFF19E02320FEF7D4
:103E7000D1FEA8B1022208212846FEF7D4FE20B1C7
:103E8000022260212046FEF71FFF0222042128465D
:103E9000FEF7C9FE20B1022280212046FEF714FF62
:103EA000002038BD4400080008B505230090034AEF
:103EB00000210820FFF7D8FD08BD000004200308FA
:103EC00070B504460F482178FEF7A4FEFF2806D0FF
:103ED0000C48227818212C38FEF7A5FE08B10020E6
:103EE00070BD084D217853352846FEF793FE30B15A
:103EF000227800212846FFF7A5FB002070BD012095
:103F000070BD000044000800F8B5054600240121FA
:103F10000B48FEF77FFE0090094E2978761C30464C
:103F2000FEF778FE0099884205D001242A78694678
:103F30003046FFF745FD0CB10020F8BD0120F8BD6B
:103F400090000800F8B50546002402210B48FEF752
:103F500061FE0090094E2978B61C3046FEF75AFEE5
:103F60000099884205D001242A7869463046FFF737
:103F700027FD0CB10020F8BD0120F8BD900008001D
:103F800010B504460F482178FEF744FEC0B205285C
:103F900003D006280AD0012010BD0A4821786238D3
:103FA000FFF7A6FE022808D1012010BD05482178A0
:103FB0006138FFF79DFE022801D0002010BD0120CE
:103FC00010BD00006700080008B501230090034AF7
:103FD00000210820FFF748FD08BD0000DC2F030882
:103FE00070B50446074D227820212846FEF71BFEB7
:103FF00030B1227820212846FEF78EFB002070BDCC
:10400000012070BD5F0008002DE9F04105460E4615
:104010001746002409E004EB440006EBC000182218
:104020003946DCF754FC641CE4B2AC42F3D3BDE87F
:10403000F0810000F8B50746254E3A46102130467B
:10404000FEF742FE4FF4A0612248DCF79CFC4FF4DF
:1040500090712148DCF797FC1D483A466946533079
:10406000FDF716FC00249DF8002001212046DFF713
:10407000F5FF3F2200212046DFF7F0FF0522022155
:104080002046DFF7EBFF641CE4B2072CEBD90025D8
:1040900000243F2229462046E0F762F80022294604
:1040A0002046E0F73DF8641CE4B2072CF1D96D1C02
:1040B000EDB22F2DECD9DFF7CFFEDFF7CDFEDFF726
:1040C00049FF3A4610213046FEF726FBF8BD0000B6
:1040D00018000800247A0120247F01202DE9F047F0
:1040E00026494FF6FF7A524651F820008168406910
:1040F0000F89D0E90050814600200AE000EB400122
:1041000055F831108BB2934201D28AB20646401C58
:1041100080B2B842F2D3A9F804601948DCF7A8FFCE
:104120000124C9F8000025E00020534609EBC40C27
:1041300015E03CF8042C00EB400102EB420255F87C
:10414000318035F832201FFA88F192B2914204D9B9
:10415000994202D21FFA88F30646401C80B2B84248
:10416000E7D3ACF804600648DCF782FF49F8340076
:10417000641CA4B2BC42D7D3BDE8F087007801200C
:1041800014F602082DE9F04726494FF6FF7A524609
:1041900051F8200080690789D0E90050814600204D
:1041A0000AE000EB400155F831108BB2934201D286
:1041B0008AB20646401C80B2B842F2D3A9F8046025
:1041C0001948DCF755FF0124C9F8000025E000205C
:1041D000534609EBC40C15E03CF8042C00EB4001FD
:1041E00002EB420255F8318035F832201FFA88F18F
:1041F00092B2914204D9994202D21FFA88F306463C
:10420000401C80B2B842E7D3ACF804600648DCF743
:104210002FFF49F83400641CA4B2BC42D7D3BDE8D8
:10422000F08700000078012014F602082DE9F05F05
:104230001E46154689468046FE48FF4F0A9C017877
:104240004FF0000A59B180F800A0002051460A2220
:1042500047F82010401C80B28A702028F8D3202C08
:1042600002D30520BDE8F09F57F8240020B1417823
:10427000414551D00A20F5E7DC210120DFF7A4FFFA
:1042800047F82400002875D0047057F8241081F8EE
:10429000018057F824005146C0F814A057F82400B4
:1042A000C0F818A057F82400C0F808A057F8240058
:1042B000C0F80CA057F82400C0F810A057F824004C
:1042C00080F803A000201C2202EB800C57F8243059
:1042D000401C80B243F80C102028F5D357F8240076
:1042E000017100209C2202EB800C57F82430401C06
:1042F00080B243F80C100828F5D357F82400417118
:104300000020BC2202EB800C57F82430401C80B205
:1043100043F80C100828F5D3484606F0FF094FF083
:10432000040B082868D2DFE800F00426466888AA53
:10433000FEFD57F82400806800285CD10C21012084
:10434000DFF742FF57F82410002888609BD00560F3
:1043500057F824000821806806813046DFF734FFD3
:1043600057F824100028896848608CD0204600F057
:10437000E5F9ABE166E157F82400C068D8BB0C2131
:104380000120DFF721FF57F824100028C860DDD096
:10439000056057F824000821C06806813046DFF721
:1043A00013FF57F824100028C9684860CED0204673
:1043B00000F0AEFA8AE157F824000069D8B90C2160
:1043C0000120DFF701FF57F8241000280861BDD055
:1043D000056057F824000821006906813046DFF7A0
:1043E000F3FE57F82410002809694860AED0204633
:1043F00000F06EFC6AE124E06EE157F824004069A9
:10440000F8B90C210120DFF7DFFE57F8241000284F
:1044100048619BD0056057F8240008214069068157
:104420003046DFF7D1FE57F824100028496948606C
:104430008CD02046FFF752FE48E157F824008069EF
:1044400008B10E200EE70C210120DFF7BDFE57F862
:1044500024100028886188D0056057F824000821BE
:10446000806906813046DFF7AFFE57F82410002838
:10447000896948608BD02046FFF784FE26E157F813
:10448000240090F80380B8F1200F7DD208F10101DB
:10449000C170694F1C210120DFF796FE57F82420D8
:1044A0001C2101EB88070028D05190D0DFF88881CB
:1044B0004560624858F82410C95981F80090DCF72B
:1044C000D7FD58F824104FF0010CC959886158F8ED
:1044D00024100220C959487258F8241000200825D9
:1044E000C95981F808C058F82410C95981F80AA0A0
:1044F0001CE058F824200BEB0013D1594968CB5C21
:104500007BB905EB0013C95864290AD20A23B1FB11
:10451000F3F111F0FF01917058F8242001D182F8D5
:1045200002C001E068E004E0401C80B2B042E0D389
:10453000CCE057F8240090F80480B8F1080F23D29B
:1045400008F101010171BA461C210120DFF73CFE90
:104550005AF824209C2101EB88070028D05171D003
:10456000E96841605AF82400D046C05980F80090AC
:104570005AF82400C05904725AF82400A968C05996
:10458000C1602879012100E0A4E0DFF71DFE58F8A2
:1045900024100028C959486154D02979DCF7D1F991
:1045A000286820B158F82410C959086104E058F867
:1045B00024002349C059016101213046DFF704FE80
:1045C00058F82420D2599061E0B3002511E058F842
:1045D000240005EB8502C05941680BEBC20008447A
:1045E000DCF7C6F858F82410C959896948556D1C7C
:1045F000ADB2B542EBD369E057F824004679082EF6
:1046000068D2711C4171AC210120DFF7DDFD57F844
:104610002420BC2101EB8606905198B1E9684160E5
:1046200057F82410895981F8009057F824008059D0
:10463000047208E0E40501200078012014F6020865
:10464000919A020844E057F82410A8688959C86074
:1046500057F8241028688959086157F82410895997
:1046600081F814A057F82400802180591830DCF715
:104670008AF957F8241000222020895981F899A03E
:1046800057F82410895981F898A01146DDF7AEF942
:1046900057F8241000228959C1F8A40020210846A7
:1046A000DDF7A4F957F824108959C1F8A80057F884
:1046B0002400A9888059A0F8A0100120DFF784FD0C
:1046C00057F824108959C1F89C0008B10020C9E5A9
:1046D0000D20C7E50C20C5E50620C3E5F0B58446EE
:1046E00015480022042550F82100114686683389B8
:1046F000746836681F4602EB530005EBC00E34F8B1
:104700000EE006EB0E1EBEF800E01FFA8EFEE64538
:1047100001D9034601E00DD20246A3EB020000EBF3
:10472000D07001F1010102EB6000C9B280B2102922
:10473000E3D93846F0BD0000007801202DE9F047AC
:1047400025494FF6FF7A524651F8200080680789C4
:10475000D0E900508146002009E005EB001109680E
:104760008BB2934201D28AB20646401C80B2B84254
:10477000F3D3A9F804601948DCF77AFC0124C9F8DE
:10478000000025E00020524609EBC40316E033F890
:1047900004CC05EB001105EB0C1CD1F80080BCF833
:1047A00000C01FFA88F11FFA8CFC614504D99142C0
:1047B00002D21FFA88F20646401C80B2B842E6D305
:1047C0009E800648DCF754FC49F83400641CA4B20F
:1047D000BC42D7D3BDE8F0870078012014F6020868
:1047E00008B50A46694600F005FD9DF8000008BDC1
:1047F000F0B52E4F054687B057F82500164680685D
:10480000406800EBC1044FF0FF312068DCF70CFC7E
:1048100057F82500A28880680168082000EB021084
:10482000095819B1E8B288478DF8140057F82500E7
:10483000A1880422806802EB01110068405C002816
:104840009DF8140001D070BB01E060B300208DF82A
:1048500014000120307057F82500A38881680A6889
:104860000C2101EB0313D258B2B18DF800508268CD
:10487000A388126802EB03121268019200228DF8DD
:10488000082005AACDE903268068A288006801EB0C
:1048900002114158684688472068DCF7FBFB9DF809
:1048A000140007B0F0BDFFE70120D0E70078012039
:1048B000F0B5844615480022042550F82100114621
:1048C000C6683389746836681F4602EB530005EBEF
:1048D000C00E34F80EE006EB0E1EBEF800E01FFA24
:1048E0008EFEE64501D9034601E00DD20246A3EB58
:1048F000020000EBD07001F1010102EB6000C9B2CF
:1049000080B21029E3D93846F0BD000000780120BC
:104910002DE9F04725494FF6FF7A524651F820001D
:10492000C0680789D0E900508146002009E005EB06
:10493000001109688BB2934201D28AB20646401C2C
:1049400080B2B842F3D3A9F804601948DCF790FBB1
:104950000124C9F8000025E00020524609EBC403F9
:1049600016E033F804CC05EB001105EB0C1CD1F874
:104970000080BCF800C01FFA88F11FFA8CFC61456A
:1049800004D9914202D21FFA88F20646401C80B236
:10499000B842E6D39E800648DCF76AFB49F834004B
:1049A000641CA4B2BC42D7D3BDE8F08700780120D4
:1049B00014F60208F0B52F4F054687B057F82500CA
:1049C0001646C068406800EBC1044FF0FF31206814
:1049D000DCF72AFB57F82500A288C0680168082088
:1049E00000EB02100B582BB10021EAB208469847A1
:1049F0008DF8140057F82500A1880522C06802EB45
:104A000001110068405C00289DF8140001D070BBC3
:104A100001E060B300208DF814000120307057F8D9
:104A20002500A388C1680A680C2101EB0313D25842
:104A3000B2B18DF80050C268A388126802EB03126D
:104A40001268019200228DF8082005AACDE90326FC
:104A5000C068A288006801EB021141586846884787
:104A60002068DCF717FB9DF8140007B0F0BDFFE7E6
:104A70000120D0E7007801202DE9F041DFF8A8807F
:104A8000054686B058F825001E461746C06840689F
:104A900000EBC1044FF0FF312068DCF7C5FA58F88D
:104AA0002500A388C1680A680C2101EB0313D258C2
:104AB000AAB18DF80050C268A388126802EB0312F5
:104AC0001268019201228DF80820CDE90376C068B2
:104AD000A288006801EB0211415868468847307887
:104AE000022819D058F82500A2880521C06801EBDA
:104AF00002110068415C0029397801D091B901E0C8
:104B000081B10021082303EB0212835813B1EAB2EA
:104B100001209847032030702068DCF7BBFA06B00C
:104B2000BDE8F0810121EDE70078012010B50346D2
:104B3000002006E003EB00142468944203D0401CDC
:104B4000C0B28842F6D310BD2DE9F04393B0DEF732
:104B5000CDFD242109A8DBF716FF20204401CDE973
:104B60000E4024216846DBF70EFF05941D4E0024FD
:104B70004FF09C084FF0BC0956F8241049B3C87890
:104B800018B109AA1848DCF7A1FF0025474609E03B
:104B900007EB8501415819B16A461448DCF796FFC6
:104BA0006D1CEDB256F824000179A942F0D8002519
:104BB0004F4609E007EB8501415819B16A460C4898
:104BC000DCF784FF6D1CEDB256F824004179A94250
:104BD000F0D8641CE4B2202CCED313B00020BDE882
:104BE000F083000000780120A1980208999A020839
:104BF000CD55020838B504460623134A0721002084
:104C00000094FFF713FB0123104A022100200094B7
:104C1000FFF70CFB0D4A05231832194600200094BB
:104C2000FFF704FB094A0523683219460020009467
:104C3000FFF7FCFA054A0423B8320521002000944E
:104C4000FFF7F4FA38BD0000680901205438030862
:104C5000F8B50C4615460646114600F05DF9A0432E
:104C600000902A466946304605F070F9F8BD00000C
:104C7000F0B5844615480022042550F8210011465D
:104C800006693389746836681F4602EB530005EBEA
:104C9000C00E34F80EE00EEB4E0E36F83EE01FFA72
:104CA0008EFEE64501D9034601E00DD20246A3EB94
:104CB000020000EBD07001F1010102EB6000C9B20B
:104CC00080B21029E3D93846F0BD000000780120F9
:104CD0002DE9F04726494FF6FF7A524651F8200059
:104CE00000690789D0E90050814600200AE000EB06
:104CF000400155F831108BB2934201D28AB2064678
:104D0000401C80B2B842F2D3A9F804601948DCF71D
:104D1000AFF90124C9F8000025E00020534609EB53
:104D2000C40C15E03CF8042C00EB400102EB4202FD
:104D300055F8318035F832201FFA88F192B291424D
:104D400004D9994202D21FFA88F30646401C80B269
:104D5000B842E7D3ACF804600648DCF789F949F8B3
:104D60003400641CA4B2BC42D7D3BDE8F087000075
:104D70000078012014F602082DE9F04788B00346B8
:104D80000D46914600240020069005904FF0010842
:104D9000CDF81080CDF80C8002905C48006801903E
:104DA000012B06D049460020FDF734FF08B0BDE8CE
:104DB000F0874A4629460020FEF744FC042801D02B
:104DC0000020F3E7002D64D0E8074FF4806A4FF02D
:104DD000100606D0544649461920FDF71BFF0690E1
:104DE0000496A8074FF0040707D544F40064494629
:104DF0001920FDF70FFF06900497680707D544F4C4
:104E0000005449461A20FDF705FF0590039728072F
:104E100007D544F4805449461A20FDF7FBFE05905F
:104E20000396E80603D544F4804440200290A80687
:104E300002D544F400440296680604D544F4007494
:104E40004FF480000290280604D544F480744FF497
:104E500080700290680500D50297E80501D5CDF86D
:104E60000880E80402D54FF480400290A80402D5DF
:104E70004FF480500290A80501D5CDF808A0280570
:104E800001D544F080044A4600210E20FEF7DAFBEB
:104E900006E0DBF7F7FF01464A460E20FEF7D2FB9D
:104EA0004A4607A90D20FCF7F3FC9DF81C2002A937
:104EB0001748FEF785FD16489DF81C2006A9401CE2
:104EC000FEF77EFD12489DF81C2005A9801CFEF708
:104ED00077FD0F489DF81C2004A9C01CFEF770FD4B
:104EE0000B489DF81C2003A9001DFEF769FD200A50
:104EF0008DF8060044F00C008DF807009DF81C208A
:104F000001A90448FEF75CFD28464FE75038030826
:104F1000610008000700081008B50A46694600F05D
:104F200069F9009808BD00002DE9F041474F05469A
:104F300086B057F8250016460069406800EBC104AA
:104F40004FF0FF312068DCF76FF857F82500006953
:104F50000168A08800EB4002102000EBC2000B5853
:104F6000002B70D00021EAB208469847059057F808
:104F700025004FF008080C2300690168A08800EBA9
:104F8000400008EBC0028A5C022A10D0032A0ED02F
:104F900003EBC000085857F8251009690A68A18872
:104FA00001EB410308EBC301515CB9B118E003EB1D
:104FB000C0000858E9B2FDF72DFE57F82510096921
:104FC0000A68A18801EB410308EBC301515C022987
:104FD00004D0E0E70599400849080591C107F9D0D8
:104FE0000599014001200591307057F825001422E1
:104FF00001690B68A18801EB410102EBC10159581D
:10500000C9B18DF8005001690B68A18801EB41011D
:1050100053F83110019100218DF8081005A9CDE950
:10502000031600690168A08800EB400002EBC00095
:105030000958684688472068DCF72CF8059806B0C0
:10504000BDE8F081FFE70720CEE7000000780120EF
:10505000F8B50C46154606461146FFF75DFF20439E
:1050600000902A466946304604F070FFF8BD10B53E
:1050700012210020DEF7E0FA0106090C41EA1020B7
:10508000C04310BD10B512210020DEF7BBFA0106A7
:10509000090C41EA1020C04310BD08B500916946D3
:1050A00004F054FF08BD00002DE9F04FDFF8408107
:1050B000044685B058F824001F461646006940682B
:1050C00000EBC1054FF0FF312868DBF7ADFF58F862
:1050D0002400142201690B68A98801EB410102EB4D
:1050E000C1015958C1B18DF8004001690B68A98808
:1050F00001EB410153F83110019101218DF80810A5
:10510000CDE9036700690168A88800EB400002EB65
:10511000C0000958684688473878022861D058F896
:1051200024004FF0080900690268A88800EB4003DA
:10513000102000EBC303D358CBB383460021E2B267
:1051400008469847824658F8240036680C230069C0
:105150000168A88800EB400009EBC0028A5C022AC3
:1051600011D0032A0FD003EBC0000858024658F8AC
:10517000241009690B68A98801EB410C09EBCC01EB
:10518000595CB9B118E003EBC0000858E1B2FDF773
:1051900041FD58F82410024609690B68A98801EB03
:1051A000410C09EBCC01595C022903D0DFE716E082
:1051B00040087600C107FBD058F824002AEA020113
:1051C000314300690268A88800EB40030BEBC30081
:1051D0001358E2B2012098470320387001E087F8A5
:1051E00000902868DBF756FF05B0BDE8F08F00009F
:1051F00000780120F8B50D46274E144607218DF89A
:10520000001056F82410C0F307424978914201D0AB
:105210000A20F8BD010E05D0012914D0022924D09E
:105220000620F8BD80B22146FFF758FA56F8241040
:1052300080B289680989814222D0C1B26A4620467B
:10524000FFF7D6FA0FE080B22146FFF731FB56F8A0
:10525000241080B2C9680989814211D0C1B26A465E
:105260002046FFF7A7FB287012E080B22146FFF727
:10527000FFFC56F8241080B209690989814201D1E6
:105280000B20F8BDC1B26A462046FFF74DFE2860EC
:105290009DF80000F8BD0000007801202DE9F041E4
:1052A0002F4E1446C0F3074356F824C09CF8012043
:1052B0009A4202D00A20BDE8F0810022BC2505EB0D
:1052C00082035CF8033013B1DB688B4203D0521CBD
:1052D000D2B2082AF3D3082A09D005EB82055CF87C
:1052E0000520117D012904D00021137811E0092047
:1052F000E1E70F20DFE701EB410ED2F804C00EEB2F
:10530000C10E5CF83EC0844501D10F4603E0491C44
:1053100089B28B42EFD88B4201D10B20CBE74FF003
:10532000FF31D2F8A800DCF71FFB56F82400182242
:10533000405990F8981002EB8101475056F824002C
:10534000405910F8981F491C01F01F01017056F8D0
:1053500024004059D0F8A400DCF75AFB0320AAE748
:10536000007801202DE9F04107460E46134C3146E6
:10537000204607F0E3FB254603E03146012007F015
:10538000DDFA3146284607F0A5FC0428F5D132465F
:105390004FF0E1613846FFF781FF3146084807F0DA
:1053A000C3F9032807D000243146284607F0F8FB4C
:1053B0002046BDE8F0810124F6E700000100080066
:1053C0000100080130B500220321D0E9023404E0D5
:1053D0005D5C2A44D2B2491CC9B28C42F8D8C2F1F1
:1053E000FF011955C168491CC1608268091F91708D
:1053F00081898068091F090A417030BDF8B50446EB
:1054000009202178FDF706FC0546E0682A0E411CBC
:10541000E160A1680A54E0682A0C411CE160A168BF
:105420000A54E0682A0A411CE160A1680A54E06855
:10543000411CE160A1680D54280E07D0012805D059
:105440000026102823D0112848D132E0227869465E
:105450002846FCF71DFA0098020EE068411CE16046
:10546000A1680A540098020CE068411CE160A16840
:105470000A540098020AE068411CE160A1680A54DD
:10548000E0680099421CE260A268115426E0D4E969
:105490000201014422782846FCF7FAF921782846CF
:1054A000FCF77CF9E1680844411CE160A1680E54F6
:1054B00014E021782846FEF7B7F9054675B1D4E91E
:1054C000020108442946DBF72FF92846DBF750F99B
:1054D000E1680844411CE160A1680E542046FFF7D2
:1054E00071FFF8BD70B50446094DD4E902010144CD
:1054F00022782846FCF7CCF921782846FCF74EF9AB
:10550000E1680844E0602046BDE87040FFF75ABFFC
:105510000A00001010B50446D4E902010844401CFA
:1055200005F07AFFD4E902128854E1680844401C6F
:10553000E0602046BDE81040FFF744BF10B50446C8
:10554000D4E902010844217805F0EEFFC0B2E16819
:105550000844E0602046BDE81040FFF733BF10B5B7
:10556000044608202178FDF755FBD4E902121144C6
:10557000227806F077F8C0B2E1680844E06020467F
:10558000BDE81040FFF71EBFF0B5DFF83CC00024B7
:10559000BC275CF8236007EB8405755915B1ED68ED
:1055A000854203D0641CE4B2082CF4D3082C09D043
:1055B00007EB8400345861605CF8231008580270CF
:1055C0000320F0BD0920F0BD0078012090B0044612
:1055D000C0680E90207A0790D4F89CB00120DBF7C9
:1055E00015FC4FF0FF31D4F8A400DCF7BDF994F8B6
:1055F000990004EB8001401C098B00F01F0084F827
:1056000099008EB2D4F8A800DCF702FAB4F8A01022
:105610005846DBF796F9002506EB4600A94600EB55
:10562000C6060B957BE03C2804D109F10603D35C48
:105630003E2B04D00BF805006D1CADB26BE009F1F8
:10564000050012F800800B98401C80B20B900128D6
:105650001ED002281ED04FF0FF308246B8F14D0F09
:105660001DD0B8F14C0F1AD0FF200C90D0B10128FA
:105670002ED010282CD0B8F1310F2FD0B8F1320F26
:105680002ED0B8F1330F2DD0B8F1340F2CD02CE040
:10569000442000E0482000EBC6000858DDE74FEA50
:1056A0001A60E2E70DA95046079AFCF75BF90D98DE
:1056B000FF2801D801271BE0B0F5803F01D2022767
:1056C00016E0B0F1807F01D2032711E004270FE03C
:1056D00050460799FCF762F8074606E0012704E008
:1056E000022702E0032700E004270C98FF2829D0B6
:1056F0000BEB05015046079AFCF7CAF80BEB0502C5
:105700003B4641460C98DEF7E1FAE81985B209F10B
:1057100002001FFA80F909F101001FFA80F961689F
:1057200009F1040001EBC602105C10B1402DFFF43A
:105730007AAFCDE902B54C21606801EBC601425851
:1057400062B906E04BF805A000204FF04C080C9021
:10575000D4E7542202EBC6028058E8B107988DF8CE
:1057600000000422606802EBC6021044049044204A
:10577000626800EBC600105805904820626800EB94
:10578000C60010580690606850F8360001906068B6
:10579000415809B1684688470E98089002980990C8
:1057A00003980A90216908A888476168502000EB97
:1057B000C600085A08B1DBF729FB5420616800EBEA
:1057C000C600095800293FF409AF6846884705E735
:1057D0002DE9F047814688460024174D4FF0E166D9
:1057E0004FF08477424631464846FFF757FD414621
:1057F000384606F099FF03280CD041462846FDF7AD
:1058000009FA411C42462846FDF71CFF641CE4B21D
:105810000A2CE7D30A2C02D00120BDE8F087064C01
:105820004146641C2046FDF7F5F9411C42462046DE
:10583000FDF708FF0020F0E70A00080030B500225D
:105840000321D0E9023404E05D5C2A44D2B2491C51
:1058500089B28C42F8D8C2F1FF011955C168491CC0
:10586000C1608268091F917081898068091F090AD7
:10587000417030BD38B500246846DDF715FD0028BD
:1058800003D0641CE4B2FF2CF6D338BD10B5044637
:1058900040F24C40217807F051F82046BDE8104016
:1058A000FFF7E8BF2DE9F84307460025E846002446
:1058B00008EB05063046DDF7F7FC38B939780120EA
:1058C00007F03CF8641CE4B2642CF3D3642C10D0D1
:1058D0006D1CEDB2032DEAD300208DF8030069465C
:1058E00005A0DBF777F8002803D13978034806F0E4
:1058F000F1FEBDE8F88300004F4B0D0001000801E8
:10590000F8B5044638482178FDF784F90546E06883
:105910002A0E411CE160A1680A54E0682A0C411C6F
:10592000E160A1680A54E0682A0A411CE160A168AC
:105930000A54E068411CE160A1680D54280E07D0AC
:10594000012805D00026102823D0112848D132E0A4
:10595000227869462846FBF79BFF0098020EE06814
:10596000411CE160A1680A540098020CE068411CE7
:10597000E160A1680A540098020AE068411CE160F5
:10598000A1680A54E0680099421CE260A2681154C0
:1059900026E0D4E90201014422782846FBF778FF8B
:1059A00021782846FBF7FAFEE1680844411CE160D3
:1059B000A1680E5414E021782846FDF735FF05460E
:1059C00075B1D4E9020108442946DAF7ADFE28464C
:1059D000DAF7CEFEE1680844411CE160A1680E548C
:1059E0002046FFF72BFFF8BD1700080070B50446EE
:1059F000094DD4E90201014422782846FBF748FF0B
:105A000021782846FBF7CAFEE1680844E06020469A
:105A1000BDE87040FFF712BF1200081010B5044631
:105A2000D4E902010844401C05F0F6FCD4E9021256
:105A30008854E1680844401CE0602046BDE81040FE
:105A4000FFF7FCBE10B50446D4E9020108442178F2
:105A500005F06AFDE1680844E0602046BDE81040BA
:105A6000FFF7ECBE10B5044608482178FDF7D2F8E0
:105A7000D4E902121144227805F0F4FDE1680844EB
:105A8000E0602046BDE81040FFF7D8BE15000800D2
:105A900070B5044600210320D4E9022304E0155C1C
:105AA0002944C9B2401CC0B28342F8D8C1F1FF00FA
:105AB000D054E068401CE060A168001F8870A08995
:105AC000A168001F000A4870054D21782846FDF79F
:105AD000A1F8411C22782846BDE87040FDF7B2BD10
:105AE00093000800F8B5044638482178FDF792F88D
:105AF0000546E0682A0E411CE160A1680A54E0688E
:105B00002A0C411CE160A1680A54E0682A0A411C81
:105B1000E160A1680A54E068411CE160A1680D548D
:105B2000280E07D0012805D00026102823D01128E0
:105B300048D132E0227869462846FBF7A9FE009852
:105B4000020EE068411CE160A1680A540098020C52
:105B5000E068411CE160A1680A540098020AE0680C
:105B6000411CE160A1680A54E0680099421CE260AF
:105B7000A268115426E0D4E90201014422782846A3
:105B8000FBF786FE21782846FBF708FEE16808440B
:105B9000411CE160A1680E5414E021782846FDF70D
:105BA00043FE054675B1D4E9020108442946DAF7F7
:105BB000BBFD2846DAF7DCFDE1680844411CE160E2
:105BC000A1680E542046FFF763FFF8BD17000800D8
:105BD00070B50446094DD4E90201014422782846F3
:105BE000FBF756FE21782846FBF7D8FDE16808440C
:105BF000E0602046BDE87040FFF74ABF1200081081
:105C000010B50446D4E902010844401C05F004FC28
:105C1000D4E902128854E1680844401CE060204640
:105C2000BDE81040FFF734BF10B50446D4E90201C7
:105C30000844217805F078FCC0B2E1680844E060CF
:105C40002046BDE81040FFF723BF000010B5044612
:105C500009482178FCF7DEFFD4E9021211442278CA
:105C600005F000FDC0B2E1680844E0602046BDE8F0
:105C70001040FFF70DBF000015000800F0B58BB015
:105C80000446DBF7FFF8064622780AA95548FBF7D9
:105C9000FFFDE368A268591C9D18481C8F18330E3D
:105CA000411CE1601354E068320C411CE160A168C2
:105CB0000A54E068320A411CE160A1680A54E068B5
:105CC000411CE160A1680E540520287000263E703A
:105CD00050E09DF8282006A94348FBF7D9FD02288B
:105CE0004AD13878401C3870E0689DF81B20411C70
:105CF000E160A1680A54E0689DF81A20411CE16047
:105D0000A1680A54E0689DF81920411CE160A1686F
:105D10000A54E0689DF81820411CE160A1680A540B
:105D20009DF81C00C0F38301800941EAC012E068BD
:105D3000411CE160A1680A54002006AA0AE011187B
:105D400091F808C0E1684B1CE360A36803F801C048
:105D5000401CC0B29DF81C10C1F383018142EED8F3
:105D60009DF81C002978C0F38300401D084428706A
:105D7000761CF6B2052EACD31B48227801A9401F31
:105D8000FBF786FDE0689DF80420411CE160A168F6
:105D90000A54E0689DF80520411CE160A1680A549E
:105DA0002878801C2870D4E9020108449DF8052059
:105DB0000DF10601DAF746FD9DF80510E06808448C
:105DC000E06028789DF8051008442870387820B1E4
:105DD0009DF82810054806F07DFC2046FFF758FE88
:105DE0000BB0F0BD5E00080027000810030008019A
:105DF0002DE9FF470446A568627803A92748FBF709
:105E000047FD039890B1C6B2C0F30727A5F1A16082
:105E1000DFF88C8032384FF002014FF001090CD0CE
:105E2000204A012821D0022835D104E01D48801CD9
:105E300004B0BDE8F08715462DE0207890B18DF8CC
:105E400008108DF80060627869464046FDF7B8FD9D
:105E50008DF808908DF80070627869464046FDF72D
:105E6000AFFD18E00F4D6D1C15E0207890B18DF856
:105E700008108DF80070627869464046FDF7A0FD75
:105E80008DF808908DF80060627869464046FDF70D
:105E900097FD00E015462846CAE7000054000800B8
:105EA00019000810320008052DE9F04F04462DEDC9
:105EB000048B89B04FF00008A768627801A9AD484B
:105EC000FBF7E6FCA7F1A160AB4DDFF8B0923438E8
:105ED0004FF0020A4FF0030B06D001283CD00228F5
:105EE00074D003281FD148E02078E8B162781021EF
:105EF0002846FCF798FE002815D021208DF81800C0
:105F00008DF811A0627804A94846FDF759FD8DF877
:105F100011B0627804A94846FDF752FD627810215D
:105F20002846FCF7F9FB17E19348627808A9C01CE2
:105F3000FBF7AEFC08981028F5D1914F0298019913
:105F4000C0B20290002060F31F210191627801A984
:105F50008848FDF735FDFFE02069FA28E3D961782C
:105F60002846FCF757FE0028DDD1854F7F1C62785C
:105F700010212846FCF7A8FEEEE020780028D2D1B8
:105F800000252E46627807A97E48FBF781FC9DED2F
:105F9000070A7D4910EE100ADFED7C8A9FED7C8AAE
:105FA000B3EE059A884201DA00220CE030EE680A6E
:105FB0008DED070AC0EE080A20EE890ABCEEC00A81
:105FC00010EE100AC2B20020724B0BE095E053F8BD
:105FD0002010002903DA21F000410E4300E00D43B8
:105FE000401CC0B29042F2D36648627807A9401CB8
:105FF000FBF74EFC9DED070A634910EE100A88423C
:1060000001DA00220CE030EE680A8DED070AC0EEDE
:10601000080A20EE890ABCEEC00A10EE100AC2B2CD
:1060200000205C4B54330AE053F82010002903DAB7
:1060300021F000410E4300E00D43401CC0B29042ED
:10604000F2D30198B6EB102F24D018208DF8180049
:106050008DF811A000208DF813000198000AB043BC
:106060000590627804A94846FDF7AAFC8DF811A0B6
:10607000019826EA1020059023208DF818006278F8
:1060800004A94846FDF79CFC019866F31F20019087
:106090004FF001080298B5EB102F24D018208DF88E
:1060A00018008DF811B000208DF813000298000A36
:1060B000A8430590627804A94846FDF781FC8DF855
:1060C00011B0029825EA1020059023208DF81800C1
:1060D000627804A94846FDF773FC029865F31F2017
:1060E00002904FF00108244862781021C01CFCF790
:1060F0009AFD88BB224F7F1E2EE08DF811A0272528
:106100008DF8185083268DF81360627804A94846EC
:10611000FDF756FC25208DF818006C278DF81370BC
:10612000627804A94846FDF74BFC8DF811B0242095
:106130008DF818008DF81370627804A94846FDF7B1
:106140003FFC8DF818508DF81360627804A948461A
:10615000FDF736FC0A4FBF1CB8F1000F04D062787F
:1061600001A90448FDF72CFC09B03846BDEC048BAE
:10617000BDE8F08F1A000810400008001900081050
:106180003500080503000801CDCC4C40CDCC4C4077
:10619000FCFF7F3FF40701202DE9F04F04462DED71
:1061A000028B89B00027A668627801A9A848FBF78E
:1061B0006FFBA6F1A160A74DDFF89C9234384FF039
:1061C00000080CD0DFF894A2012837D005F1060BA7
:1061D000B2EE048A022841D0032818D1B3E0207817
:1061E000B0B1627802212846FCF71DFD00280ED0D0
:1061F00021208DF814008DF80D80627803A948469F
:10620000FDF7DEFB627802212846FCF785FA12E1F1
:106210009048627808A9C01CFBF73AFB089802284E
:10622000F5D18E4E761E01988DF80A8068F31F20F6
:10623000019001208DF804000127FCE02069FA2874
:10624000E5D961782846FCF7E5FC0028DFD1564601
:10625000627802212846FCF737FDECE02078002820
:10626000D5D100257B4861780C30FCF7D3FC00EEDB
:10627000100AF8EE400A80EE880A02F0C9FA40B22D
:10628000774E04E036F810100D43401C40B2082849
:10629000F8DB704861780D30FCF7BCFC00EE100AAA
:1062A000F8EE400A80EE880A02F0B2FA41B200200D
:1062B00004E036F810201543401C40B209B1884272
:1062C000F7DB9DF80A00A84203D1019810F0FF0FF8
:1062D00032D0CDF81080FF208DF80F0018208DF8F7
:1062E00014008DF80D80627803A94846FDF768FB1D
:1062F00062780DF109015846FBF7CAFA9DF80900CA
:1063000004281CD025208DF81400E8438DF80F00D8
:10631000627803A94846FDF753FB8DF80F502420FF
:106320008DF81400627803A94846FDF749FB8DF803
:106330000A508DF804800127484E761C7BE0262009
:106340008DF81400E1E7207878BB61785846FCF7B7
:1063500061FC9DF80910DFF804B18842ABF1020B33
:1063600068D13C48627807A90B30FBF791FA3948AD
:10637000627806A90A30FBF78BFA00258DF80F80AA
:106380009DED070AF8EE400A80EE880A03F0B8F99E
:1063900001460698C822B0FBF2F20692881A40B273
:1063A00011444AB22E4B603B0EE040E0002801DA77
:1063B000002104E0172801DD172100E0014653F811
:1063C00021100D43401C40B29042EFDD0198B5EB27
:1063D000102F20D018208DF814008DF80D80019812
:1063E000000AA8430490627803A94846FDF7E8FA3A
:1063F0008DF80D80019825EA1020049023208DF857
:106400001400627803A94846FDF7DAFA019865F3AB
:106410001F20019001270F4862780221C01CFCF761
:1064200002FC28B1019810F0FF0F04D0564602E09C
:106430005E4600E05E4627B1627801A90448FDF798
:10644000BFFA09B03046BDEC028BBDE8F08F00000A
:106450001B0008103E00080019000810360008054F
:106460009C0701202DE9F04F89B004464FF0000849
:10647000A768627801A9BA48FBF70AFAA7F1A160F8
:10648000B84DDFF8E49234384FF001064FF0020ABD
:106490004FF0030B06D001283ED002287CD0032801
:1064A0001FD14AE02078E8B1627808212846FCF73D
:1064B000BAFB002815D021208DF818008DF811A006
:1064C000627804A94846FDF77BFA8DF811B062782E
:1064D00004A94846FDF774FA627808212846FCF7BB
:1064E0001BF9EAE09F48627807A9C01CFBF7D0F9C6
:1064F00007980828F5D19D4F02980021C0B202905C
:10650000019861F31F2001908DF80460627801A961
:106510009348FDF755FAD0E02069FA28E1D961786F
:106520002846FCF777FB0028DBD1904F7F1C627870
:1065300008212846FCF7C8FBBFE0207800287DD161
:1065400000252E468748627808A91230FBF7A0F98B
:106550009DF8202072B300204FF00A0CB2FBFCF330
:10656000DFF80CE20AE05EF82010002903DA21F0DF
:1065700000410E4300E00D43401CC0B29842F2D3EC
:106580000020B2FBFCF1494201EB810102EB410129
:10659000CBB2774A24320BE069E052F82010002990
:1065A00003DA21F000410E4300E00D43401CC0B26D
:1065B0009842F2D30198B6EB102F21D018208DF815
:1065C00018008DF811A00198000AB0430590627878
:1065D00004A94846FDF7F4F98DF811A0019826EAC0
:1065E0001020059023208DF81800627804A94846F1
:1065F000FDF7E6F9019866F31F2001904FF00108BE
:106600000298B5EB102F23D018208DF818008DF8C4
:1066100011B00298000AA8430590627804A9484680
:10662000FDF7CEF98DF811B0029825EA10200590FB
:1066300023208DF81800627804A900E016E048468F
:10664000FDF7BEF9029865F31F2002904FF0010894
:10665000444862780821C01CFCF7E5FA08B9434FAA
:106660007F1E2069C82828D9404F7F1C25E001984B
:106670002421C0B20F25E02701282AD01E2202289B
:106680003ED0032853D08DF804608DF818208DF883
:1066900011A08DF81370627804A94846FDF790F9AF
:1066A0008DF811B08DF81350627804A94846FDF7B3
:1066B00087F94FF001082D4FBF1CB8F1000F04D02F
:1066C000627801A92648FDF77BF909B03846BDE894
:1066D000F08F8DF804A08DF818108DF811A08DF8AA
:1066E0001350627804A94846FDF76AF98DF811B095
:1066F0008DF81370627804A94846FDF761F9D8E770
:106700008DF804B08DF818208DF811A08DF8135075
:10671000627804A94846FDF753F98DF811B08DF859
:106720001370627804A94846FDF74AF9C1E70420CE
:106730008DF804008DF818108DF811A08DF81370E5
:10674000627804A94846FDF73BF98DF811B08DF841
:106750001350627804A94846FDF732F9A9E7000012
:106760001A0008104000080019000810350008053C
:10677000AC0701202DE9F04F87B00446A5688A4F89
:10678000A5F1A160DFF824A234384FF003084FF0E0
:1067900002090CD0DFF818B201280BF1010651D024
:1067A0004FF0000A04287DD005281FD164E020782E
:1067B000E8B1627804215046FCF735FA002815D07C
:1067C00021208DF814008DF80D90627803A93846C9
:1067D000FDF7F6F88DF80D80627803A93846FDF7CD
:1067E000EFF8627804215046FBF796FFD8E06F4837
:1067F000627806A9C01CFBF74BF806980428F5D16F
:106800006B4DED1E694862780DF10901001DFBF723
:106810003FF89DF80910032910D01B208DF80800BF
:106820008DF80A100D20FCF7F5F98DF809005E4887
:10683000627801A9401CFDF7C3F8B1E01A208DF879
:106840000800EDE72069FA2813D961785046FCF773
:10685000E1F900280DD1627804215046FCF734FAA2
:1068600052489DF8092010211330FCF7DCF908B1DB
:106870005D4695E0354693E02078C0B118208DF84C
:106880001400FF208DF80F00CDF810A08DF80D90AA
:10689000627803A93846FDF793F88DF80D80627889
:1068A00003A900E01CE03846FDF78AF878E03E488E
:1068B000627801A9401CFAF7EBFF3C489DF80920DB
:1068C00010211330FCF7AFF900B15D46374862780C
:1068D0000421C01CFCF7A7F9E0BB354D2D1F5FE07C
:1068E000DFF8C4B062780BF1010B01A95846FAF742
:1068F000CFFF207880B19DF80A2020210B20FCF7E3
:1069000092F970B319208DF81400FE208DF80F0055
:1069100001208DF804002EE024489DF80920102164
:106920001330FCF780F900B935462048627804211D
:10693000C01CFCF778F908B91D4D2D1F9DF80A20E1
:1069400020210B20FCF76FF928B1019810F0FF0F00
:1069500026D1354624E00198C0B2012820D1354621
:106960001EE0FFE79DF808008DF81400FF208DF869
:106970000F008DF804A0627801A95846FDF720F8B1
:10698000CDF810A08DF80D90627803A93846FDF778
:1069900017F88DF80D80627803A93846FDF710F8D6
:1069A00007B02846BDE8F08F190008104000080025
:1069B000380008052DE9F04F85B00446A568DFF8DA
:1069C0003CA1A5F1A160DFF838B134384FF00106E1
:1069D000AAF103080BD04B4F01282CD04FF0000830
:1069E0004FF0FF09022835D0032818D144E0207861
:1069F000B0B1627801214046FCF715F9002879D042
:106A00008DF8016021208DF80800627869465846AB
:106A1000FCF7D6FF627801214046FBF77DFE69E076
:106A2000627803A95046FAF733FF0398012861D131
:106A3000344DAD1E5EE02069FA285BD9617840468E
:106A4000FCF7E8F8F0BB3D46627801214046FCF7D0
:106A50003BF94FE02078A8BB8DF80160CDF80480A9
:106A60008DF8039025208DF8080062786946584615
:106A7000FCF7A6FF3D463DE0207818BB1F48627832
:106A800004A93C38FAF704FF04983146401C8640BC
:106A9000761E0496CDF804808DF801108DF80390D1
:106AA00018208DF80800627869465846FCF788FF80
:106AB00004991F2088438DF803001A208DF80800E0
:106AC000627800E016E069465846FCF779FF0498C2
:106AD0008DF8030019208DF8080062786946584641
:106AE000FCF76EFF627801215046FCF79CF808B96C
:106AF000044DED1E05B02846BDE8F08F42000800A9
:106B000019000810370008052DE9FF410546AE6859
:106B10006A7803A92648FAF7BBFEA6F1A160254FC3
:106B2000303808D02449012820D004283CD10398CB
:106B300098B30E4638E02878A8B111208DF80800E7
:106B400000240398C00706D08DF800406A78694693
:106B50003846FCF735FF641CE4B203984008039004
:106B60000C2CEED320E0144E761C1DE02878A8B142
:106B70000E208DF8080000240398C00706D08DF879
:106B800000406A7869463846FCF71AFF641CE4B294
:106B90000398400803900C2CEED305E0039808B14D
:106BA0000E4601E0044E361D04B03046BDE8F081CB
:106BB0001D00080019000810300008052DE9F04FED
:106BC00004462DED048B8BB04FF0000BD4F808A0D9
:106BD000627802A9FE48FAF75BFEAAF1A160FD4DBA
:106BE000FD4F34384FF002084FF0030608D001285B
:106BF00042D0B2EE049A022851D003281FD13AE1C4
:106C00002078E8B1627801212846FCF70CF80028CA
:106C100015D021208DF81C008DF81580627805A90B
:106C20003846FCF7CDFE8DF81560627805A9384628
:106C3000FCF7C6FE627801212846FBF76DFDDCE11A
:106C4000E44862780AA9C01CFAF722FE0A980128D3
:106C5000F5D1DFF888A3029820F0FF00C1B20290BE
:106C6000039861F31F20010A0390029861F31F202B
:106C700002904FF0010BC0E12069FA28DFD961785A
:106C80002846FBF7C7FF0028D9D1DFF850A30AF147
:106C9000010A627801212846FCF716F8ADE1207858
:106CA0000028CCD100250695FF208DF817004FF065
:106CB00018098DF81C908DF81560627805A9384682
:106CC000FCF77EFE8DF81580627805A93846FCF742
:106CD00077FEC048627804A9001DFAF7D9FD039831
:106CE000C0B2022830D025208DF81C008DF8156028
:106CF000627805A93846FCF763FE8DF81580627846
:106D000005A93846FCF75CFEB2486178C01DFBF768
:106D100081FF00EE100AB8EE408AAE486178801D0F
:106D2000FBF778FF00EE100AF8EE408AAC4918EE47
:106D3000900A88420CD118EE100A884208D14FF010
:106D4000000B4FF0000A3DE026208DF81C00CDE737
:106D500038EEC80A10EE100ADDF79AFE41EC100B6F
:106D6000DBF74BFF9FED9F1B51EC100B53EC112BEE
:106D7000DDF7FEFD03D24FF0FF0BDA4622E088EE8E
:106D8000090A01F06FFD42B288EE890A01F06AFD3E
:106D900043B24FF0000AD34606959449102A00DB0F
:106DA000002231F812005FEA004C04D520F40040C4
:106DB00040EA0B0B01E040EA0A0A9A4202D0521C58
:106DC00052B2EBE78DF815808DF817B08DF81C9056
:106DD000627805A93846FCF7F3FD8DF815608DF84B
:106DE00017A08DF81C90627805A93846FCF7E8FDDD
:106DF000DFF8DC91627809F1030969464846FAF741
:106E000047FD9DF8102008210A20FBF70CFF48B130
:106E100027208DF81C009DF8040040F040008DF8FC
:106E2000040008E024208DF81C009DF8040020F0E8
:106E300040008DF80400627869464846FCF7C0FDC2
:106E40008DF815808DF817B0627805A93846FCF7E3
:106E5000B7FD8DF815608DF817A0627805A9384642
:106E6000FCF7AEFD8DF808504FF0010BDFF86CA178
:106E70000AF1020AC1E0207800287DD155486178E6
:106E8000001DFBF7C7FE9DF81010884275D15148D0
:106E9000627809A9401DFAF7FBFC4E48627808A900
:106EA0000830FAF7F5FC0025A94600208DF81700F8
:106EB0009DED090AF8EE400A80EE890A02F04AFCCC
:106EC000014608989622B0FBF2F20892881A40B266
:106ED00011444AB2454BC03B18E0002803DA00F1E8
:106EE000300149B206E02F2803DDA0F1300149B29C
:106EF00000E0014653F82110002904DA21F0004196
:106F000041EA090900E00D43401C40B29042E4DD33
:106F10000298B9EB102F22D018208DF81C008DF8A4
:106F200015800298000A20EA09000690627805A9F7
:106F30003846FCF745FD8DF81580029829EA1020A7
:106F4000069023208DF81C00627805A93846FCF7CE
:106F500037FD029869F31F2002904FF0010B039850
:106F6000B5EB102F24D018208DF81C008DF815607B
:106F70000398000AA84301E029E03CE0069062780B
:106F800005A93846FCF71CFD8DF81560039825EA25
:106F90001020069023208DF81C00627805A9384641
:106FA000FCF70EFD039865F31F2003904FF0010BD3
:106FB000084862780121C01CFBF735FEC0B1029879
:106FC00010F0FF0F19D0DFF814A00AF1010A14E045
:106FD0001A000810400008001900081035000805C4
:106FE0000000E14400000000008036401C07012042
:106FF000DFF824A001E0DFF820A0BBF1000F04D0EF
:10700000627802A90548FCF7DBFC0BB05046BDECEA
:10701000048BBDE8F08F0000340008051A0008104A
:107020002DE9F04F89B004464FF00008A768627858
:1070300001A9D148FAF72CFCA7F1A160CF4DDFF8E8
:10704000409334384FF001064FF0020A4FF0030B23
:1070500006D001283ED002286FD003281FD14AE075
:107060002078E8B1627802212846FBF7DCFD002891
:1070700015D021208DF818008DF811A0627804A990
:107080004846FCF79DFC8DF811B0627804A948468B
:10709000FCF796FC627802212846FBF73DFB5CE199
:1070A000B648627807A9C01CFAF7F2FB07980228D5
:1070B000F5D1B44F02980199C0B20290002060F35C
:1070C0001F2101918DF80460627801A9AA48FCF79C
:1070D00077FC42E12069FA28E1D961782846FBF77C
:1070E00099FD0028DBD1A74F7F1C6278022128463A
:1070F000FBF7EAFD31E120780028D0D100252E46AB
:107100009E48627808A91130FAF7C2FB9DF820006A
:107110000A2801D10020089000209DF820200A2193
:10712000B2FBF1F30893984A0BE052F820100029C3
:1071300004DA21F000410E4301E083E00D43401CDE
:10714000C0B29842F1D38D48627808A91130FAF79D
:107150009FFB00209DF820100A22B1FBF2F2524260
:1071600002EB820201EB4201CBB20893864A243241
:107170000AE052F82010002903DA21F000410E4302
:1071800000E00D43401CC0B29842F2D30198B6EB28
:10719000102F21D018208DF818008DF811A001981B
:1071A000000AB0430590627804A94846FCF708FC41
:1071B0008DF811A0019826EA1020059023208DF863
:1071C0001800627804A94846FCF7FAFB019866F3B8
:1071D0001F2001904FF001080298B5EB102F21D02D
:1071E00018208DF818008DF811B00298000AA843F5
:1071F0000590627804A94846FCF7E2FB8DF811B0CF
:10720000029825EA1020059023208DF81800627856
:1072100004A94846FCF7D4FB029865F31F200290AE
:107220004FF00108554862780221C01CFBF7FBFCB7
:1072300008B9544F7F1E2069B0F5C87F01D9514F5E
:107240007F1C8AE001982621C0B225220F25E02765
:10725000012809D020234FF01F0C022822D0032838
:107260003ED004285BD074E08DF804A00298C0B230
:10727000022814D08DF818208DF811A08DF8135025
:10728000627804A94846FCF79BFB8DF811B08DF895
:107290001370627804A94846FCF792FB59E08DF818
:1072A0001810E9E78DF804B00298C0B2022814D093
:1072B0008DF818C08DF811A08DF81350627804A9CC
:1072C0004846FCF77DFB8DF811B08DF8137062789D
:1072D00004A94846FCF774FB3BE08DF81830E9E759
:1072E00004208DF804000298C0B2022814D08DF852
:1072F00018208DF811A08DF81370627804A9484603
:10730000FCF75EFB8DF811B08DF81350627804A97C
:107310004846FCF755FB1CE08DF81810E9E78DF89E
:1073200004600298C0B2022823D08DF818C08DF8EE
:1073300011A08DF81370627804A94846FCF740FB51
:107340008DF811B08DF81350627804A94846FCF707
:1073500037FB4FF001080B4FBF1CB8F1000F04D0F2
:10736000627801A90448FCF72BFB09B03846BDE858
:10737000F08F8DF81830DAE71A0008104000080086
:107380001900081035000805AC0701202DE9F04769
:1073900088B00446A568DFF8EC91A5F1A160DFF89C
:1073A000E88134384FF00007A9F103060AD001281C
:1073B0002BD0DFF8D0A102280AF1320A35D00328F9
:1073C0006AD160E02078B0B1627801213046FBF7E5
:1073D0002AFC002860D08DF8057021208DF80C0063
:1073E000627801A94046FCF7EBFA62780121304649
:1073F000FBF792F950E0627805A94846FAF748FA97
:107400000598012848D1614D46E02069FA2843D902
:1074100061783046FBF7FEFBA0BB5C4D6D1C6278CB
:1074200001213046FBF750FC36E0207850BB8DF848
:107430000570029724208DF80C0003208DF80700BA
:10744000627801A94046FCF7BBFA27208DF80C00B2
:107450003C208DF80700627801A94046FCF7B0FA9D
:1074600025208DF80C00C0208DF80700627801A956
:107470004046FCF7A5FA627800215046FCF7E2F896
:10748000424DAD1C08E03F4E2078143640B1627882
:1074900000213046FCF7D6F808B02846BDE8F08752
:1074A0003848627807A9C01CFAF7F2F9627804A993
:1074B0003046FAF7EDF99DED040AB8EE400A34497A
:1074C000DFED340A10EE100A884201DDB0EE600AEA
:1074D000B5EEC00AF1EE10FA0ED070EEC00A9FEDC4
:1074E0002E1A80EE810AF3EE080A20EE200ABCEE86
:1074F000C00A10EE106A00E00026FEB1627806A90C
:107500005046FAF7C5F906980121864217D901FAC3
:1075100000F1029100F101000690627806A9504640
:10752000FCF74EFA8DF8057023208DF80C008DF8CD
:107530000770627801A94046FCF742FA17E016D2BC
:1075400001FA00F10291A0F101000690627806A90B
:107550005046FCF735FA8DF805701D208DF80C00AB
:107560008DF80770627801A94046FCF729FA627825
:1075700001214846FBF757FB00288DD1034D6D1EB6
:107580008AE70000410008001900081035000805CE
:107590000000B4420000B442000058422DE9F04F10
:1075A00089B004460026A568627801A9B648FAF7B2
:1075B0006FF9A5F1A161B548DFF8D492DFF8D4B234
:1075C00034394FF000084FF001070AD0DFF8C8A2A5
:1075D000012951D0AF480D3802295DD0032928D1A7
:1075E000CAE0217831B3627802218046FBF71BFBA9
:1075F00000281ED021208DF814008DF80D706278BF
:1076000003A94846FCF7DCF914208DF81400FF208C
:107610008DF80F003F208DF80E008DF80D70627808
:1076200003A94846FCF7CCF9627802214046FBF7F3
:1076300073F81BE19548627807A9C01CFAF728F98E
:1076400007980228F5D1944D6D1E01988DF80A8097
:1076500068F30700C1B261F31F2001908B48627884
:107660000DF10901401DFAF713F96278002158461F
:10767000FBF7E8FF0126F9E02169FA29D9D96178F9
:107680000746FBF7C7FA0100D3D1554662780221BD
:107690003846FBF719FBE9E0217881B16178FBF707
:1076A000B9FAC2B208A97D48FAF7F2F89DF82000AD
:1076B000E8B364284CD30020FF2200214BE001985E
:1076C000050E0198C0F3074A0198C0F3072BCDF8C7
:1076D0001080FF208DF80F0018208DF814008DF811
:1076E0000D70627803A94846FCF76AF98DF80D70B1
:1076F000CDF810804DB124208DF814008DF80F5076
:10770000627803A94846FCF75BF9BBF1000F09D08A
:1077100027208DF814008DF80FB0627803A9484631
:10772000FCF74EF9BAF1000F0BD0252000E00BE07A
:107730008DF814008DF80FA0627803A94846FCF775
:107740003FF9554D6D1C91E0FF200022002102E021
:10775000012080227E21000440EA02200843019992
:10776000B0EB112F02D14C4D6D1C7FE0019960F3FD
:107770001F210191012679E02178E9BB8DF80D7078
:107780008DF80F806178FBF745FAC2B208A943482B
:10779000FAF77EF89DF8200000EE100AB8EE400AD5
:1077A000B5EEC00AF1EE10FA0CD09FED3D1AC0EE16
:1077B000010AB3EE080A20EE800ABCEEC00A10EE01
:1077C000105A00E00025627806A95846FAF760F8DA
:1077D0007DB30698854216D907FA00F7049700F1A1
:1077E000010006904FF023008DF81400627803A981
:1077F0004846FCF7E5F800E038E0627806A958460C
:10780000FCF7DEF82AE029D207FA00F70497A0F186
:10781000010006904FF01D008DF81400627803A956
:107820004846FCF7CDF8627806A95846FCF7C8F838
:1078300014E0FFE7069888B1CDF818806FF07F401C
:10784000049018208DF81400627803A94846FCF7CC
:10785000B7F8627806A95846FCF7B2F80B48627888
:107860000221C01CFBF7DFF950B1554626B1627802
:1078700001A90548FCF7A4F809B02846BDE8F08F37
:10788000054DAD1EF2E700001C0008103F00080087
:1078900019000810740008003600080505000200F1
:1078A0000000C842F8B50446A568627801210A20A4
:1078B000FBF7B9F94FF0A06698B1627804210B206C
:1078C000FBF7B1F978B161780D20FBF7A3F9C2B2EB
:1078D00069462A48F9F7DCFF0098C00605D5012063
:1078E00004E03046F8BD3046F8BD0020244AA5F13A
:1078F000A061971E052933D2DFE801F0030B1C17A6
:107900002A00627801210B20FBF78DF9F8B13D4682
:1079100026E02178D9B920B92169C82901D91546AD
:107920001EE001281CD135461AE0012818D1144D5B
:107930006D1E15E0217851B9012801D015460FE0E0
:10794000206940F2DC5188420AD90D4D6D1C07E0D8
:10795000217829B930B12069B0F57A7F00D33D464E
:107960002846F8BD3D46627820210B20FBF7ACF994
:107970006278D0210B20FAF7CFFEF1E75300080020
:1079800003000005F8B50446A568627801210A20C5
:10799000FBF749F94FF0A06698B1627804210B20FB
:1079A000FBF741F978B161780D20FBF733F9C2B2EA
:1079B00069462948F9F76CFF0098C00605D50120F3
:1079C00004E03046F8BD3046F8BD0020234BA5F159
:1079D000A062DF1E40F2DC51062A2FD2DFE802F05F
:1079E000030B2E26171B627801210B20FBF71BF9D6
:1079F00020B33D4622E0217801BB012804D1216952
:107A0000642901D91D4619E0C0B9354616E0A8B968
:107A1000124D6D1C12E0227882B908B11D460DE0AE
:107A2000206988420AD90D4D6D1E07E022782AB9D7
:107A3000012805D02069884200D33D462846F8BD7C
:107A40003D46627840210B20FBF73EF96278B02179
:107A50000B20FAF761FEF1E753000800040000056F
:107A6000F8B50446A568627801210A20FBF7DBF827
:107A70004FF0A06798B1627804210B20FBF7D3F890
:107A800078B161780D20FBF7C5F8C2B269462B4882
:107A9000F9F7FEFE0098C00605D5012004E038463F
:107AA000F8BD3846F8BD0020254EBD4209D07142D0
:107AB00069180ED040F6AC52022928D003292BD1E8
:107AC00011E0627801210B20FBF7ADF820B33546B9
:107AD00022E0217801BB012802D0194DED1C1BE0EA
:107AE000174DAD1C18E02178B1B908B1354613E047
:107AF0002069904210D93546627810210B20FBF79F
:107B0000E3F86278E0210B20FAF706FE04E0217822
:107B100011B9012802D035462846F8BD20699042A7
:107B2000FAD93546627880210B20FBF7CDF86278D0
:107B300070210B20FAF7F0FDEEE70000530008007B
:107B4000010000052DE9F041154D0C46002155F8C6
:107B500024201C2303EB810696597668864203D0C5
:107B6000491CC9B22029F5D34FF0FF37202914D082
:107B700003EB8106394690598069D9F755FA55F8D3
:107B800024008059827A4168806901EB02110C68F7
:107B9000D9F780FA2046BDE8F0813846FBE70000BF
:107BA000007801202DE9F04106460D4614460027D5
:107BB00028684FF0A161A0F1A160052855D2DFE847
:107BC00000F0030D252F4E007E2E4ED18A21204637
:107BD000D8F7B7FE26702648286046E06088304314
:107BE0006080B4F8861021B94FF6FF7202EA0020D7
:107BF0006080491C88B2A4F88600012835D900208D
:107C0000A4F886001A48401C28602EE084F885609D
:107C100026710120A4F888001548801C286024E003
:107C2000863414F8010C304404F8010C6088401CC0
:107C3000608034F88629601D1654B4F886007F28C9
:107C40000BD2401CA4F886006088B4F888108842E3
:107C50000BD10748C01C286007E0296005E014F834
:107C6000850F30442070296001273846BDE8F08137
:107C700001000805F0B504462DED028B83B0A56820
:107C8000434FA5F1A1601538424EDFED438AB7EEB0
:107C9000088A082876D2DFE800F024537575754805
:107CA0000404207818B11120DAF7E8FF6AE0DBF766
:107CB00029F800EE100ADFED390AB8EE400A80EE2E
:107CC000801A8DED021A627802A93846FBF778FE19
:107CD000B54202D12F4DAD1F54E01120DAF7CEFF8F
:107CE00050E0207818B10820DAF7C8FF4AE062783F
:107CF00001A93846F9F7CCFDDBF704F800EE100ACD
:107D0000DDED010AB8EE400A20EE280A20EE200A36
:107D100020EE080A8DED020A1D48627802A9401F74
:107D2000FBF74EFE1B4D6D1E2CE0207818B1122083
:107D3000DAF7A4FF26E0DAF7E5FF164D6D1F21E024
:107D4000207818B10920DAF799FF1BE0627801A9C1
:107D50003846F9F79DFDDAF7D5FF00EE100ADDEDA4
:107D6000010AB8EE400A20EE280A20EE200A20EE92
:107D7000080A8DED020A0648627802A9001FFBF787
:107D80001FFE354603B02846BDEC028BF0BD000057
:107D9000080008011B0008050000803948E19A45E9
:107DA0002DE9F04F89B00446A568627801A9FB4827
:107DB000F9F76EFDFA4EA5F1A160401F15D09DF8B0
:107DC0000800410704D520F004008DF8080035466E
:107DD000A5F1A1603F3808D0B54206D062781821DD
:107DE000F048FAF720FF00B13546ED49EC4F1B395A
:107DF000681A2837A1F1010901F101084FF0060ABC
:107E00004FF0070B8D4272D00BDCA5F1A160A0F101
:107E10000500082828D2DFE800F0132727B1F2F187
:107E2000F0EF1B2821D006DC012872D0022871D087
:107E3000032819D113E232286DD04328F9D1F1E398
:107E4000D84862780221401CFAF73EFFD54F62788D
:107E500002213846FAF7E7FE002805D062780121B2
:107E60003846FAF759FC354605E22078F0B3CD489C
:107E700062780021401DFBF7E5FB00208DF8200013
:107E8000C64E6278361F06A93046FBF799FD0420DE
:107E90008DF820009DF80800000711D4C1486278D1
:107EA00000212B30FBF7CEFBBE4862780021293041
:107EB000FBF7C8FBBB48627800212A30FBF7C2FB06
:107EC000032201210A20FAF7AEFE58B1B5486178C5
:107ED000801DFAF79FFE8DF81800627806A93046DB
:107EE000FBF76EFD042201210A2001E014E0CFE33C
:107EF000FAF799FE0028B7D0AA486178C01DFAF7B2
:107F000089FE8DF81800627806A93046FBF758FD07
:107F1000B1E177E38CE0FDE3A24861782830FAF71D
:107F200079FE58B99F4861782630FAF773FE28B970
:107F30009C4861782730FAF76DFE18B19DF808006B
:107F4000000791D59DF8080020F008008DF8080082
:107F5000627818219348FAF766FE10B1904D1735F4
:107F600089E19DF80500C00702D08D4D203D82E1DA
:107F70009DF808000006CBD53D467CE1207840B155
:107F80009DF805008DF807009DF804008DF80600A7
:107F900071E19DF80500810708D562789DF804001D
:107FA000002101F0B7F87E4D1F3D64E1410707D580
:107FB00061789DF8040000F0C3FE794D1D3D5AE143
:107FC000010706D561789DF8040000F0B9FE4D4622
:107FD00051E1C10607D561789DF8040000F0E0FF8B
:107FE0006F4D1B3D47E181060AD561789DF804007D
:107FF00000F0A6FE4546FAE30AE296E194E0ECE0E2
:10800000410602D5664D193DF1E3000607D56178BA
:108010009DF8040000F094FE614D183DE7E362789E
:108020009DF80400012101F075F85D4D1E3DDEE371
:10803000207870B35B4861781030FAF7EBFD8DF86B
:10804000180005208DF82000544E6278361F06A9CE
:108050003046FBF7B5FC534861781D30FAF7DAFD7E
:10806000014650486278401DFAF72EFE9DF8040044
:1080700003284FD08DF820B04A486178C01DFAF728
:10808000C9FD8DF81800627806A93046FBF798FC08
:10809000ADE3FFE79DF804109DF80600814201D092
:1080A000354615E09DF80500820702D53C4D1F3D81
:1080B0000EE0400601D435460AE00020FBF718FE2A
:1080C000022820D062789DF80410012000F0B0FD55
:1080D000A5F1A1600F3885D0324862780021401D9B
:1080E000FBF7B0FA02208DF820002E48617810309E
:1080F000FAF790FD8DF818002848627806A9001F4D
:10810000FBF75EFC73E362789DF80410002000F03A
:108110008FFDDDE78DF820A022486178801DFAF7F9
:1081200079FD8DF81800AEE720784FF4803830B133
:108130009DF8042041460B20FAF7EEFA57E39DF82C
:1081400004109DF80600814203D19DF80500012826
:1081500001D035464BE39DF80800000601D53D46A9
:1081600045E3206941F28832904291D90020FBF723
:10817000BFFD022818D00B4861781D30FAF74AFD80
:10818000014608486278401DFAF79EFD9DF80420DC
:1081900041460B20FAF747FDC0B128E31D00081047
:1081A0002800080518000800FE4E61783046FAF7EE
:1081B00031FD0028A6D0627800213046FBF742FA54
:1081C00062780121FF2000F0A5FF10E39DF8042054
:1081D00000212320FBF736FA09E32078002891D10B
:1081E0009DF804109DF80600814201D03546FEE25C
:1081F0009DF80500020601D5EB4DF8E2800701D499
:108200003546F4E29DF80800000601D53D46EEE251
:108210000020FBF76DFD022813D062789DF8041052
:10822000012000F005FDDF4861781C38FBF760FD98
:1082300002280DD062789DF80410012001F02AFA7E
:10824000D5E262789DF80410002000F0F1FCEAE726
:1082500062789DF80410002001F01CFAC7E2207833
:1082600050B1D04861781830FAF7D4FC01466278F2
:10827000CC48FAF729FDBAE29DF804109DF80600F3
:10828000814201D0354629E09DF80500820601D5DE
:10829000454623E0020609D4354640071ED59DF821
:1082A000080040F008008DF8080017E00020FBF7F8
:1082B0001FFD02282BD062789DF80410012000F0E9
:1082C000B7FCB84861781C38FBF712FD022825D0AE
:1082D00062789DF80410012001F0DCF9A5F1A1609D
:1082E000103884D062780021AE48FBF7ABF9022049
:1082F0008DF82000AB4861780B30FAF78BFC8DF8D5
:108300001800627806A9A948FBF75AFB6FE2627869
:108310009DF80410002000F08BFCD2E762789DF8F5
:108320000410002001F0B6F9D8E72078002887D1A2
:108330009DF804109DF80600814201D0354656E2B2
:108340009DF80500020701D54D4650E2820601D591
:1083500045464CE2420709D4354640068BD59DF888
:10836000080040F008008DF8080040E29DF8080081
:10837000000601D53D463AE20020FBF7B9FC022891
:1083800032D062789DF80410012000F051FC85483D
:1083900061781C38FBF7ACFC02282CD062789DF881
:1083A0000410012001F076F99DF808004006ADD5D3
:1083B00020694FF40071642824D99DF804200B2013
:1083C000FAF731FC0028A1D0784E6278761C03A918
:1083D0003046F9F75DFA01208DF80C00627803A9A8
:1083E0003046FBF7EDFA02E262789DF804100020B7
:1083F00000F01EFCCBE762789DF80410002001F02D
:1084000049F9D1E79DF804200B20FAF785F9EEE150
:10841000207848B3634861781630FAF7FBFB0146D1
:1084200062786048FAF750FC9DF8040003287DD07C
:108430008DF820B05B4861780C30FAF7EBFB8DF8D3
:108440001800627806A95948FBF7BAFA9DF804208B
:108450004FF480610B20FAF75FF99DF8080020F0D7
:1084600030008DF80800C2E19DF804109DF8060068
:10847000814201D035468CE09DF80500420702D5C7
:10848000494D6D1F85E0820601D5454681E0000714
:1084900001D435467DE09DF80800000601D53D4633
:1084A00077E00020FBF724FC02284CD062789DF88E
:1084B0000410012000F0BCFB3A4861781C38FBF73F
:1084C00017FC022846D062789DF80410012001F0C4
:1084D000E1F84FF480669DF8042031460B20FAF74E
:1084E000A2FBA0B19DF8042031460B20FAF714F945
:1084F0002E4E6278761C03A93046F9F7C9F901209F
:108500008DF80C00627803A93046FBF759FA9DF804
:108510000800C10625D581063BD440F020008DF827
:10852000080005208DF82000617800E067E01D4814
:108530000A30FAF76FFB8DF81800627806A91B481D
:10854000FBF73EFA25E062789DF80410002000F069
:108550006FFBB1E762789DF80410002001F09AF8F3
:10856000B7E7810615D520F020008DF808009DF8AA
:108570000400032840D08DF820B00A4861780A3002
:10858000FAF748FB8DF81800627806A90748FBF750
:1085900017FA4D452FD0034861781630FAF73AFBA9
:1085A000014605E01D00080010000805190008102C
:1085B00062789448FAF7B0F801208DF820009148CD
:1085C00061780C30FAF726FB8DF818008E4E627831
:1085D00006A93046FBF7F4F902208DF820008948FF
:1085E00061780A30FAF716FB8DF81800627806A950
:1085F0003046FBF7E5F9FAE08DF820A0BDE78DF8ED
:1086000020A017E72078A0BB9DF804109DF8060075
:10861000814201D03546EAE09DF80500420702D5C7
:108620007A4DE4E0B7E0020701D54D46DFE0800671
:1086300001D43546DBE09DF80800000601D53D4633
:10864000D5E00020FBF754FB022813D062789DF898
:108650000410012000F04CFA6A4861781C38FBF7DE
:1086600047FB02280DD062789DF80410012001F02C
:1086700011F8BCE062789DF80410002000F038FA90
:10868000EAE762789DF80410002001F003F8AEE0FC
:10869000207830B19DF8080020F003008DF8080024
:1086A000A5E09DF804109DF80600814201D03546F2
:1086B00027E09DF80500820601D5454621E0C00669
:1086C00001D435461DE09DF80800000601D53D4661
:1086D00017E00020FBF70CFB022833D062789DF8EE
:1086E0000410012000F0FCFB464861781C38FBF7C1
:1086F000FFFA02282DD062789DF80410012000F0C6
:10870000C9FF9DF80800C1072DD080076FD49DF8E0
:10871000040000E054E0032822D08DF820B039484E
:1087200061780B30FAF776FA8DF81800627806A9AE
:108730003548FBF745F99DF8080040F003008DF837
:10874000080054E062789DF80410002000F0C8FB97
:10875000CAE762789DF80410002000F09BFFD0E784
:108760008DF820A0DBE7800741D505208DF820009B
:10877000244861780B30FAF74DFA8DF818006278CA
:1087800006A92148FBF71CF99DF8080020F003001A
:108790008DF808002BE0207860B11A48627810212B
:1087A0002630FAF74FFF1748627801212430FAF794
:1087B00049FF1CE09DF80800000618D4354616E075
:1087C000207828B161789DF8040000F0F1F90EE0FE
:1087D0000C4F62787F1F08213846FAF724FA30B927
:1087E000627810213846FAF71EFA00B93546064875
:1087F000627801A9001DFBF7E3F809B02846BDE83F
:10880000F08F00001D000800190008100B0008057B
:1088100010EE100A1049884201DB9FED100A9FED0F
:10882000101AC0EE010AB2EE000A20EE800AFCEE39
:10883000C00A10EE900AC0B207280CD200EE900ACF
:10884000F8EE600A30EE600A10EE101AB1F17C5FAB
:1088500001DD401CC0B270470000344366E633437C
:108860000000344310EE100A1049DFED110A88426F
:1088700001DB30EE600A80EE201AB3EE000A21EE32
:10888000000AFCEEC00A10EE900AC0B20F280CD20B
:1088900000EE900AF8EE600A30EE600A10EE101A50
:1088A000B1F17C5F01DD401CC0B270470000B443F1
:1088B0000000B4432DE9FC470446A568644E627885
:1088C00012213046FAF7AFF9614FA6F101082B37B4
:1088D00000B3627802213046F9F71EFF6278182152
:1088E0004046FAF7A0F990B10220DAF711FA617860
:1088F0003846FAF78FF9C0B2617800F0E7FA002045
:10890000DBF72BFE627818214046F9F705FF514846
:10891000BDE8FC874F4EA5F1A160B61DDFF8309190
:108920002538A6F1010A4FF47A7109F103090828E4
:1089300007D2DFE800F00407288B6B427B89454DA6
:108940006D1C83E02078002819D141486178401CD3
:10895000FAF760F9401E00EB4001C1EBC01021693D
:10896000B1EBC00F72D9627801A93846F8F790FFD1
:108970009DF80400032803D0042801D0354665E0A3
:10898000344DAD1C62E0207828B162780821404661
:10899000FAF79AF95AE02069884257D9627810218B
:1089A0004046FAF791F90120DBF7D7FD6278002104
:1089B0004846FAF747FE554648E0207818B10120AE
:1089C000DAF7A6F942E04F46627869463846F8F78A
:1089D0005FFF1F486178801CFAF71CF940F2537161
:1089E00048430099B1EB401F01D935462EE020697C
:1089F00040F6B832904229D908440090627869461E
:108A00003846FAF7DDFF134D2D1D1FE0207858B1D1
:108A10000220DAF77DF961783846FAF7FBF8C0B240
:108A2000617800F053FA11E055460FE0207828B144
:108A3000627804214046FAF747F907E02069884246
:108A400004D9044DED1D01E0DBF714FE28465FE775
:108A500019000800250008052DE9FF4106461746C4
:108A6000032921D004291DD139461F48FAF7D2F82D
:108A7000C5B21D4839460C30FAF7CCF80446DFF889
:108A800068803A46A8F1020803A94046F8F700FFBB
:108A9000012E16D00398204204D13A462146404682
:108AA000FAF712F9BDE8FF810F483946401EFAF780
:108AB000B1F8C5B20C4839460B30FAF7ABF80446AA
:108AC000DDE703982042EDD03A4621464046F9F7CB
:108AD00023FE02208DF808008DF800503A466946C2
:108AE0000248FAF76DFFDDE71F00080019000810C3
:108AF0002DE9F04704460F46904639462320FAF701
:108B000089F82A4DEE1E80B3681F00F103092CB1CD
:108B100042460221FAF787F8B0B11AE04246022134
:108B2000FAF781F820B1424600214846FAF78AFD5B
:108B3000424608213046FAF776F850B34246002103
:108B40002846FAF77FFD2AE0424602214846FAF716
:108B500079FD424608213046FAF765F8C8B9424621
:108B600008212846FAF76EFD19E0FFE734B14246C6
:108B700004213046FAF757F860B110E0424604216C
:108B80003046FAF750F820B1424600212846FAF75D
:108B900059FD04E0424604212846FAF753FD4246B7
:108BA00039462046BDE8F047FFF756BF43000800AE
:108BB00070B586B004460D462A4600211A48FAF7D9
:108BC00041FD00208DF81400184E2A4603A93046B6
:108BD000FAF7F6FE032C19D002208DF804000720C6
:108BE0008DF8140010482946801CFAF713F88DF808
:108BF0000C002A4603A93046FAF7E2FE0B482A4643
:108C00006946401CFAF7DCFE06B070BD01208DF805
:108C1000040006208DF8140003482946401CF9F78B
:108C2000F9FF8DF80C00E4E71D000800190008109A
:108C30002DE9F04704468946924649462320F9F734
:108C4000E9FF3E4DEF1C002858D0AE1E05F101088B
:108C50003CB152464FF480410B20F9F7E4FF10B3CA
:108C60002CE0524602213046F9F7DDFF20B1524692
:108C700000214046FAF7E6FC524601212846F9F762
:108C8000D2FF20B1524600213846FAF7DBFC5246AB
:108C900004212846F9F7C7FF48B352460021384659
:108CA000FAF7D0FC43E0524602213046F9F7BBFF09
:108CB00020B9524602214046FAF7C4FC52464FF40E
:108CC00000410B20F9F7AFFF30B15246042128468E
:108CD000F9F7A9FF60B12AE0524601212846F9F7C9
:108CE000A2FF20B9524601213846FAF7ABFC1EE03C
:108CF000524604213846FAF7A5FC18E034B1524632
:108D000004212846F9F78FFF60B110E05246042194
:108D10002846F9F788FF50B1524600213846FAF745
:108D200091FC04E0524604213846FAF78BFC524687
:108D300049462046BDE8F047FFF78EBE40000800D8
:108D40002DE9F34F8DB006460122102109A8D7F76F
:108D5000F0FD31462320F9F75DFF0024594F4FF015
:108D600001084FF0060A4FF0070B4FF0020909AD5A
:108D7000002864D003A9781C0E9AF8F789FD01A990
:108D8000B81C0E9AF8F784FD032E43D00D208DF801
:108D9000200006A938460E9AFAF712FE8DF820B088
:108DA0008DF810908DF8089047480E99F9F732FF2A
:108DB0002C5445480E990B30F9F72CFF2C544148A0
:108DC00003A9401C0E9AFAF7FBFD3E4801A9801C3E
:108DD0000E9AFAF7F5FD0024285D30B18DF81840A1
:108DE00006A938460E9AFAF7EBFD641CE4B2082C8B
:108DF000F2D34FF40074324621460B20F9F713FFEB
:108E0000002804D0324621460B20F9F785FC0FB02C
:108E1000BDE8F08F0C208DF8200006A938460E9A88
:108E2000FAF7CEFD8DF820A08DF810808DF808801F
:108E300025480E99401CF9F7EDFE2C54B9E7032E96
:108E400035D08DF820B08DF810901F480E99F9F7A5
:108E5000E1FE2C5431462620F9F7DCFE012805D02E
:108E600019480E990930F9F7D5FE2C5431462620C1
:108E7000F9F7D0FE022805D013480E990830F9F70B
:108E8000C9FE2C540F4803A9401C0E9AFAF798FD0E
:108E90000024285D30B18DF8184006A938460E9A96
:108EA000FAF78EFD641CE4B2082CF2D3AFE78DF81C
:108EB00020A08DF8108004480E99401CF9F7AAFEF6
:108EC0002C54C7E7190008101E00080010B5DAF787
:108ED000C3FFDAF7C1FFBDE81040DBF73BB8000085
:108EE0002DE9F04704460F46904639462320F9F70E
:108EF00091FE2A4DEE1E80B3681F00F103092CB1CC
:108F000042460221F9F78FFEB0B11AE04246022133
:108F1000F9F789FE20B1424600214846FAF792FB54
:108F2000424602213046F9F77EFE50B34246002108
:108F30002846FAF787FB2AE0424602214846FAF71C
:108F400081FB424602213046F9F76DFEC8B9424620
:108F500002212846FAF776FB19E0FFE734B14246D2
:108F600004213046F9F75FFE60B110E0424604216B
:108F70003046F9F758FE20B1424600212846FAF75C
:108F800061FB04E0424604212846FAF75BFB4246B7
:108F900039462046BDE8F047FFF75EBD43000800B4
:108FA0002DE9F34F8BB006460122102107A8D7F711
:108FB000C0FC31462320F9F72DFE544F4FF0010835
:108FC0004FF006094FF0070A4FF0020B002407ADDF
:108FD000E0B301A9781C0C9AF8F75AFC032E36D09E
:108FE0008DF818A08DF808B049480C99F9F712FED1
:108FF0002C5447480C990930F9F70CFE2C5443487F
:1090000001A9401C0C9AFAF7DBFC00243E46285DBF
:1090100030B18DF8104004A930460C9AFAF7D0FC14
:10902000641CE4B2082CF2D339480C990A30F9F7E1
:10903000F1FD8DF8100005208DF8180004A93046C8
:109040000C9AFAF7BDFC0DB0BDE8F08F0AE08DF880
:1090500018908DF808802E480C99401CF9F7DAFD1D
:109060002C54C6E7032E45D08DF818A08DF808B013
:1090700027480C99F9F7CEFD2C5431462620F9F7F4
:10908000C9FD012805D022480C990930F9F7C2FD25
:109090002C5431462620F9F7BDFD022805D01C4886
:1090A0000C990830F9F7B6FD2C54184801A9401C5A
:1090B0000C9AFAF785FC00243E46285D30B18DF805
:1090C000104004A930460C9AFAF77AFC641CE4B20A
:1090D000082CF2D30E480C990A30F9F79BFD8DF855
:1090E000100005208DF8180004A930460C9AFAF7F4
:1090F00067FCA8E78DF818908DF8088004480C9953
:10910000401CF9F787FD2C54B7E700001900081040
:109110001E000800F0B587B00E461746274D6C1E9E
:10912000032802D0042817D02DE001208DF8080074
:1091300006208DF8180039462148F9F76BFD8DF8A7
:1091400010003A4604A92046FAF73AFC3A4601A92B
:109150002846FAF735FC16E002208DF808000720B3
:109160008DF8180016483946401CF9F753FD8DF864
:1091700010003A4604A92046FAF722FC3A4601A913
:109180002846FAF71DFC0E4839460A30F9F742FD29
:109190008DF8100005208DF818003A4604A92046E5
:1091A000FAF70EFC16B104218DF818103A4604A9FE
:1091B0002046FAF705FC07B0F0BD00001A000810C1
:1091C0001E0008002DE9F04F8DB00446A5686278B6
:1091D00009A9FA48F8F75CFBF84862780AA9801CEC
:1091E000F8F756FBF54862780CA9401CF8F750FBDD
:1091F0009DF828200BA90E20F8F74AFB627801A9F8
:10920000EF48F8F745FB0C98C10609D5EB486278A2
:109210001021401CF9F780FAEA480DB0BDE8F08F44
:10922000C00711D0E5489DF824101A38F9F7F2FC70
:109230009DF82810884207D1E0489DF82420182185
:109240004638F9F7F0FC08B12846E6E7DD4EDB4882
:10925000F61DA5F1A161DFF864A34039B71EDFF860
:1092600068B32930A6F106080AF1380A4FF0E1691F
:1092700018291BD2DFE801F0F30C1B2A3D5B9AF2A0
:109280001A1A1A1AF1F0EFEE1A1AEDECEBEAE9E805
:109290000C98000600D53D462078002806D162785B
:1092A00049465846FBF7FAFFC64DAD1CEDE10B9859
:1092B00010B1C44DED1CE8E120780028F6D16278A9
:1092C00049465846FBF7EAFF4546DEE10B9810B1E8
:1092D000207810B1D9E14546D7E162784946584631
:1092E000FBF7DCFF2069B0F5FA7FDFD3B54D2D1D0C
:1092F000CBE10B9931B10C99090600D53D46217897
:1093000011B10DE04546FAE762781021F9F78BFCC0
:1093100030B1AD489DF8242049460F30FBF7BEFF21
:10932000A94862784946401CFBF7B8FFADE12078B8
:109330000028BBD19DF806008DF810009DF80700AD
:109340008DF811009DF808008DF812009C48627895
:1093500004A9801FFAF734FB0B9830B1D7F792FDC0
:109360000B99401AB0F5FA7F03D261789748F7F766
:109370004BFD924862784FF40071401CF9F7CCF92C
:109380009148627849461430FBF788FF8B4C9DF872
:10939000241037342046F9F73DFC411C9DF8242069
:1093A0002046FAF74FF9874D16356EE10C990906FC
:1093B00000D445462178002987D1627801210546ED
:1093C000F9F731FC10B17F4D0D355EE16278022175
:1093D0002846F9F728FC10B17A4D0C3555E1627832
:1093E00004212846F9F71FFC10B1764D0E354CE1EB
:1093F000627808212846F9F716FC10B1714D0F3537
:1094000043E1627810212846F9F70DFC08B1354692
:109410003BE1627820212846F9F705FC10B1694D3F
:10942000133532E1627840212846F9F7FCFB10B190
:10943000644D143529E1627880212846F9F7F3FB61
:1094400070B1604D123520E181E09AE064E0DDE02A
:10945000D2E0E5E00CE101E1F6E0EBE0B8E011E19B
:109460009DF80400401CC0B28DF804009DF8051062
:10947000884202D901208DF804009DF8040000EB19
:10948000400101A8084481788DF81010C1788DF84A
:10949000111000798DF812004948627804A9801FE4
:1094A000FAF78EFA627801A94548FAF789FA0B981B
:1094B00030B1D7F7E7FC0B99401AB0F5FA7F03D229
:1094C00061784248F7F7A0FC3C4862784FF440715D
:1094D000401CF9F721F93C48627849461430FBF703
:1094E000DDFE364C9DF8241037342046F9F792FB08
:1094F000411C9DF824202046FAF7A4F89DF810009E
:10950000062803D0152804D03D46BEE02D4D153564
:10951000BBE02C4D1735B8E02069642801D93D46E1
:10952000B3E0264862784FF48071401CF9F77BFB6A
:1095300000280BD09DF824105046F9F76BFB411C16
:109540009DF824205046FAF77DF83D469DE02069BD
:10955000642801D93D4698E0184862784FF40071BC
:10956000401CF9F760FB38B39DF824105046F9F71A
:1095700051FB411C9DF824205046FAF763F83D4604
:1095800083E0104E2069B61D642801D935467CE081
:109590000A4862784FF40071401CF9F744FB58B157
:1095A0009DF824105046F9F735FB411C9DF8242006
:1095B0005046FAF747F8354667E000005E000800BD
:1095C00028000810400008050C00080703000801E7
:1095D000217821BB62781021F9F725FB28B19DF88D
:1095E000242049462A48FBF759FE627849465846E6
:1095F000FBF754FE3D4648E0207880B92448627865
:1096000049460C30FBF74AFE35463EE0207830B93B
:109610001F48627849460D30FBF740FE354634E07E
:10962000207820BB1A48627849460B30FBF736FE9B
:1096300035462AE02078D0B9154862784946083086
:10964000FBF72CFE354620E0207880B91048627880
:109650004946C01DFBF722FE354616E0207830B99A
:109660000B48627849460930FBF718FE35460CE096
:10967000207850B90648627849460A30FBF70EFE5A
:10968000354602E0207800B945462846C5E5000089
:109690001B00080770B5044616462320F9F7BAFAEE
:1096A000164D0100A5F103001AD064B13246022123
:1096B000F9F7B9FA002820D132462846BDE87040B3
:1096C0000221F9F7BFBF32460221F9F7ACFA0028B0
:1096D00013D032462846BDE870400021F9F7B2BFEA
:1096E00032460221F9F79FFA002806D03246284672
:1096F000BDE870400021F9F7A5BF70BD4200080029
:1097000010EE100A1049884201DB9FED100ADFEDD0
:10971000100A80EE201AB3EE080A21EE000ABCEE11
:10972000C00A10EE101AC8B217280BD2091A00EEA0
:10973000101AB8EE400A10EE101AB1F17C5F01DD8C
:10974000401CC0B2704700000000344366E633435B
:109750000000344310EE100A1049DFED110A884270
:1097600001DB30EE600A80EE201A9FED0E0A21EE3A
:10977000000AFCEEC00A10EE900AC0B22F280CD2EC
:1097800000EE900AF8EE600A30EE600A10EE101A51
:10979000B1F17C5F01DD401CC0B270470000B443F2
:1097A0000000B443000040422DE9F0411A4E144637
:1097B0000F46002156F824201C2303EB8105555940
:1097C0006D68854203D0491CC9B22029F5D32029F0
:1097D00012D003EB81054FF0FF3150598069D7F764
:1097E00023FC56F824004059477256F824100120F3
:1097F000495908721FB107E00920BDE8F08156F809
:10980000241000204959887256F824004059806974
:10981000D7F740FC0320F0E7007801202DE9F04164
:109820001E4E1446884603460327002056F824108F
:109830001C2202EB80054D596D689D4203D0401CEF
:10984000C0B22028F5D320281CD002EB800548594F
:109850004FF0FF318069D7F7E7FB56F82400424606
:10986000405901784068FBF761F956F824104959CE
:109870000A78824209D0887256F82410012049598A
:10988000087203E00920BDE8F081092756F824009A
:1098900040598069D7F7FEFB3846F4E7007801208D
:1098A00090F80080794C86B054F828008778D7F774
:1098B000E9FA54F8285081461C35D7F7E3FAA0EBB3
:1098C0000900B84201D3012000E0381AD7F79EFA08
:1098D000D7F7D8FA81460024CFE055F824004FF09E
:1098E000FF3A51468069D7F79FFB55F82400417A2B
:1098F00002297CD1017A867A01293FD04169C36867
:10990000A9EB01029A4272D30822436802EB0612C5
:109910004FF0000B9A58114441618DF8018055F8C1
:1099200024000930019055F824000169A9EB0100D9
:10993000049055F82400406800EB0610006802907F
:1099400055F82400C06803908DF800B055F8240045
:1099500041680C2000EB0610095800296DD06846BC
:109960008847824655F82400417A022965D00121B2
:10997000017255F82400417AD1B35EE000210172F2
:10998000D7F780FA55F82410042202EB061248613A
:1099900055F82410086155F824104868825C002AA4
:1099A0004FF0080202EB061280583ED042460C31BE
:1099B000F7F76EFF55F82400C168B94200D2C760BE
:1099C0008DF8018055F824000930019055F82400E5
:1099D0000169A9EB0100049055F82400406800EBF0
:1099E00006100068029055F82400C06801E03FE0CE
:1099F00021E04FF0010B03908DF800B055F82400E2
:109A000041680C2000EB06100958B1B16846884740
:109A1000824655F82400417A02290ED080F808B019
:109A200055F82400417A19B107E0C01BC860C1E7AE
:109A30000021817201E080F80AB0BAF1FF3F15D031
:109A400055F82410486800EB061213685246534537
:109A50000CD00978FBF76AF855F824100A7882428E
:109A600004D0887255F824100120087255F824009B
:109A70008069D7F70FFB641CE4B2044850F8280053
:109A8000C078A0427FF619AF27E7000000780120D8
:109A90008068002101707047A0B00446007A8DF8FC
:109AA0006C008DF86000E0681E90199060694FF0BE
:109AB00000084FF6FF751D901A90ADF820508DF8F4
:109AC0000080216918A888470DF1200B4FF0040A87
:109AD000A9460120D7F79AF9B8F1000F09D1202241
:109AE00068466169D6F763FE18B100208DF8000062
:109AF00002E0216918A888476169087800285BD0CE
:109B000020226846D6F7D2FD6846D6F731FE4FF0E0
:109B10000008BDF8201087B24945454646461CD08E
:109B200041E0A0693A46405DB84200D2024605EBEA
:109B3000850361680AEBC30008446946D6F737FE1F
:109B400048B92BF81650761CB6B24FF00108202EFB
:109B500001D22BF816906D1CADB22078A842E0D847
:109B60002FE02178884202D3ADF820901FE0A16950
:109B70003A46095CB94200D20A4600EB80036168AC
:109B80000AEBC30008446946D6F711FE38B93BF822
:109B900015102BF81610761C4FF00108B6B26D1C8C
:109BA000ADB2202D03D23BF815004845D9D1202E67
:109BB00007D22BF8169004E000208DF80000ADF8D5
:109BC0002090BDF820002178884229D2BDF82210CB
:109BD0004D46A94224D1A16900EB80030A5C61686B
:109BE0000AEBC30008446946D6F7E1FD00287FF47C
:109BF00070AFBDF82010242201EB8101606802EBF8
:109C0000C102835833B150F831001C90606881580C
:109C10001BA8884700208DF80000ADF8205058E7B9
:109C20006846D6F7A5FD202802D0B8F1000FF6D17E
:109C3000ADF820904DE7000038B504461123414AA5
:109C4000072108200094FAF7F1FA3E4A0623103261
:109C5000072108200094FAF7E9FA0D233A4A052172
:109C600008200094FAF7E2FA374A0523D032194661
:109C700008200094FAF7DAFA0723344A052108206D
:109C80000094FAF7D3FA314A0323703205210820F1
:109C90000094FAF7CBFA2D4A0323A03205210820BD
:109CA0000094FAF7C3FA294A0423D0320521082088
:109CB0000094FAF7BBFA0423254A052108200094F2
:109CC000FAF7B4FA224A042340320521082000940E
:109CD000FAF7ACFA1E4A04238032052108200094CA
:109CE000FAF7A4FA1A4A0423C03205210820009486
:109CF000FAF79CFA0423174A052108200094FAF782
:109D000095FA144A04234032052108200094FAF7FA
:109D10008DFA104A04238032052108200094FAF7B6
:109D200085FA0C4A0423C032052108200094FAF772
:109D30007DFA0323084A022108200094FAF776FAF4
:109D400038BD00009C080120300F030850100308A4
:109D50006011030860120308601303080B46112208
:109D600002494FF0E160FBF70FBC000058090308FF
:109D700038B504460C230B4A072108200094FAF753
:109D800055FA084A06231032072108200094FAF7F2
:109D90004DFA1323044A052108200094FAF746FAE5
:109DA00038BD0000FC080120242E03082DE9F34FE4
:109DB00097B00D4600274FF47A60D7F727F82A4668
:109DC00002215848F8F72FFF00287DD0482101A82C
:109DD000D6F7D9FD544C2A4601A92046F9F7F0FDE3
:109DE0002A460DF104080DF10501A01CF9F7E8FD64
:109DF000DFF8389108F101014846179AF9F7E0FDBC
:109E000009F1010A08F101015046179AF9F7D8FD46
:109E100008F1010109F10200179AF9F7D1FD09F1E2
:109E2000030B08F101015846179AF9F7C9FD3D489F
:109E30002A464FF480312730F9F704FC39482A4686
:109E40003B492630F9F7FEFB4FF084762946304631
:109E500002F06AFC03285DD14FF47A70D6F7D6FF82
:109E600030482A4601212830F8F72EFF294630468F
:109E700002F05AFC03284DD12A4601A92046F7F7E3
:109E800007FD002500263FE0C5EBC50000EB0804F8
:109E9000611C13A8F7F7DCFF042226A113A8D6F74C
:109EA00017FC58B1042225A113A8D6F711FC28B13C
:109EB000042224A113A8D6F70BFC18BB01273046B7
:109EC000761CF6B2012800E029E009D002280DD066
:109ED000032812D0611C4846179AF9F771FD11E06A
:109EE000611C5046179AF9F76BFD0BE00F48611C97
:109EF000801C179AF9F764FD04E0611C5846179A14
:109F0000F9F75EFD6D1CEDB29DF80400A84201D981
:109F1000042EB9D31FB1012019B0BDE8F08F002085
:109F2000FAE700005F0008003A000810190000106E
:109F300040F8030031303532000000003130343257
:109F4000000000003130333200000000F8B50E464A
:109F50001E4D144608218DF8001055F82410C0F34A
:109F600007424978914201D00A20F8BD010E01292B
:109F700003D0022913D00620F8BD80B22146FAF79B
:109F800097FC55F8241080B2C9680989814211D024
:109F9000C1B26B4632462046FAF76EFD12E080B23F
:109FA0002146FAF765FE55F8241080B2096909893F
:109FB000814201D10B20F8BDC1B26B46324620462A
:109FC000FBF772F89DF80000F8BD00000078012052
:109FD0001FB5D6F757FF4FF0010BDFF8B0914FF0E8
:109FE000000A0390D6F74EFF0399401A142801D3B4
:109FF000012001E0C0F11400D6F708FFD6F742FFB8
:10A000000026039059F82600002837D04068002821
:10A0100034D0D0E90074C0683146FAF7E1FB207112
:10A0200059F82600314640680069FAF7D9FB60719B
:10A0300059F82600314640684069FAF7D1FBA07113
:10A0400059F82600314640688069FAF7C9FBE0718B
:10A05000617AA1B101292168227907EB01110B79FD
:10A0600033D09A4279D162794B799A4275D1A279EB
:10A070008B799A4271D1C97988427FD180E059F8B1
:10A080002610002549680A891CE007EB0511237991
:10A0900091F804C0634513D1637991F805C0634515
:10A0A0000ED1A37991F806C0634509D1C9798842D8
:10A0B00006D1256084F809B0D6F7E4FEE0605FE0E1
:10A0C0006D1CEDB2AA42E0D85AE09A4256D16279AC
:10A0D0004B799A4252D1A2798B799A424ED1C97961
:10A0E00088424BD1D6F7CEFEE168401A216807EBD3
:10A0F00001110989884243D307EB05108DF80060F0
:10A100000168019107218DF80810C1684FF000081F
:10A1100011B16846884780462078401CC5B259F87E
:10A120002600406801891BE007EB051022790379BE
:10A130009A4213D1627943799A420FD1A2798379F5
:10A140009A420BD1E279C079824207D1256084F826
:10A1500009B0D6F797FEE06004E00FE06D1CEDB2A9
:10A16000A942E1D859F8260040680089A84207D1E1
:10A17000B8F1010F02D00220607201E084F809A05A
:10A18000761CF6B2202EFFF43DAF2BE7807801203D
:10A190002DE9F04780466D488A466D4E4178089C0F
:10A1A0001D4617464FF0000949B180F80190494615
:10A1B000002046F82010401CC0B22028F9D3202CE3
:10A1C00002D30220BDE8F08756F8240020B1417880
:10A1D000414516D00520F5E710210120D9F7F4FFFD
:10A1E00046F8240000287DD0047056F8241081F829
:10A1F000018056F82410C1F8049056F82410C1F8D4
:10A2000008905FEA0A0008D005F0FF08012843D053
:10A21000BAF1020F76D00320D4E756F82400406844
:10A22000002873D11C210120D9F7CEFF56F8241045
:10A230000028486056D0076056F824001021406876
:10A2400005812846D9F7C0FF56F824100028496830
:10A25000486079D000200922494608E056F82430A9
:10A2600002EB0017401C5B68C0B25B68D955A8427E
:10A27000F4D356F824104FF0FF304968C86056F800
:10A2800024104968086156F824104968486156F856
:10A2900024104968886155E056F82400806880BB26
:10A2A00014210120D9F790FF56F824108860C8B116
:10A2B000476056F824102846896881F800800121FB
:10A2C000D9F782FF56F824108968C86050B1082178
:10A2D0002846D9F779FF56F824108968886008B1B4
:10A2E000002001E030E00DE0494607E056F8242068
:10A2F0009268926802F83010401CC0B2A842F5D3B0
:10A3000020E003E056F82400C06808B10A2059E7AD
:10A310000C210120D9F758FF56F82410C86098B1D5
:10A32000476056F824102846C96881F80080022149
:10A33000D9F74AFF56F82410C968886020B1204632
:10A3400001F0ACF800203DE709203BE7E5050120DE
:10A35000807801202DE9F04F87B004461021227843
:10A360009048F8F7B1FC207A00287DD16068A0F110
:10A3700084711B3904D0A0F184711C390AD012E019
:10A380004FF0030887482178401DF8F743FC054645
:10A39000062708E04FF0040882482178801DF8F76E
:10A3A00039FC05460727424606A90D20F7F770FA43
:10A3B0007C489DF8182040214630F8F785FC42463D
:10A3C00001212320F9F73EF9424601210A20F8F73E
:10A3D0002AFCA8B1424600210A20F9F733F9724E4F
:10A3E000227804A93046F7F753FA9DF8140040F09C
:10A3F00004008DF81400227804A93046F9F7E0FA39
:10A40000DFF8A091227809F12B09FF214846F9F7DE
:10A4100019F9207804F03EFC424604210B20F8F79D
:10A4200053FC22780121A9F10300F8F74DFC2278B2
:10A430000121A9F10200F8F747FC5A4821781030B1
:10A44000F8F7E8FB06468DF80C708DF80450564F6F
:10A4500022783F1F01A93846F9F7B2FA8DF8046057
:10A46000227801A9384600E052E0F9F7A9FADFF8AE
:10A4700034A122780AF13B0A45EA06215046F9F751
:10A48000E1F821789DF8180005F06AF883462278F3
:10A4900000215046F9F7D6F84FF0010ABBF1010F41
:10A4A0003FD08DF80CA08DF80450227801A93846D1
:10A4B000F9F786FA424600210A20F9F7C3F8227814
:10A4C000FF214846F9F7BEF88DF80CA08DF804601E
:10A4D000227801A93846F9F773FA32482278002128
:10A4E0002830F9F7AFF82F48227800212930F9F702
:10A4F000A9F8227810212B48F8F70EF929489DF881
:10A50000182040214630F8F707F9207804F0DAFBEC
:10A51000227810212348F8F7FFF807B00220BDE8A1
:10A52000F08F02208DF80C008DF80450227801A9DC
:10A530003846F9F745FA424601210A20F9F782F830
:10A54000227841464846F9F77DF89DF818104046B4
:10A55000FFF72CFC01280AD0424600212320F9F7FE
:10A5600071F8424600210E20F9F76CF8ACE742463C
:10A5700001212320F9F766F842464FF400510B20E1
:10A58000F8F7A2FB074D9DF818206E35602128468C
:10A59000F8F79AFB9DF8182080212846F8F794FBDD
:10A5A000DFE70000190008001D0008103EB50D4649
:10A5B0008DF8080029461848F8F72CFB8DF80000A4
:10A5C000164C2A4669462046F9F7FAF912482946F8
:10A5D000401CF8F71FFB8DF800002A46694620460C
:10A5E000F9F7EEF90C482946801CF8F713FB8DF8B3
:10A5F00000002A4669462046F9F7E2F9064829464E
:10A60000C01CF8F707FB8DF800002A466946204673
:10A61000F9F7D6F93EBD0000200008001900081027
:10A6200038B5044621460420FFF7C0FF224669469C
:10A630001748F7F72DF916482146401CF8F7EAFAB3
:10A6400000990843009012482146801CF8F7E2FA6E
:10A650000099084300900E482146C01CF8F7DAFA2A
:10A660000099084300900A4D01460F3D22462846B6
:10A67000F8F72AFB4FF4FA60D6F7C8FB22462846C3
:10A680000099F8F749F821460120FFF78FFF38BD00
:10A690002C0008007047000070B50C4615462A468D
:10A6A00018210948F8F7BFFA00280CD12CB1294627
:10A6B000BDE870401020FFF779BF2946BDE8704023
:10A6C0000F20FFF773BF70BD180008007CB504466B
:10A6D0000025227802211D48F8F7F6FA207A90BB6F
:10A6E0001A4E2278523669463046F7F73BF92278FF
:10A6F00001A93046F7F7CCF86068A0F184711E39E3
:10A7000004D0A0F184711F390AD00FE09DF8040035
:10A710009DF80010884209D2401C0190012505E0F7
:10A720009DF8040010B1401E019001255DB1227812
:10A7300001A93046F9F744F9042804D121789DF89D
:10A74000040004F08BFE03207CBD0000190008000B
:10A7500070B50546007A0E46002410B1012802D0DB
:10A7600015E0E86803E01146E868F8F753FA297C39
:10A7700021B1012905D0022906D008E0864205D082
:10A7800005E0B04302D002E0064200D0012420469A
:10A7900070BD000070B50446022122781948F8F710
:10A7A00093FA207A40BB2078FFF73AFF154A606899
:10A7B0002B32154DA0F18471213908D0A0F184719C
:10A7C00022390FD0A0F18471203916D017E02178FA
:10A7D0001046F8F71FFA032811D103212846F6F78F
:10A7E00013FB0CE021781046F8F714FA042806D180
:10A7F00004212846F6F708FB01E0D9F73BFF0220C9
:10A8000070BD0000190008000500000170B5044685
:10A810002D4D227802212846F8F756FA207A48BBB7
:10A82000294A60682B32294EA0F1847119390CD065
:10A83000A0F184711A3913D0A0F184711D391AD096
:10A84000A0F18471233923D03CE021781046F8F739
:10A85000E1F9032836D103213046F6F7D5FA31E085
:10A8600021781046F8F7D6F904282BD10421304678
:10A87000F6F7CAFA26E000210120D9F775FF227801
:10A8800010212846F8F720FA2078FFF7C9FE19E0D2
:10A89000032201210A20F8F7C6F998B90422012100
:10A8A0000A20F8F7C0F968B907482178103802F093
:10A8B000DFF901210846D9F757FF227810212846F1
:10A8C000F8F702FA022070BD190008000600000126
:10A8D0002DE9F04104462D482178F8F79BF9C6B2DE
:10A8E00031460A20F8F796F90546284822780221D1
:10A8F0002B38F8F7E9F9324601210A20F8F793F9E5
:10A9000090B1224B207A1C3B4FF0007770B1227837
:10A9100000211846FFF7C0FE324600213846FAF7FC
:10A92000BCFB0220BDE8F0810020FBE7227801217A
:10A930001846FFF7B1FE6068A0F1847118390BD09A
:10A9400005F0040005F01001084319D032464021FB
:10A950003846FAF7A2FBE4E7E806E2D532460821DA
:10A960000B20F8F760F90028DBD03246802138460A
:10A97000FAF793FB324608210B20F7F7CDFED0E71C
:10A98000324680213846FAF788FBCAE744000800BF
:10A990000446806886B000780590D6F773FA049074
:10A9A000A66894F800A04FF00108D6E9010B0390C7
:10A9B000F16840684FF0000908608BF8019041464B
:10A9C00023E0039BC1EBC102002003EB82020BE0FA
:10A9D000F368546853F82030A34203D10BEBC10352
:10A9E000587003E0401CC0B24045F1D340450AD145
:10A9F0000BEBC1035870F368526808F1010043F88B
:10AA0000282000F0FF08491CC9B205988142D8D31C
:10AA100004214046D9F7D8FB306128B94FF47A7445
:10AA20002046D6F7F3F9FBE7D6F72CFA0499401A3B
:10AA30000A2801D3012001E0C0F10A00D6F7E6F9A7
:10AA4000D6F720FA002404900AE03069524600EB61
:10AA50008401F06850F82400FAF7CCFB641CE4B2DF
:10AA60004445F2D3002795E00398C7EBC7010BEBF1
:10AA7000C70400EB8105207805282DD2DFE800F01F
:10AA800003123246670061783069524650F821104F
:10AA90002846FFF75DFE00287AD0D6F7F3F960600C
:10AAA00001201DE061680498401A698A88426FD3CA
:10AAB00061783069524650F821102846FFF748FE69
:10AAC000F0B3287D20B1012807D0022807D05DE02F
:10AAD000042020708DF808905AE0022000E0032046
:10AAE000207055E06178306950F8210038BB287D2E
:10AAF000012807D084F800908DF800A02868019004
:10AB0000012016E00420207001201DE061783069EA
:10AB1000524650F821102846FFF71AFE78B9287DD2
:10AB200002280ED084F800908DF800A028680190CB
:10AB300002208DF80800A96909B16846884727E016
:10AB400024E00420207002208DF8080020E08DF819
:10AB500000A028680190A96911B168468847207053
:10AB6000287D20B101280AD002280CD00EE02078E0
:10AB700003280DD002280BD0012807D108E0207847
:10AB8000032803D104E02078022801D084F8009043
:10AB90007F1CFFB205988742BFF446AF64E7000010
:10ABA0002DE9F041044625482178F8F733F8C7B27B
:10ABB0002248227802212B38F8F786F83A46BC2141
:10ABC0000A20F8F730F880B36068A0F1847110397A
:10ABD00031D11A48217A1E3846124FF40068F50325
:10ABE00079B122780021FFF757FD3A4631462846D1
:10ABF000FAF72EF839462620F8F70CF8022815D077
:10AC000019E022780121FFF747FD3A4631462846F0
:10AC1000FAF71EFA39462620F7F7FCFF02280AD178
:10AC20003A4641462846FAF713FA04E03A464146C6
:10AC30002846FAF70DF80320BDE8F081440008002B
:10AC40002DE9F04104462D482178F7F7E3FFC5B21E
:10AC50002A48227802212B38F8F736F82A461021A4
:10AC60000A20F7F7E0FF254E1B3EE8B1207A50B1ED
:10AC7000227800213046FFF70FFD2A4608210B20DD
:10AC8000F7F74AFD24E02A4608210B20F7F7CBFF0F
:10AC9000F0B9227801213046FFF7FEFC2A46082150
:10ACA0000B20F8F711F813E02A4608210A20F7F7DD
:10ACB000BAFF68B1207A4FF4006760B122780021B2
:10ACC0003046FFF7E9FC2A4639460B20F7F724FD0A
:10ACD0000220BDE8F0812A4639460B20F7F7A3FF92
:10ACE0000028F5D1227801213046FFF7D5FC2A460D
:10ACF00039460B20F7F7E8FFEAE7000044000800B8
:10AD00007CB50446022122780B48F7F7DDFF0B4D96
:10AD1000227869462846F6F7BBFD9DF80400010637
:10AD200008D440F080008DF8040022786946284657
:10AD3000F8F746FE00207CBD190008001D00081031
:10AD40002DE9F04F87B00446DFF8609222780221A7
:10AD50004846F7F7B9FF22780221A9F10100F7F779
:10AD600062FFE0B3924D227801A92846F6F790FDE4
:10AD70009DF80800010608D520F080008DF8080035
:10AD8000227801A92846F8F71BFE894F874DDFF886
:10AD90001C82DFF818B2DFF814A2606801263F1F9A
:10ADA0002D1D08F110080BF11E0B0AF12B0AB0F152
:10ADB000847F1CD06FF08471C84213D12178504633
:10ADC000F7F728FF04280DD0042201210A20F7F705
:10ADD0002AFF00287AD022780421504600E002E0C1
:10ADE000F8F730FCCDE0002007B0BDE8F08F217807
:10ADF0005046F7F70FFF0328F4D0032201210A2061
:10AE0000F7F711FF28B1227803215046F8F71AFC12
:10AE1000B7E02278FF215046F8F714FC207803F0C1
:10AE200039FF06208DF81400DFF880A121780AF19F
:10AE3000050A5046F7F7EEFE8DF80C00227803A9BC
:10AE40003846F8F7BDFD21784046F7F7E3FE8DF868
:10AE50000C00227803A93846F8F7B2FD534822784F
:10AE600006A91130F6F714FD21785846F7F7D2FEFF
:10AE7000069908430690014622782846F7F724FFF2
:10AE80004FF47A70D5F7C2FF227828460699F7F773
:10AE900043FC8DF8146021785046F7F7BBFE8DF81F
:10AEA0000C00227803A93846F8F78AFD217840463D
:10AEB000F7F7B0FE8DF80C00227803A93846F8F7B2
:10AEC0007FFD207803F0FEFE5BE0FFE72278FF21A4
:10AED0005046F8F7B7FB207803F0DCFE07208DF82A
:10AEE0001400DFF8C8A021780AF1060A5046F7F7E7
:10AEF00091FE8DF80C00227803A93846F8F760FD22
:10AF000021784046F7F786FE8DF80C00227803A9D9
:10AF10003846F8F755FD2548227806A91230F6F78D
:10AF2000B7FC21785846F7F775FE06990843069056
:10AF3000014622782846F7F7C7FE4FF47A70D5F716
:10AF400065FF227828460699F7F7E6FB8DF814602E
:10AF500021785046F7F75EFE8DF80C00227803A9A1
:10AF60003846F8F72DFD21784046F7F753FE8DF867
:10AF70000C00227803A93846F8F722FD207803F068
:10AF8000A1FE227810214846F7F74DFE40B100217E
:10AF90000846D9F7E9FB227810214846F7F7BCFBB1
:10AFA0004FF4FA70D5F732FF00201DE719000800B2
:10AFB0001D0008102DE9F041044637482178F7F7C5
:10AFC00029FEC6B23448227802212B38F7F77CFEDE
:10AFD0003246BC210A20F7F726FE18B32E4B6068D4
:10AFE0001D3BA0F184714FF00075113904D0A0F120
:10AFF0008471123933D040E0207A4FF480774FF4D7
:10B00000006880B1227800211846FFF745FB3246E0
:10B0100039462846F9F71CFE31462620F7F7FAFD97
:10B02000012816D029E0227801211846FFF734FBC9
:10B03000324639462846FAF70BF831462620F7F70C
:10B04000E9FD012819D1324641462846FAF700F8B1
:10B0500013E0324641462846F9F7FAFD0DE0207A22
:10B060004FF4007760B1227800211846FFF714FBF7
:10B07000324639462846F9F7EBFD0320BDE8F0815A
:10B08000227801211846FFF707FB32463946284649
:10B09000F9F7DEFFF1E700004400080070B5044650
:10B0A00034482178F7F7B6FDC5B23248227802213C
:10B0B0002B38F7F709FE2A4601210A20F7F7B3FDDE
:10B0C00078B360684FF00076A0F184710E3904D037
:10B0D000A0F184710F3925D032E0264B207A203B35
:10B0E00050B1227800211846FFF7D6FA2A461021DF
:10B0F0003046F9F7ADFD23E0227801211846FFF72D
:10B10000CBFA2A4610213046F9F7A2FF2A46082139
:10B110000B20F7F788FD20B12A4608210B20F7F70E
:10B12000FBFA0DE0134B207A1F3B58B12278002127
:10B130001846FFF7B1FA2A4620213046F9F788FD74
:10B14000032070BD227801211846FFF7A5FA2A4690
:10B1500020213046F9F77CFF2A4608210B20F7F71B
:10B1600062FD0028ECD02A4608210B20F7F7D4FA1C
:10B17000E6E70000440008002DE9F0410446864857
:10B180002178F7F747FDC7B28348227802212B3890
:10B19000F7F79AFD3A4601210A20F7F744FD90B1EE
:10B1A0007D4861682438A1F18471891E431C851C87
:10B1B000C61C4FF00078082977D2DFE801F0071DA0
:10B1C000354D65CAA8860020BDE8F081217A49B1D5
:10B1D00022780021FFF75EFA3A4604214046F9F74B
:10B1E00037FDD5E022780121FFF754FA3A460421D1
:10B1F0004046F9F72DFFCBE0207A50B122780021AC
:10B200001846FFF747FA3A4608214046F9F720FD6D
:10B21000BEE0227801211846FFF73CFA3A460821A1
:10B220004046F9F715FFB3E0207A50B122780021AB
:10B230002846FFF72FFA3A4602214046F9F708FD63
:10B24000A6E0227801212846FFF724FA3A46022197
:10B250004046F9F7FDFE9BE0207A50B122780021AC
:10B260003046FFF717FA3A4601214046F9F7F0FC5D
:10B270008EE0227801213046FFF70CFA3A46012190
:10B280004046F9F7E5FE83E0217A79B12278002182
:10B29000FFF700FA227800212846FFF7FBF93A462B
:10B2A00006214046F9F7D4FC72E073E022780121D0
:10B2B000FFF7F0F9227801212846FFF7EBF93A462B
:10B2C00006214046F9F7C4FE62E0207A78B1227880
:10B2D00000211846FFF7DEF9227800212846FFF703
:10B2E000D9F93A460A214046F9F7B2FC50E02278F3
:10B2F00001211846FFF7CEF9227801212846FFF7F1
:10B30000C9F93A460A214046F9F7A2FE40E0207A00
:10B3100078B1227800211846FFF7BCF92278002185
:10B320003046FFF7B7F93A4609214046F9F790FC55
:10B330002EE0227801211846FFF7ACF9227801218E
:10B340003046FFF7A7F93A4609214046F9F780FE53
:10B350001EE0217A71B122780021FFF79BF9227853
:10B3600000213046FFF796F93A4605214046F9F7A5
:10B370006FFC0DE022780121FFF78CF92278012182
:10B380003046FFF787F93A4605214046F9F760FE57
:10B39000032019E7002017E744000800F0B589B042
:10B3A00024216846D5F7EFFA4FF480600024104E50
:10B3B000104D0127059055F8240088B1406838B138
:10B3C000307828B937706A4600210B48D6F77EFBE3
:10B3D00055F82410886818B16A460848D6F776FBF5
:10B3E000641CE4B2202CE6D309B00020F0BD0000BC
:10B3F000E505012080780120D19F020891A902086B
:10B4000008B509230090034A02210020FEF7C0FE80
:10B4100008BD00004C39030830B504460020084B35
:10B42000014653F821202AB1D5681DB11278225463
:10B43000401CC0B2491CC9B22029F2D330BD000063
:10B4400080780120F0B507461348002250F821000B
:10B450001146C4682378D4E901569C4602EB530098
:10B4600036F81040C4EBC40435F82440A4B2BC4202
:10B4700001D9034601E00DD20246A3EB020000EB26
:10B48000D07001F1010102EB6000C9B280B2102955
:10B49000E6D96046F0BD0000807801202DE9F04734
:10B4A00020494FF6FF7A534651F82000C068D0E992
:10B4B000012C067800200AE0C0EBC00152F82110F0
:10B4C0008CB29C4201D28BB20546401C80B2B04285
:10B4D000F2D3ACF80050012020E0002157460CEBDD
:10B4E000400815E038F8024CC1EBC103C4EBC404BA
:10B4F00052F8239032F824401FFA89F3A4B2A342F1
:10B5000004D9BB4202D21FFA89F70D46491C89B201
:10B51000B142E7D32CF81050401C80B2B042DCD3CB
:10B52000BDE8F087807801202DE9FC5F0D46424997
:10B530000446002651F82500B146002879D0C0689D
:10B54000002876D0002020706070A070E07051F864
:10B55000250006268A46C06890F800B0002060E00A
:10B560005AF82520C8EBC8071821D06801EB8701DD
:10B5700043685B5863B18DF80050406850F827006D
:10B580000190D06840684158684688470D2845D0EA
:10B590005AF8251009F101001FFA80F9C9685046D0
:10B5A000496851F82710090EA1555AF82520761C34
:10B5B000B1B2D268526852F82720120C625450F887
:10B5C0002520491C89B2D268526832F82720120A15
:10B5D000625450F82520491C89B2D268526812F88A
:10B5E000272062545AF82500491C8EB2C068416871
:10B5F000042000EB870008582946F8F715F90700E2
:10B600000CD0A0193946D5F78FF83846D5F7B0F8E1
:10B61000304480B200212154401C86B208F1010060
:10B6200080B2804658459BD34FEA1920207184F898
:10B6300005903046BDE8FC9F8078012010B5017868
:10B640002320F7F7E7FA08B10F2010BD0D2010BD39
:10B6500010B501782320F7F7DDFA08B10D2010BDF1
:10B660000F2010BD2DE9F0470C4688B0924600250A
:10B6700080B21146FFF7E6FE7D4980B251F82A10EC
:10B68000C9680A78824250D98A6849680A2532F81E
:10B690001000C0EBC00001EB800651463068000E80
:10B6A00020703068000C60703088000AA07030781C
:10B6B000E070307A2071707A6071B07AA071B089D0
:10B6C000000AE071307B2072B07B60723069F8F75D
:10B6D000ABF807004FF000080DD004F10A0039461E
:10B6E000D5F722F83846D5F743F80A3080B204F887
:10B6F0000080401C85B2B07A20B1012816D0022803
:10B7000013D16BE07069000E60556D1C7169A8B2B1
:10B71000090C2154401CB18A80B2090A2154401CF2
:10B7200080B2317D2154401C85B29DE0524604A96F
:10B730007069F6F7ADF80498000E60556D1C049919
:10B74000A8B2090C2154401C049980B2090A215462
:10B75000401C80B204992154401C80B29DF8141002
:10B760002154401C85B2002633E00698112150F880
:10B770002600B1EB106F0AD15146F8F755F80700D3
:10B7800025D060193946D4F7CFFF384617E010218D
:10B79000B1EB106F1BD15146F6F700F8C7B206980F
:10B7A0006119894650F826005246F6F771F82FB114
:10B7B000E81985B2611901F8018C08E04846D4F710
:10B7C000D7FF284480B204F80080401C85B2761C64
:10B7D000F6B29DF81400B042C7D845E0524669461B
:10B7E0007069F6F755F80098E946000E60556D1C33
:10B7F0000099A8B2090C2154401C009980B2090A92
:10B800002154401C80B200992154401C019980B2FF
:10B81000090E2154401C019980B2090C2154401C8E
:10B82000019980B2090A2154401C80B20199215427
:10B83000401C85B2002609EB860051468068F7F768
:10B84000F3FF07000CD060193946D4F76DFF384676
:10B85000D4F78EFF284480B204F80080401C85B2E3
:10B86000761CF6B2022EE6D308B02846BDE8F08773
:10B870008078012038B504461F23074A012108209B
:10B880000094FEF785FC2823044A02210820009436
:10B89000FEF77EFC38BD000040180308A41B030817
:10B8A00070B505460020024640F2FF34074E09E01D
:10B8B000AB5C83EA9003DBB204EA002036F8133075
:10B8C0005840521C8A42F3D3604070BD34F60208DF
:10B8D0002DE9F05FDFF82CA280468B4F9AF8030029
:10B8E0000A9C1E4691468B46002570B18AF803508B
:10B8F000002047F82050401C80B22028F9D3814A0C
:10B900003832111D101FD8F7E7FC202C02D301207C
:10B91000BDE8F09F57F8240020B10178414511D0CF
:10B920000420F5E70C210120D8F74EFC47F824004D
:10B9300000287CD080F8008057F82400456057F834
:10B94000240085605FEA0B004FF0040B03D0012850
:10B9500052D00220DCE757F82400406878BB0C2165
:10B960000120D8F731FC57F82410002848605ED039
:10B97000C0F8009057F8240008214068068130463E
:10B98000D8F722FC57F824100028496848604ED0A8
:10B99000002059460EE057F8242001EBC0035268FE
:10B9A000526842F8305057F82420401C80B2526848
:10B9B0005268D550B042EED30025564615E01FE040
:10B9C0000068214650F83500F5F7E8FEF188884216
:10B9D00009D957F8240021464068006850F835001E
:10B9E000F5F7DCFEF0806D1CADB257F8240040681E
:10B9F0000189A942E4D87EE057F82400806808B1A4
:10BA0000072085E70C210120D8F7DEFB57F824102A
:10BA10008860E8B34946016057F82400B9463D46BE
:10BA20008068182106813046D8F7CEFB00E030E070
:10BA300055F824108968486058B3002559E0D8F7B4
:10BA400049FC59F82410142789684B6805EB450117
:10BA500007EBC107D85159F824309B685F68C0B123
:10BA6000DAF8140047F8310059F824000BEB810292
:10BA7000DAF8388080680768BF58B7FBF8F7D0F865
:10BA800004800BEBC10048F8007059F824C001E0B5
:10BA900031E034E0DCF808C0DAF83830DCF8008057
:10BAA00058F80220B2FBF3F803FB18221AB1DCF8B5
:10BAB00004207F1C175059F82420DAF838C0926807
:10BAC00053681F5807FB0CF74FF0080C0CEBC10133
:10BAD0005F5059F82410896849680958DAF8140049
:10BAE0000844DAF83C10884207D26D1CADB2CAF89F
:10BAF0001400B542A3D300200AE70B2008E7062074
:10BB000006E70000EC0501208079012070B51A4E8F
:10BB10001A4D8AB0002456F8240018B3406808B3C0
:10BB2000A878F8B90120A870E88881074FEA90004A
:10BB300000D0401CA8810421D8F746FB686204218C
:10BB4000A889D8F741FBA86298B124216846D4F7A8
:10BB50001AFF4FF4007005906A4600210848D5F797
:10BB6000B5FF2863641CE4B2202CD4D300200AB0B3
:10BB700070BD0620FBE7000080790120EC05012064
:10BB80000DBE020808B5002100900923024A0846AC
:10BB9000FFF79EFE08BD0000483C030870B5164D37
:10BBA00051B12A460129128900EBC20406D00229AC
:10BBB00006D003291AD105E0044604E0183C02E04F
:10BBC000103C00E0083C204600F018F801462068D0
:10BBD000C0F30902914209D12A89C0F38F21914211
:10BBE00004D1002802DB10F0F84F01D0082070BD0E
:10BBF00060682861002070BDEC0501201CB5D0E90B
:10BC000000106FF30901CDE9001008216846FFF725
:10BC100047FE1CBD02490A6B0260087870470000AD
:10BC2000EC05012004498969884201D1002000E027
:10BC30000120D8F785BB0000EC050120034608462B
:10BC4000084910B50C8909E003EBC001D1E90021D6
:10BC5000D24372EA010203D0401C80B2A042F3D367
:10BC600010BD0000EC0501202DE9F05F0024054621
:10BC700000684FF001082646A3462746A146002843
:10BC800078DBDFF8F4A0410064D5B8F1010F14D0DF
:10BC90004FF00108012CC0F383614FD9B14269D143
:10BCA000810CC0F38352090701EB0251C0F38720D6
:10BCB00001EB002149455DD113E04FF00008012C54
:10BCC0004AD9C0F38361B14254D1C0F38341C0F378
:10BCD0008352090601EB0241C0F387200844B842B1
:10BCE00048D1DAF82800696840F82410641C083547
:10BCF000E4B2D5E90001C04370EA01000AD0284649
:10BD0000FFF77CFF01462868C0F30902914231D158
:10BD10000028B8DB49EA07004BEA0601CAF82C0004
:10BD20008AF80410F5F73AFD81074FEA900000D039
:10BD3000401CA0421ED12046BDE8F09F8B46810CDE
:10BD4000C0F38352090701EB0251C0F3872001EBD6
:10BD50000029C6E7002CB4D1C0F38341C0F383525D
:10BD6000C0F38366090601EB0241C0F387200F1878
:10BD7000B7E7FFE70020DFE7EC05012070B5224DB3
:10BD8000044600212A8909E004EBC100D0E9003013
:10BD9000DB4373EA000303D1491C89B29142F3D318
:10BDA000914201D1012070BD00212046FFF7F6FE2F
:10BDB00008BB01212A8909E004EBC100D0E9003069
:10BDC000DB4373EA000303D1491C89B29142F3D3E8
:10BDD000914201D1022070BD03212046FFF7DEFE13
:10BDE00058B102212046FFF7D9FE40B1012120467B
:10BDF000FFF7D4FE28B1002070BD052070BD0420DF
:10BE000070BD032070BD0000EC050120FE4A86B025
:10BE100002F11401081FD8F77BFAFB4C083CA0691B
:10BE2000FFF7ACFF4FF0000B059003282DD0E06921
:10BE3000FFF7A4FF0490032829D00598042824D0F4
:10BE40000498042823D0059805281ED004980528B6
:10BE50001DD00220C4F820B0607001202070142092
:10BE6000D4F7D4FFDFF8A0A3AAF1080A9AF80100DA
:10BE700001280FD002287BD003284CD0042878D08A
:10BE80004FF47A70D4F7C2FFE9E7A06900E0E069F7
:10BE90002062E4E70124564627E07481306A00EB13
:10BEA000C405D5E90001C04370EA010020D028464E
:10BEB000FFF7A4FE2988C1F30901884213D128465F
:10BEC000FFF7D2FE10F0FF000DD02044401E84B2D8
:10BED00032792946F06A00F0B7F920B9D6E90A109C
:10BEE0003279F7F76DFD641CA4B230898442D4D353
:10BEF000B169306A884208D1059807E0022000E065
:10BF00000320707001203070A9E704980428F5D050
:10BF10000528F5D1F2E70025BC4F57F82500002889
:10BF200048D04068002845D01420D4F76FFF57F858
:10BF3000250000244068D0E900967DE00220D4F777
:10BF400065FF59F834002946CAF82C00F5F726FC9D
:10BF500007462A46DAF82410DAF82C00F5F798FCA0
:10BF600006EBC408D8F8040020B1FFF77DFE08E016
:10BF7000ABE06FE0DAF82410DAF828000968C9436A
:10BF80000160DAE909103A46D4F7A2FBE8B3B80732
:10BF90004FEA970000D0401CBAF80A10574600FA42
:10BFA00081F1BAF80800C01E00B2401A03D504217E
:10BFB0008AF8011048E009EBC400416869B18DF8C6
:10BFC0000050F96A01918DF80CB056F834100291C6
:10BFD00041686846884701282CD17889396ABA4671
:10BFE00001EBC000294600F071F910F0FF070DD0F9
:10BFF000D4F748FF46F83400BAF80A00DAF82010FF
:10C0000001EBC001C8F8041002E013E0C8F804B066
:10C01000BAF80A10394489B2AAF80A10DAF82000EE
:10C0200000EBC102D2E90032DB4373EA020301D024
:10C03000FFF704FE641CA4B2744850F82500406861
:10C040000089A0423FF67AAF6D1CEDB2202DFFF4BF
:10C0500063AF04E7DAF82010DAF81800544681429A
:10C0600004D1D0E90023C4E9102304E0E269D2E955
:10C070000032C4E91032644D3835D5E90023D2438B
:10C0800072EA030218D08142686800D1401C206126
:10C0900068605D483830FFF7B1FD296860F3090139
:10C0A00029602189206A00EBC100574910383831D6
:10C0B00000F0F6F80220C2E02189286861F3992097
:10C0C00020F07C40C5E9000BE3E7DAF82010DAF84D
:10C0D00018005446814204D1E069FFF7A3FDE069EE
:10C0E00002E0FFF79FFDA0692062A0462546218956
:10C0F000454C3834206861F3992020F07C40206062
:10C10000286960602046FFF779FD216860F3090126
:10C1100021602146286A00F0C3F801206881DFF819
:10C12000ECA0002557465AF8250078B3406868B35C
:10C130001420D4F76BFE57F825000024BA46406857
:10C14000D0E9009653E00220D4F760FE59F834009D
:10C150002946C8F82C00F5F721FB07462A46D8F8EF
:10C160002410D8F82C00F5F793FBB8074FEA970096
:10C1700000D0401CB8F80A1000FA81F3B8F80800A3
:10C18000C01E00B2C01A02D588F801B035E0D8F858
:10C19000200000EBC100294600F098F810F0FF07DE
:10C1A0000DD0D4F76FFE46F83400B8F80A00D8F87E
:10C1B000201001EBC00006EBC401486003E006EB71
:10C1C000C401C1F804B0B8F80A10394489B2A8F81B
:10C1D0000A10D8F8200000EBC102D2E90032DB439C
:10C1E00073EA020301D0FFF729FD641CA4B25AF8D8
:10C1F000250040680089A042A5D86D1CEDB2202D15
:10C2000090D3444604E00000F40501208079012029
:10C21000B8F80810D8F8200000EBC1000949183818
:10C2200000F03EF8216AA069814200D1E0692189CD
:10C2300000EBC1000349083800F032F803206070B9
:10C240000DE600002C0601202DE9F041134E1546A5
:10C250000F4656F82510002449680A8919E00B6832
:10C2600053F83430834212D1D4F70CFE56F825101F
:10C270004968496841F8340056F82500042101EB6B
:10C28000C4014068406847500020BDE8F081641C4C
:10C29000E4B2A242E3D80320F7E70000807901204E
:10C2A000094AD369984207D29269801AC0F3CF0035
:10C2B0000A460146002005E0C01AC0F3CF000A4636
:10C2C00001460120D8F754B8EC0501202DE9FF47BD
:10C2D000424F04460D46F86A0299020F62F39541F7
:10C2E000020D62F39951020A62F391212A0962F365
:10C2F0009D610291012689014FF00008090E08D1C5
:10C30000029911F47F3F04D1029911F0705F00D1BE
:10C31000B0462946F5F742FA81074FEA900000D06F
:10C32000401C81462A46796AF86AF5F7B1FAF86A3C
:10C330000099020C60F3912162F399510091010E72
:10C34000009861F3954065F39D60002500903EE004
:10C35000B8F1000F16D000988DB140F00040009069
:10C36000786A50F8250001906846FFF747FC00996D
:10C3700060F30901204600910834694623E020F06B
:10C380004040ECE700982DB140F0004000905EB1D5
:10C390000026E5E720F0004040F080400090029841
:10C3A00040F040400290F2E7786A012650F82500FC
:10C3B000039002A8FFF722FC029960F309012046CE
:10C3C0000291083402A9FFF76BFF6D1CEDB24D45D9
:10C3D000BED304B02846BDE8F0870000EC0501207C
:10C3E00038B504460123074A194608200094FFF790
:10C3F0006FFA044A1123883A002108200094FFF7BD
:10C4000067FA38BDF020030808B503230090034AFB
:10C4100000210820FFF75CFA08BD0000C42F0308C4
:10C420002DE9F05F0546A9488A46A94E01780A9C85
:10C43000994617464FF0000849B180F80080414600
:10C44000002046F82010401C80B22028F9D3202C70
:10C4500002D30120BDE8F09F56F8240020B14078B7
:10C46000A84211D00220F5E70C210120D7F7ACFE3D
:10C4700046F8240000287DD0047056F8240045704A
:10C4800056F82410C1F804805FEA0A0009F0FF059D
:10C490004FF00C0B4FF0040A03D001286BD005209D
:10C4A000D8E756F82400406800287DD10C210120EF
:10C4B000D7F78AFE56F82410002848605AD0476003
:10C4C00056F824003421406805704846D7F77CFEB2
:10C4D00056F824100028496888604BD00027A1E056
:10C4E00056F8240007EB870303EBC705416807EB09
:10C4F00087004A68896802EB800241F8252056F8D7
:10C5000024100AEB8502496889688C5456F8241077
:10C5100049684A688B68082101EB850152F82020A0
:10C520005A5056F824100AEB800049684A68896816
:10C53000125C0BEB85000A5456F82410102202EB13
:10C5400085024968896841F8028001210022084675
:10C55000D5F74CFA56F824101C2202EB85024968E4
:10C5600089688850012100220846D5F73FFA56F81D
:10C57000241001E05AE05BE04968182202EB8502D2
:10C5800089688850012100220846D5F72FFA56F80D
:10C590002410202202EB850249688968885056F8E9
:10C5A00024104968896800E046E0142202EB850205
:10C5B00041F8028056F82410242202EB85024968D3
